:020000040000FA
:040000006FD00400B9
:101000006F00907E00000000000000009020002093
:10101000AA220020A9BDF9F56C23002000000000E1
:10102000000000006C230020902000200000000041
:101030000000000090200020000000009020002010
:101040000000000090200020902000209020002030
:101050009020002090200020582F00209424002071
:101060000000000090200020902000201E2400207E
:1010700090200020D22300209020002090200020EB
:101080009020002090200020902000209020002020
:101090009020002001A04111B7170040985F3AC688
:1010A000945F3247E39CE6FE3245410182800111A4
:1010B00013078008F337078093F787083EC20100C3
:1010C0000100B7170040930570052380B70413068D
:1010D00080FA2380C7040100010083C6B70493F699
:1010E000F60DA385D704238007049246F3A6068055
:1010F0000100010093760502D5CEF336078093F602
:10110000860836C4010001002380B7042380C70489
:1011100001000100B70614007D89558D88C70100C4
:1011200001000100010023800704A246F3A6068007
:101130000100010073370780137787083AC6010062
:1011400001002380B7042380C704010001000100CF
:1011500001003727004093061005A303D7802380A2
:101160000704B247F3A70780010001009307800836
:10117000F3B7078093F787083ECE01000100B71749
:101180000040130770052380E704130780FA2380CB
:10119000E7040100010003C7B70413670708A3852C
:1011A000E70423800704F247F3A70780010001004A
:1011B0000561828093760504BDC6F336078093F6F9
:1011C000860836C8010001002380B7042380C704C5
:1011D00001000100B7061400938606047D89558D31
:1011E00088C7010001000100010023800704C246F6
:1011F000F3A6068001000100733707801377870884
:101200003ACA010001002380B7042380C70401000B
:1012100001003727004093062005A303D7802380D1
:101220000704D24781B773370780137787083ACC12
:10123000010001002380B7042380C70401000100DE
:1012400098471367070C98C723800704E24719BF24
:101250000111814601468145114506CE97000000E7
:10126000E780605893078008F3B7078093F78708F3
:101270003EC601000100B717004013077005238028
:10128000E704130780FA2380E7040100010003C785
:101290006704136717002383E70423800704B2471A
:1012A000F3A7078001000100F2400561828041112F
:1012B000814601468145114597000000E780A05214
:1012C00013078008F337078093F787083EC40100AF
:1012D0000100B7170040130670052380C70493066A
:1012E00080FA2380D70401000100FD552396B70240
:1012F00023800704A245F3A5058001000100733790
:101300000780137787083AC6010001002380C704CD
:101310002380D7040100010003C767041367170087
:101320002383E70423800704B247F3A70780010063
:10133000010001A0BD473305F50201007D1575FDD3
:101340008280411122C426C206C6AA8401446317C2
:101350009400B24022449244410182800504130566
:10136000803E420497000000E78000FD4180C5B741
:101370009305000273A04580824573901534924016
:101380002242B2424243D2436244F2440255925551
:101390002256B2564257D2576258F25806499649D9
:1013A000264AB64A464BD64B664CF64C065D965DD1
:1013B000265EB65E465FD65F09617300203041113C
:1013C000B7170040985F3AC6945F3247E39CE6FE49
:1013D000324541018280B71700401307000323887C
:1013E000E702854717170000232EF74673002030C9
:1013F000411122C42D6426C24AC006C637190040D6
:101400001304A4AAB704002023208900977000E0E9
:10141000E780A0B59C408297977000E0E780E0B439
:10142000E5B737370040834747009146BD8B639E41
:10143000D702B73600401306F00F973500009385AA
:10144000651E9737000083D7E72D03C7A6001377E3
:10145000F70F1DE3B7E70400BC4F09468945171590
:1014600000000345A5F7829731A099466394D70001
:10147000834757007300203003C786001377F70FA8
:10148000E365F6FC13851700AE9717380000231BA1
:10149000A8282380E70075B7B787004003C7670017
:1014A000098B6309071003C77700930600031377BE
:1014B0000703630DD708173800000348F87717367D
:1014C0000000130666740547B30606012380E60094
:1014D00083C577001737000013070775429793F508
:1014E000F50F2300B70003C58700973500009385EB
:1014F000A572C2951375F50F2380A5000347070059
:1015000089451377F703630CB70C63E7E50A6306B5
:10151000071A8545630CB7129737000083C7D77148
:101520003307F600034707001377F70F19CB85073A
:1015300093F7F70F3D476363F71A17370000A30DC2
:10154000F76EB787004009472383E700B78700405D
:1015500083C77700E207E18763DE0704973700005F
:1015600083C7976D173700001307076A3E978546B4
:101570002300D700173700001307076B3E97930629
:1015800000032300D700173700001307E7683E97D2
:10159000A14685072300D70093F7F70F3D47636403
:1015A000F71417370000A309F768B7870040094709
:1015B0002383E70073002030930610026300D70EE8
:1015C000930620026305D70693060002E316D7F4BC
:1015D00003C727021377C70F13672700D5A803C7D0
:1015E00067001377070465CB03C7A702173800000D
:1015F00013080843173500001305453A1347070839
:101600002385E70203C7A7021377370F1367870005
:101610002385E702814713070004B305F5008C41D9
:10162000B306F80091078CC2E399E7FEF5B503C74E
:10163000A702134707042385E70203C7A70213770E
:10164000C70F136727002385E702F9B503C76700B3
:101650001377070449C303C767021738000013084C
:10166000E82F1735000013052527134707082383A4
:10167000E70203C767021377370F136787002383D7
:10168000E702814713070004B305F5008C41B30658
:10169000F80091078CC2E399E7FEBDBD03C767025E
:1016A000134707042383E70203C767021377C70FB3
:1016B000136727002383E70285B503C76700137705
:1016C000070411CB03C727021377370F136787006F
:1016D0002381E70291B5238006003DBD97370000C6
:1016E000A38C0754B9BD97370000A387075475BD75
:1016F0002303048015472303E48001002302A48010
:10170000828083076480E3CE07FE23030480828007
:1017100083076480E3CE07FE03454480828083070D
:101720006480E3CE07FE2302A4808280411126C498
:101730004AC24EC006C61377F50BAD47AA892E895B
:101740009544630CF700194597000000E78080FA84
:1017500097000000E78020FB8D444E859700000035
:10176000E78040F9FD59FD1463983401B240A2446A
:101770001249824941018280135509011375F50F01
:1017800097000000E780E0F92209F1BF011126CCA3
:1017900006CEB704080097000000E780C0F61545A4
:1017A00097000000E78000F597000000E78080F6D2
:1017B00097000000E78000F62AC697000000E78047
:1017C00080F432459377150089EB13651500137586
:1017D000F50FF240E24405618280FD14E9F0014515
:1017E000CDBF397126DC4ADA4ED852D656D45AD2F9
:1017F0005ED006DE62CE66CCB7E700E07D5783AAF6
:10180000070022C603AA470023A0E71823A2E7186F
:10181000B7170040130770052380E704130780FA09
:101820002380E70483C74704930B75FFB684E20760
:1018300093FBFB0F8546AA892E8B32893724004003
:10184000E187015763FA76016308D50089461307DB
:1018500000026313D5000157D98F93F7F70FB71C18
:1018600000402382FC0411472303E4801305F00F9A
:1018700097000000E78000E8094C97000000E7802F
:1018800080E863657C15B7050700DA9537870700A0
:10189000795563FEE504B3879500636AF704370B57
:1018A0000800A94733EB65016395F90881E8814495
:1018B00097000000E78020E5268515A8DA85094510
:1018C00097000000E780C0E605090345F9FFFD1415
:1018D000050B97000000E780C0E481C49377FB0FFD
:1018E000E5F797000000E780A0EA69F17D55B7179A
:1018F0000040130770052380E704130780FA238054
:10190000E70403C74704418B2382E704F250B7E79B
:1019100000E023A0571123A24711E2543244525948
:10192000C259325AA25A125B825B724CE24C21615C
:101930008280A547639BF90685691309F00FB306FA
:101940009900B3742B01B6941349F9FFB37499004D
:10195000856B33796901416B9387F9FFB3F72701F1
:1019600099E363FC340193D94900C147E3E637FFAB
:101970003DBF0569C1697D19D9B71305800D63881D
:101980006901130500026384790113051008CA85F3
:1019900097000000E780C0D997000000E78040DF93
:1019A00031D54E99B38434416DBFDA852D4597000A
:1019B0000000E780E0D7CA94E30B99EE0509970091
:1019C0000000E78020D5A30FA9FEFDB79387F9FF9C
:1019D00093F7F70F636DFC0C83C71C0413073008E3
:1019E0006315F706370708006361EB06B3079B0032
:1019F000B706100063FBD704334BEB0089476399AC
:101A0000F9068980D549E38404EADA850945970017
:101A10000000E780E0D111090327C9FF9147232087
:101A2000E48003076480E34E07FE23033481FD173F
:101A3000EDFBFD14110B81C49377FB0FE9FF9700B9
:101A40000000E780E0D461F155B5B717004003C747
:101A50005704B70708001377070219E3B787070091
:101A60007955E376FBE833079B00E3F9E7F841B5E6
:101A70008547E380F9F0DA852D4597000000E7807F
:101A800020CB9389F4FFE38404E297000000E78011
:101A900060C893F7390091EB83260480032709007F
:101AA00093074900E396E6E03E89CE84D9BFB54767
:101AB0006399F9001305900B97000000E78080C33D
:101AC000FDB3B1471305B00AE388F9FE9947639760
:101AD000F904B7050800B365BB002D459700000069
:101AE000E78000C581448D4BA14997000000E78045
:101AF00060C263967401832704802320F900850463
:101B0000E39534FF8327048013172B0163550700E7
:101B10002312F90069BB2322F90051BB9D47639F43
:101B2000F90281451305B00497000000E78040C02A
:101B3000BD442320090023220900FD59970000001D
:101B4000E78040BD93F77400CA9703C70700FD14F0
:101B5000398D2380A700E39334FF91BBA14763979E
:101B6000F90697000000E780A0C28144630D0B00D6
:101B70008D479304C0036308FB00930400056304CE
:101B80008B01930440041375C507E30295D21945F0
:101B900097000000E78000B697000000E780A0B63D
:101BA000054597000000E780E0B426859700000017
:101BB000E78020B7094597000000E78080B69700CE
:101BC0000000E780E0BCE31405CE0DB39147639FAE
:101BD000F9001305600697000000E780A0B19700A8
:101BE0000000E78040B213059009F9B5E38109CC04
:101BF000F1547DB9BD660147173600001306063063
:101C0000938606A685458347060093F7F70F91C391
:101C100082800507E3F9E6FE973700002380B72EA0
:101C2000DDB77D166206618693178601E18763D46E
:101C3000070001458280931726003307F500AE9711
:101C400018439C4363E7E7007D16E37FF7FC7D556F
:101C5000828005458280FD15E205E18513978501A7
:101C6000618793F7F50F63480700FD15139725006B
:101C70002A97584365D713851700620561858280CE
:101C80003308B5021C4283A80600B335B502C297DB
:101C900033B50701AE98469585486367B5006394F0
:101CA000A50063E3070181480C43C6950CC388C2B5
:101CB0001CC2828081471397870161876343B70005
:101CC0008280139727002A97232007008507E5B70E
:101CD0008147014793968701E18663C5B6001335B6
:101CE0001700828093962700AA9694428507558F05
:101CF000D5B793D755408A07AA979C430545331516
:101D0000B5007D8D828017F3FFDFE702833D2A84D3
:101D100097000000E78060F405C5931725003E9406
:101D20000327C4FF814711EB7D1516053E9542053B
:101D3000418517F3FFDF6700033D05838507E5B79E
:101D40000145C5BF81471397870161876343C7007A
:101D5000828013972700B386E50094422A9785076F
:101D600014C3D5B77D1662066186014793178601B5
:101D7000E18763D50700133517008280931726008B
:101D8000B306F500AE9794429C437D16B58F5D8FE8
:101D9000F1BF8A05AA9501476363B500828083A6D7
:101DA000C5FFF11593D71600D98F9CC11397F60183
:101DB000E5B72A830148014701456343D700828084
:101DC000B387050183A80700B30706019C43C697A4
:101DD000AA976384F80033B517010507B308030118
:101DE000620723A0F80061871108C1BF2A83014759
:101DF0008147014563C3D70082803388E50083288B
:101E00000800330EE600032E0E003388A840330886
:101E1000C8416384080133B508018507B308E300AE
:101E2000E20723A00801E1871107E9B717F3FFDFF5
:101E3000E702232B0111B286B2842E86AA850A8579
:101E400097000000E780C0FA2A84A6850A859700DB
:101E50000000E78020E833348000060413351500C5
:101E6000018D056117F3FFDF6700E32917F3FFDF3B
:101E7000E702A3244111AA89AE8A328BB68402C23A
:101E800002C402C60144131C8401135C8C416349E3
:101E90009C02939B1400FD1B0549138CF4FFF15C1D
:101EA00033048901620461846340740792478E049D
:101EB000CE9423AEF4FE410117F3FFDF67006323E6
:101EC00013192400B30B2B01014A93172A00D6974C
:101ED00083A50B0088437800340050009700000071
:101EE000E78040DA050A93178A01E187F11BE35E78
:101EF000FCFC92474E9905042320F900A2473EC2FC
:101F0000B24702C63EC441B7131A8901135A8A4127
:101F1000131D240093178A01E18763CF970092472E
:101F20000A044E941CC0A24705091379F90F3EC25A
:101F3000B24702C63EC4ADB7B3079A0313152A00D1
:101F400056950841780034005000050AEA97DA9760
:101F50008C4397000000E780E0D26DBF197106C284
:101F600012C416C61AC81ECA22CC26CE2AD02ED219
:101F700032D436D63AD83EDA42DC46DECAC0CEC2C9
:101F8000D2C4D6C6DAC8DECAE2CCE6CEEAD0EED2F9
:101F9000F2D4F6D6FAD8FEDA971500009385058CB0
:101FA0008841E700050092402242B2424243D243B8
:101FB0006244F244025592552256B2564257D257C5
:101FC0006258F25806499649264AB64A464BD64BBD
:101FD000664CF64C065D965D265EB65E465FD65F45
:101FE0000961730020300000972100209381810156
:101FF000175100201301018117F5FFFF1305C500DC
:102000009705002093850500171600201306C6FDCE
:1020100063FAC5008322050023A055001105910530
:10202000E3EAC5FE170502001305457B971500205E
:102030009385C5FB171600201306C66563FAC50015
:102040008322050023A0550011059105E3EAC5FE92
:102050001715002013050564974500209385053664
:102060006377B500232005001105E36DB5FEFD4241
:10207000739002BC8D4273904280B722000093821D
:10208000828873900230970200209382A2F793E235
:10209000320073905230975200009382A2C0739026
:1020A00012346FB0F47573002030397101436EC67D
:1020B00019A0397141536AC866CA62CC5ECE19A0B4
:1020C000397101535AD056D252D44ED64AD826DA54
:1020D00022DC06DE33016140828241114AC026C201
:1020E00022C406C68282B24D4101024D924C224C5E
:1020F000B24B4101024B924A224AB2494101024984
:1021000092442244B240410182803D432A87637356
:10211000C3029377F700BDEFADE5937606FF3D8AE6
:10212000BA960CC34CC30CC74CC74107E36BD7FE30
:1021300011E28280B306C3408A0697020000969699
:102140006780A6002307B700A306B7002306B700E1
:10215000A305B7002305B700A304B7002304B70005
:10216000A303B7002303B700A302B7002302B700FD
:10217000A301B7002301B700A300B7002300B700F5
:10218000828093F5F50F93968500D58D9396050182
:10219000D58D61B7939627009702000096968682A8
:1021A000E78086FA9680C1171D8F3E96E374C3F8C8
:1021B000A5B73367B500FD530D8B79E7B7877F7FF0
:1021C0009387F7F710419441B372F6003363F6003A
:1021D000BE92B3E262006397720C6318D606504158
:1021E000D441B372F6003363F600BE92B3E26200EC
:1021F0006398720A631BD60410459445B372F600C7
:102200003363F600BE92B3E262006391720A631E0A
:10221000D6025045D445B372F6003363F600BE9241
:10222000B3E26200639A72086311D60210499449BE
:10223000B372F6003363F600BE92B3E262006393BA
:1022400072085105D105E30FD6F6131706019397CF
:102250000601631CF7001357060193D706013305E7
:10226000F7409375F50F91E982804183C18333056F
:10227000F7409375F50F91E182801377F70F93F78D
:10228000F70F3305F74082800346050083C605003B
:10229000050585056313D60065FA3305D6408280AF
:1022A00011059105E312D6FE014582802105A105A5
:1022B000E31CD6FC014582803105B105E316D6FC4E
:1022C000014582804105C105E310D6FC01458280AD
:1022D000B717004003C777051377E70FA38BE70411
:1022E000130700F8A38DE7043D47238CE704130789
:1022F0005003A38CE70403C7A7051377D70F238DDB
:10230000E7048280B717004003C7E7020D89411137
:102310001377C70F498F93068008F3B6068093F6AC
:10232000860836C601000100930670052380D70495
:10233000930680FA2380D704010001002387E70277
:1023400023800704B247F3A7078001000100410181
:10235000828041112A83014E930E407E130F001993
:10236000930F400663E56E129308001913034006AD
:10237000B3781503854E0D4FA14F337365020D8958
:102380001335150063EFBE121308F6FF79467298F5
:102390004208135808013307C70213D61700BE07B7
:1023A00032976146B3F6C60213068070B386C60242
:1023B0003697A166F58F42075D8FB716004083C739
:1023C000F60293F70708A303F1000346710083C7E1
:1023D000F60293F70708E394C7FE83477100B71628
:1023E000004093F7F70F6388071293078008F3B74D
:1023F000078093F787083EC401000100B71700402B
:10240000930670052380D704930680FA2380D704AF
:102410000100010023AA070383C6170393E60608F9
:10242000A388D70223800704A247F3A707800100EF
:1024300001001166B71700407D16D45BC85F938515
:102440004703A98EF18EF5FA93068008F3B606804D
:1024500093F6860836C601000100930670052380B6
:10246000D704930680FA2380D7040100010098C1A5
:1024700003C7170313670704A388E7022380070431
:10248000B247F3A7078001000100410182807D135C
:102490003368E3039308E016630E08003368F30320
:1024A0009308D016630808009378330093B8180097
:1024B0009388D81633081E01131E0801135E0E01FF
:1024C00055B56393E5030548638608000148630337
:1024D00003002A8871087298FD15131E0801C205B1
:1024E000135E0E01C18179BD13F8150063F4BF00BE
:1024F0007908D5B713381800E5BF83C7F60293F7FC
:102500000708A303F1000346710083C7F60293F79F
:102510000708E394C7FE8347710093F7F70FF1DFD5
:10252000E9B531714AD966CB06DF22DD26DB4ED70D
:1025300052D556D35AD15ECF62CD6AC96EC7AA8C26
:1025400002D897100000E78020B12A8993078008FD
:10255000F3B7078093F787083EDA01000100B71749
:102560000040130770052380E704130780FA2380D7
:10257000E7040100010003C7F7021377770FA38771
:10258000E70203C7F70213678700A387E7022380E8
:102590000704D257F3A70780010001000545970003
:1025A0000000E78060D6130780C13347E902116A53
:1025B00093070AE893065002BD69930BA004814A71
:1025C000014B13048008930470057D1AB347F90288
:1025D0003307D7023EC0FD873ECC938709A69309F7
:1025E000803E3347F7023AC27D873AC43347390306
:1025F0008549B399990193D93940B306D702B30BF2
:102600007703B3C6F602B3CBFB0236C6FD8636C8E7
:1026100093D6FB4136CEB7460F0093860624334946
:10262000D9028566938606FAB3969601B389E902C4
:10263000130760553309D90293060010B389E902E4
:102640003349D902B3C9F9029316390036CA37198A
:102650000040FD8636D0930D090493D7F9413ED250
:10266000F336048093F6860836DC010001009307F8
:1026700070052380FD00930680FA2380DD000100B1
:1026800001008346390593F6860FA309D9048346D2
:10269000390593E61600A309D90423800D00E256FC
:1026A000F3A6068001000100130C80FA116DF336C9
:1026B000048093F6860836DE01000100930770055A
:1026C0002380FD0023808D01010001008346390530
:1026D000216693E60602A309D90483560905B3E6E9
:1026E000A6012318D90483560905D18E2318D904CD
:1026F00023800D00F256F3A60680010001008346F8
:10270000390593F606026381061A03463905218AC4
:102710006DDE081897100000E7800098733604807B
:1027200013768608B2C20100010023809D00238039
:102730008D0101000100B717004003C6370513766D
:10274000F60DA389C70403C6370513660602A389DD
:10275000C704835609052166B3E6A6012318D904E8
:1027600083560905D18E2318D90423800D0096467F
:10277000F3A60680010001008346390593F60602A0
:10278000638B061483463905A18AEDFE970000206D
:10279000E7806090AA8636D497000020E780A08F5B
:1027A000A256E30AD5FE835609054255B3E6A601B3
:1027B0002318D90497100000E780C08F834639059D
:1027C000A18AEDDE03560905834629058247337643
:1027D000CA00B306DA0293D5F641B296B388F64042
:1027E000E24733B8C6002E983308F840A247B3B684
:1027F00016013308D84063C70701631DF8009247EC
:1028000063FA1701C247634FF80E63950701B24799
:1028100063EAF80E894663E9660FF24693151800DD
:1028200013D3F8015E8613951800B365B30042D642
:1028300046D497C00100E78000553258050B137B42
:10284000FB0F63470001631A0838A25863870838F2
:1028500013081500B336A800B69513D6F5013298C3
:10286000B336C800AE9613581800FE06B3E606014C
:102870007336048013768608B2C6010001002380F7
:102880009D0023808D01010001000356C902B2960C
:10289000C206C1822316D90223800D00B646F3A6D4
:1028A00006800100010021B5F336048093F6860806
:1028B000B6C00100010023809D0023808D0101002E
:1028C00001008346390593E60602A309D904238053
:1028D0000D0086460DB5F336048093F68608B6C41F
:1028E0000100010023809D0023808D010100010073
:1028F0008346390593E60602A309D90423800D0017
:10290000A646BDB5E30B0BF0F336048093F68608BC
:10291000B6C801000100930680FA23809D00238041
:10292000DD00010001008346390593F5FC0F93F6A5
:10293000860FA309D90483463905CD8EA309D9048E
:1029400023800D00C646F3A6068001000100130592
:1029500080FA03463905930639051D8A631C9629BA
:102960007336048013768608B2CC0100010013068A
:1029700080FA23809D002380CD000100010003C662
:1029800006001376F60D2380C60003C60600136604
:1029900006022380C600835609051166D18E2318CE
:1029A000D904835609052166D18E2318D9042380C2
:1029B0000D00E646F3A6068001000100130680FA2A
:1029C0008346390593F60602638006268346390559
:1029D000130C3905A18AFDDA081897000000E7807A
:1029E000A06BF336048093F68608B6D00100010090
:1029F000930680FA23809D002380DD000100010002
:102A000083460C00116693F6F60D2300DC00834626
:102A10000C0093E606022300DC0083560905D18EE4
:102A20002318D904835609052166D18E2318D904A9
:102A300023800D008656F3A60680010001001306D0
:102A400080FA8346390593F60602638A0620834698
:102A50003905A18AEDFE97F0FF1FE780C0632A8C3D
:102A600097F0FF1FE7802063E30C85FF835609057D
:102A700011664255D18E2318D90497000000E780D3
:102A800060638346390513063905A18AFDDAF336FA
:102A9000048093F68608B6D401000100930680FAFC
:102AA00023809D002380DD00010001008346060095
:102AB00093F6F60D2300D60023800D00A656F3A64C
:102AC0000680010001008356090503462905D24707
:102AD000B376DA003306CA021305800C9355F6412B
:102AE0003696330DF6408257333CD6002E9C333653
:102AF000A601330CFC40330CCC40330885039256BE
:102B00004E86B335A5033305A503C29597C00100D2
:102B1000E780602763468001631E0C16630C0D1668
:102B2000130615003335A6002E959356F5013696FB
:102B3000B335D600AA959396F50105828585D18E89
:102B40006346B000639D051A638B061A0356C902DB
:102B500015823305D6003336C500B2956348B00000
:102B6000639105241306F00F637DA622894663F363
:102B7000561593078008F3B7078093F78708BED6EA
:102B80000100010037170040930770052300F70488
:102B9000930780FA2300F704010001008356C7025F
:102BA00089678117D58FC207C1832316F7022300D7
:102BB0000704B657F3A7078001000100FA506A54D2
:102BC000DA544A59BA592A5A9A5A0A5BFA4B6A4C49
:102BD000DA4C4A4DBA4D296182801308F5FF33352E
:102BE000A800FD152E951356F5013298B336C8008E
:102BF000AA9695B9F336048093F68608B6CA010002
:102C0000010023809D002380AD0001000100834668
:102C10003905CD8EA309D90423800D00D646F3A62D
:102C200006800100010035B3F336048093F6860870
:102C3000B6CE0100010023809D002380CD0001005D
:102C400001008346390593E60602A309D9042380CF
:102C50000D00F646F3A606800100010095B3F33699
:102C6000048093F68608B6D20100010023809D00FF
:102C70002380CD00010001008346390593E606025A
:102C8000A309D90423800D009656F3A606800100FF
:102C9000010045BB9306F5FF33B5A600FD152E9543
:102CA0009355F501AE96B3B5B600AA951396F50106
:102CB000858269B5F336048093F68608B6D801009C
:102CC0000100930680FA23809D002380DD0001002F
:102CD00001008356C9020566011693F6F60FD18EE0
:102CE000C206C1822316D90223800D00C656F3A660
:102CF000068001000100850A93FAFA0F95B233E6C7
:102D0000B60045C20356C9023305D0403338A0008F
:102D1000B305B040B385054115826345B000D1E1EC
:102D20006371A608894663F0560593078008F3B7D8
:102D3000078093F78708BEDA01000100B71700404B
:102D4000130770052380E704130780FA2380E70444
:102D50000100010003D7C7027D8B2396E702238081
:102D60000704D65781BDF336048093F68608B6DC97
:102D700001000100930680FA23809D002380DD007E
:102D8000010001008356C9020566011693F6F60F8D
:102D9000D18EC206C1822316D90223800D00E656C9
:102DA000B9B793078008F3B7078093F78708BEDEAB
:102DB0000100010037170040930770052300F70456
:102DC000930780FA2300F704010001000356C702AD
:102DD00093975600B297C207C1832316F7022300C8
:102DE0000704F657C1BB914763EEB70217E701002E
:102DF0001307C7978A05BA959C41BA978287B71778
:102E0000004003A7470B1345F5FF698F23AAE70A84
:102E100003A7070B698F23A8E70A03A7070A798D81
:102E200023A0A70A8280B717004083A6470B134749
:102E3000F5FFF98E23AAD70A83A6070B558D23A881
:102E4000A70A83A6070A758F23A0E70A8280B7170F
:102E5000004003A7470B498F23AAE70A03A7070BE4
:102E60001345F5FF45BFB717004083A6470B13472F
:102E7000F5FF758F23AAE70A03A7070A598D4DB7F7
:102E8000B717004003A7470B498FEDB7914763EE93
:102E9000B70217E701001307A78E8A05BA959C4170
:102EA000BA978287B717004003A7470D1345F5FF70
:102EB000698F23AAE70C03A7070D698F23A8E70CE6
:102EC00003A7070C798D23A0A70C8280B7170040B9
:102ED00083A6470D1347F5FFF98E23AAD70C83A6C7
:102EE000070D558D23A8A70C83A6070C758F23A06B
:102EF000E70C8280B717004003A7470D498F23AA2C
:102F0000E70C03A7070D1345F5FF45BFB7170040B2
:102F100083A6470D1347F5FF758F23AAE70C03A778
:102F2000070C598D4DB7B717004003A7470D498FC0
:102F3000EDB7797122D43714004026D24AD0035914
:102F400024028354040206D64209C2044ECE52CC57
:102F500056CA13590901C1802DE11379F9F793F489
:102F6000F49F4209C20413590901C18093078008E4
:102F7000F3B7078093F787083EC401000100930769
:102F800070052300F404930780FA2300F404010081
:102F90000100231124032310940223000404A247F8
:102FA000F3A7078001000100B25022549254025945
:102FB000F249624AD24A45618280B7F507008146EC
:102FC0003000B105194597000020E7808081A247B5
:102FD00013972701E34A07FC1369090893E40440A7
:102FE00093098008F3B7098093F787083EC0010072
:102FF0000100930A700523005405130A80FA230088
:10300000440501000100231124032310940223002E
:1030100004048247F3A7078001000100294597F0C7
:10302000FF1FE7802031F3B9098093F989084EC268
:1030300001000100230054052300440501000100A4
:103040008357040293E707202310F40223000404AB
:103050009247B9B7B7170040884742054181937737
:10306000050491EB9377F5013755E80113050580C9
:103070003345F50282809377050C130700046397AC
:10308000E7009377F50137459C1CCDB72165130503
:1030900005D0828037E700E01C435443A183E20659
:1030A000D58F1CC1FD572320F7182322F7188280E3
:1030B00013178500B7E700E023A0E710618123A282
:1030C000A7108280B7F700E08847CC47828081470D
:1030D00037370040A14663C4C7003285828003456C
:1030E000B740E38EA6FE3385F5000345050085074E
:1030F0002304A740CDB797070020938727EF9C4371
:10310000173700201307872B3E95636EE5001737AE
:1031100000201307273F6368A70017070020232715
:10312000A7EC3E858280FD57EDBF8280411122C40D
:1031300006C62A8497000000E78000F22947B307FB
:10314000E502B2408D83B3D7870222449507B3D7F7
:10315000E70237370040C207C1832316F700410159
:103160008280411137150E0006C697000000E780E7
:1031700020FCB7370040130770F82381E7000D47A4
:10318000A381E70013070004A380E7000547238716
:10319000E700B24041018280373700408347270073
:1031A0001A0593F7F703C98F93F7F70F2301F70079
:1031B0008280B737004003C7170019C9D98DA38093
:1031C000B70003C70700136787002380E7008280EA
:1031D00093C5F5FFF98DA380B7008280AE872A875B
:1031E000B736004021463738004089E71703000012
:1031F0006700E3F383C8B600E30916FF05078348B9
:10320000F7FFFD17C20723041801C183F9BF41115D
:1032100022C406C62A8497000000E780E0E329471D
:10322000B307E502B2408D83B3D7870222449507E6
:10323000B3D7E70237370040C207C1832316F740F0
:1032400041018280716541111305052006C6970072
:103250000000E78000FCB7370040130770F82381B7
:10326000E7400D47A381E74013070004A380E74030
:1032700005472387E740B24041018280CC4141119C
:1032800006C6328503C6150083C5050022064D8E8D
:1032900042068D654186138875A2630C0611634B47
:1032A000C804138845A26300060D634AC8009385CD
:1032B00035A26301B6082390060029464DA0138865
:1032C00055A26305060D938565A2E316B6FE8D45EE
:1032D0001D4663E6E5081146198E63F3C7003E8676
:1032E000B7E704002390C600FC4797D501009385FB
:1032F000654B9DA0138895A263030611634E060DCE
:103300001388A5A263000613938505A5E315B6FAF5
:1033100099451D4663E5E504198E63F3C7003E86B3
:10332000B7E704002390C600FC479705002093856B
:1033300025D61DA09D451D4663E3E5022146198E55
:1033400063F3C7003E86B7E70400FC472390C6003E
:103350009705002093858534BA9582970146B2403F
:10336000328541018280AD451D46E3EAE5FE3146E6
:10337000198E63F3C7003E86B7E704002390C600AA
:10338000FC4797D5010093856544F9B7B1451D46C3
:10339000E3E7E5FC3546198E63F3C7003E86B7E7E1
:1033A00004002390C600FC4797D501009385054390
:1033B00065B78D451D46E3E4E5FA1146198E63F3C2
:1033C000C7003E86B7E704002390C600FC4797D5A8
:1033D00001009385E53D49B78D451D46E3E1E5F8DC
:1033E0001146198E63F3C7003E86B7E704002390A9
:1033F000C600FC4797D5010093850540B1BFA545A0
:103400001D46E3EEE5F42946198E63F3C7003E86B8
:10341000B7E704002390C600FC4797D501009385C9
:10342000E5391DBFB5451D46E3EBE5F23946198E7A
:1034300063F3C7003E86B7E704002390C600FC474D
:1034400097D501009385053501BFB7E7040003A3B5
:103450000713970600209386A6C24146A545170587
:1034600000201305E5B802832D455DE703C505007F
:103470000947631FE50803A84500411106C6034735
:10348000180032850346080022074168518F9308CF
:1034900028FE6307170563E9E800051863030703BF
:1034A00023900600294591A8130648FE630AC70425
:1034B0001518E31707FF15463E87637BF60015478F
:1034C00001A8130600023E876374F600130700028A
:1034D000B7E704002390E600FC471316070111A884
:1034E0003E8691C30546B7E70400FC472390C6001B
:1034F0004206CC45418282970145B240410182801B
:10350000130600083E87E375F6FC13070008C9B7E9
:103510002390060005458280828041677917630405
:10352000E504411122C406C685472A84639FF5003D
:10353000B7E7040022852244B24003A3871397050E
:1035400000209385E52F4101028389476399F500A7
:10355000B7E7040083A7070B8545829771D9B2406E
:103560002244410182808280797126D252CCAE847D
:103570002A8A97D501009385252A17D501001305BE
:10358000252C06D63AC622D44AD0368432894ECE6D
:1035900097C00100E78060CAA28517D50100130516
:1035A000252B97C00100E78040C9294597C001003D
:1035B000E78080CD83C7840093F70702F9E383C9CE
:1035C00004008947054532476396F908D44083C70C
:1035D000160083C60600A207D58FC166138616FEA5
:1035E000638CC7028D16638FD7068D6693862690EF
:1035F00029456391D706B7E70400A286225403A3A6
:103600004714B250F2494A86A6850259925452850F
:10361000624A8547456102832D450DEF93070002FD
:10362000354563E98702B7E70400FC47C844130641
:103630000002CA8582978149970700209387072156
:103640009C43014581CB9C4391C74E852286CA8508
:1036500082970145B250225492540259F249624A6B
:10366000456182802D457DF79307700F3545E3E373
:1036700087FEB7E70400FC47C8442286CA858297C4
:1036800065BF2145C1BF411122C437E4040083272F
:10369000841326C2AA84416506C697050020938537
:1036A000251A7D1582978327C40A17050000130584
:1036B00005E78588829795C0032304132244B2400E
:1036C000924497060020938626AE4146C5451705CD
:1036D00000201305659C41010283B24022449244BC
:1036E00001454101828019C59707002023A0A71634
:1036F00001458280454582801147636AA70A97D6B3
:103700000100938626100A0536951841411106C618
:103710003697AE87B2850287130700026145639D25
:10372000E700B7E70400FC47130600021705002076
:10373000130545F782970145B24041018280054754
:103740006145E39BE7FEB7E70400FC470546170524
:103750000020130525F7F9BF1307700F6145E39D9E
:10376000E7FCB7E70400FC471306700F17050020BD
:10377000130585F5C1B7130700086145E39EE7FA15
:10378000B7E70400FC4713060008170500201305DF
:1037900025034DB715476145E390E7FAB7E7040005
:1037A000FC471546170500201305C50961B70945F3
:1037B0008280411126C2B7E4040083A7C41322C447
:1037C0004AC006C62E8497050020938565072A897E
:1037D0008297058905C5970700209387E78B83D7D4
:1037E000A70BA28503A3440D2310F4002244B2408A
:1037F00092444A850249014641010283B240224473
:103800009244024949454101828097070020238163
:1038100007049707002023AF0702B717004003A74C
:10382000070CB706C0FFFD16758F23A0E70C03A792
:10383000070DB7064000558F23A8E70C03A7070C18
:103840003D9B23A0E70C03A7070D1367070123A8DF
:10385000E70C8280B717004003A5470C83A7470CED
:10386000598113451500C18B058999E3136525001E
:103870009707002083C7C7FD6380A7029707002032
:103880002388A7FC11C9970700209387A7FC03A3EF
:1038900007006303030002838280114517F3FFFFD3
:1038A000670063C8011122CC06CE3714004026CA37
:1038B0004AC84EC652C483447405034AB4058349BA
:1038C00084050349940597F0FFFFE780A0A0834794
:1038D000A40593F4F40F137AFA0F93E71700230D5E
:1038E000F40493F9F90F1379F90FB717004003C7E0
:1038F000A705058B6DFF03D5C705A38D4705238C51
:103900003705A38C2705A38B9704F2406244D24469
:103910004249B249224A05618280411193970501CB
:1039200022C406C626C2C1872E8463DC0700B7E422
:103930000400FC54829719C1BC5482972165218DE3
:1039400015A893F7150013C515008DE793F725000B
:103950009DC797000000E78020F0B7E70400BC4F48
:103960001306000A894517050020034525EF8297B5
:1039700013452400B240224492444101828093972F
:10398000250163D80702B7E4040083A7C41E829709
:1039900097000000E780A0F0BC4C375607001306E4
:1039A0000630896517050020034545EB82970965B8
:1039B00079B7939715010145E3DE07FA17D50100A2
:1039C000130505F197C00100E780009FB7E70400E9
:1039D000BC4F13060064916517050020034505E8F8
:1039E00082971165A9BF1D71A2CC37E404005C5C0D
:1039F000485886CE494697D501009385E5E88297D9
:103A000011E917D50100130565E997C00100E780AA
:103A1000A09A01A0B7F600E0795798CAFD57DCCA12
:103A20000567B7E700E023A0E7101306F00290C295
:103A300023A0E718010001003707002018471306EC
:103A4000000481459706002023A8E6E04157A38A99
:103A5000E7403C4408088297970700209387077C3B
:103A60003EC8856713870740938757D1231AE10023
:103A70002312F1021307B00F97F7FFFF9387C76474
:103A80002310E1023ED81547970700009387C7E14E
:103A9000B7F50700A30FE1003EDC054797070000DC
:103AA0009387E7DF81463000E10519452301E102F4
:103AB0003EDE97F0FF1FE780C0D218088147994685
:103AC00030003E960346060085070507A30BC70096
:103AD000E398D7FEC24791C70357410185676373D7
:103AE000F70001A0B7E7040083A7470A08088297F8
:103AF000AA8511C917D50100130585DB97B0010010
:103B0000E780A07301A0F6406644256182804111E0
:103B100026C2B7E4040083A7040806C622C417051A
:103B200000001305C5DF829717040020130404D397
:103B30002300A40097000000E780800297000000A7
:103B4000E780E0CC03450400224403A38405B2408F
:103B5000924413060032896541010283797106D6C9
:103B600022D413078008F337078093F787083EC2F3
:103B700001000100B7170040930570052380B704CA
:103B8000130680FA2380C7040100010083C6F702F0
:103B900093F6A60FA387D702238007049246F3A6C5
:103BA00006800100010073370780137787083AC445
:103BB000010001002380B7042380C7040100010035
:103BC00003C7F70213672700A387E70223800704D0
:103BD000A247F3A7078001000100054597E0FFFF1A
:103BE000E780807297000000E78060CB0147814644
:103BF0008147054685451305407E97E0FFFFE78036
:103C0000807537E404003C44680051468145829742
:103C1000B707C0A83EC8B787E803938707D03ECA56
:103C200097E7FF1F9387A7793EC67C586800829765
:103C3000B250225445618280411197D5010093858D
:103C4000252E17D501001305A5BF06C697B00100A4
:103C5000E780A05E17D501001305854597B00100E8
:103C6000E780A05DB2402945410117B3010067001C
:103C7000A361411197D501009385C52B17D501008C
:103C8000130505BC06C697B00100E780005B17D599
:103C900001001305A54097B00100E780005AB2402B
:103CA0002945410117B301006700035E411122C499
:103CB00006C6834705002A849DC797D501009385D2
:103CC000252D17D501001305A5B797B00100E78092
:103CD000C0564C4017D501001305455697B001005A
:103CE000E780A0553DA058410DEF97D50100938581
:103CF000252A17D501001305A5B497B00100E78068
:103D0000C05317D501001305E55497B00100E780B3
:103D1000C0522244B2402945410117B30100670057
:103D2000A356A1679386D7036313D70297D50100E3
:103D30009385052617D50100130585B097B00100BE
:103D4000E780A04F17D501001305C5517DBFED07D2
:103D500097D501009385C52317D50100130545AEFE
:103D6000631BF70097B00100E780204D17D50100D5
:103D70001305855059BF97B00100E780004C4C40B7
:103D800017D501001305455191BF411197D5010089
:103D90009385851B17D50100130585AA06C697B024
:103DA0000100E7808049B2402945410117B3010075
:103DB0006700834D397122DC26DA4AD82E842A899D
:103DC0008145B2844808714636C606DE97E0FFFF9B
:103DD000E780E03397F7FF1F9387075EDC4783D7C1
:103DE0000700231C2101231BF10097500000E780EE
:103DF000E060B246230DA10091E2854693070019C9
:103E00003ECE2686FD57A2854808A30DD100230289
:103E1000F10297500000E7804061F2506254D254A2
:103E20004259216182808546170300006700C3F86C
:103E30004111814617F6FF1F1306465585451705A4
:103E400000200355252306C697D00000E780A0B0C8
:103E500015C997D501009385651217D50100130583
:103E6000259E97B00100E780403D17D5010013055E
:103E7000E53897B00100E780403C294597B0010044
:103E8000E780804097D501009385450F17D5010045
:103E90001305059B97B00100E780203A17D5010074
:103EA0001305053797B00100E7802039294597B001
:103EB0000100E780603D97F7FF1F9387E74FDC47DE
:103EC000054797D501009385650B2390E70017D52B
:103ED00001001305E59697B00100E780003617D57D
:103EE00001001305253497B00100E7800035B2408A
:103EF0002945410117B3010067000339411122C46C
:103F000097D501009385050A2A8417D5010013056A
:103F1000259306C697B00100E78020324C4017D5A4
:103F200001001305252B97B00100E78000312945DA
:103F300097B00100E7804035034704009307F00F76
:103F4000631FF70297D501009385C50517D50100BA
:103F50001305058F97B00100E780202E4C4017D540
:103F600001001305252897B00100E780002D2244A9
:103F7000B2402945410117B301006700E330B24068
:103F8000224441018280411122C426C22A84AE8487
:103F900017D501001305C58A97D50100938545FC07
:103FA00006C697B00100E780402917D50100130528
:103FB000653397B00100E7804028294597B001009C
:103FC000E780802C97D50100938585F9970700201D
:103FD0002392870A17D501001305858605449707A4
:103FE00000202397970897070020239487089717A6
:103FF00000202398977297B00100E780002497155E
:10400000002083D5057217D501001305252E97B022
:104010000100E7808022294597B00100E780C02693
:1040200097170020238C875E97F7FF1F9387C73869
:10403000DC47170500200345E58203D70700C16769
:10404000FD17631EF700B7E7040003A387051306F7
:10405000000A85452244B240924441010283B7E7F9
:10406000040003A387051306001493050010DDB7B1
:10407000B1C1411122C417C501001305657C2E840E
:1040800097D50100938505ED06C697B00100E7803E
:10409000C01AA28517D501001305052497B00100A9
:1040A000E780A0192244B2402945410117B301001D
:1040B0006700831D828037A51C8137070001814777
:1040C000130555DC97F5FF1F9385057A13073719FC
:1040D00099463386F500034606008507318D330582
:1040E000E502E398D7FEA167938707E03375F502F1
:1040F0001305052042054181828041119717002058
:104100002391076297170020238A075006C61707D6
:104110000020034727019307F00A6315F70293076E
:10412000F0F88945170500201305C5FF1707002083
:10413000230AF7FE97070020A38607FE976000007A
:10414000E78000ED97600000E780C01997600000ED
:10415000E780001B8145370504009707002023A94D
:1041600007FA97070020238407FA97070020239374
:1041700007F297070020239107F097070020239666
:1041800007F897070020239707F897300000E7808B
:10419000C07E014597600000E78080F09700000036
:1041A000E780A0F1970700202392A7F6B7E7040065
:1041B000BC4F13060014894517F5FF1F0345856A98
:1041C000829797D501009385A5DA17C501001305DD
:1041D000256797B00100E78040069705002083D54A
:1041E000E5F217D501001305651197B00100E780CE
:1041F000C004B2402945410117B301006700C3085C
:10420000B7E70400FC471171A2DDCAD986DFA6DB3F
:10421000CED72E8432892E86AA8517050020130555
:1042200065F08297170700201307C7EF8347070041
:10423000930680029387E70793F7F70FE3ECF610F6
:10424000BA898A0717C701001307C768BA979C4342
:10425000BA9782878D4797D50100938525DA17C5D0
:1042600001001305E55D630FF40097B00100E780DE
:10427000C0FC17D501001305259797B00100E78012
:10428000C0FBBDA497B00100E78020FB17D501005B
:104290001305059797B00100E78020FA294597B0EC
:1042A0000100E78060FE930720F811469705002083
:1042B000938545E74A85170700202305F7E697070A
:1042C0000020A38207E697000000E78000B62A845A
:1042D0001DC997D50100938565D217C50100130547
:1042E000255697B00100E78040F5A28517D501005B
:1042F0001305C59497B00100E78020F4294597B0D5
:104300000100E78060F897D50100938525CF17C598
:1043100001001305E55297B00100E78000F217D5C0
:1043200001001305E59297B00100E78000F12945EF
:1043300097B00100E78040F54165930730FA0546E4
:1043400097050020938505DE7D1517070020230BB8
:10435000F7DC97000000E78040AD2A841DC997D59F
:1043600001009385A5C917C501001305654D97B0D8
:104370000100E78080ECA28517D501001305058CAC
:1043800097B00100E78060EB294597B00100E78016
:10439000A0EFB7E70400BC4F0566130606C8A145A9
:1043A00017F5FF1F0345054C8297FE506E54DE54EF
:1043B0004E59BE591161828091476303F40297D52B
:1043C00001009385A5C317C501001305654797B084
:1043D0000100E78080E617D501001305A58A71BDAD
:1043E000B7E70400FC4F914517F5FF1F03458547CC
:1043F000829797D50100938565C017C50100130505
:10440000254497B00100E78040E317D5010013056C
:10441000258997B00100E78040E2294597B0010067
:10442000E78080E697500000E7804014914535A46E
:1044300085476303F40297D50100938525BC17C512
:1044400001001305E53F97B00100E78000DF17D5B5
:1044500001001305658615B597070020239C27C327
:10446000B7E704000566BC4F130606C8C1450DBF7B
:104470008D476303F40297D50100938525B817C5CE
:1044800001001305E53B97B00100E78000DB17D57D
:10449000010013052584D5B3930740F8114697050D
:1044A0000020938525C84A8517070020230CF7C6EE
:1044B00097070020A38907C697000000E780E096D1
:1044C0002A84E30405EE97D50100938525B317C52B
:1044D00001001305E53697B00100E78000D6A285FC
:1044E00017C501001305857597B00100E780E0D47A
:1044F000294597B00100E78020D945BD9147E31CCD
:10450000F4F6B7E70400FC4F9305000217F5FF1F10
:1045100003454535829797D50100938525AE17C58C
:1045200001001305E53197B00100E78000D117C500
:1045300001001305A57BF1BD894763E3870297D589
:1045400001009385A5AB17C501001305652F97B032
:104550000100E78080CE17C501001305657A31BBE5
:104560009704002083C424BC9707002083C797BB0F
:1045700097D50100938585A8A20417C501001305EE
:10458000252CDD8C97B00100E78020CBA28517C5D4
:1045900001001305257897B00100E78000CAC20426
:1045A000294597B00100E78020CEC1849305D4FF50
:1045B00093960401C1824A8693F5F50F17050020F2
:1045C000130575B697300000E780E03EE35F90DCAE
:1045D000930750F8170700202306F7B483C7390064
:1045E0002286970500209385E5B385074A8517073E
:1045F0000020A30AF7B297000000E78000832A8416
:10460000E30505DA97D501009385459F17C501009D
:104610001305052397B00100E78020C2A28517D5B6
:104620000100130565CAC9B5894763E3870297D5B9
:1046300001009385A59C17C501001305652097B05F
:104640000100E78080BF17C501001305656E35B115
:1046500097500000E78080F1A28517050020130520
:1046600065AC97600000E780A09A81B38D47630333
:10467000F40297D501009385659817C501001305CD
:10468000251C97B00100E78040BB17C5010013054A
:10469000E56BE5B6B76602000146B7750200054551
:1046A00097E0FF1FE780E013930760F817070020EB
:1046B000230AF7A697070020A38707A693070006FB
:1046C000170700202302F7A6894717070020A30D2C
:1046D000F7A497070020238A07A497070020A38642
:1046E00007A4C147170700202302F7A4930720F966
:1046F00017070020A30CF7A2314697070020A388D4
:10470000A7A2970500209385E5A14A859707002079
:10471000238F07A097F0FFFFE78020712A84E3062C
:1047200005C897D501009385658D17C50100130550
:10473000251197B00100E78040B0A28517C50100A0
:104740001305456255B3B1476303F40297D50100E1
:104750009385C58A17C501001305850E97B0010022
:10476000E780A0AD17C501001305856139B6B7E72D
:104770000400FC4F9305000417F5FF1F0345850E49
:10478000829797500000E78060DEB145F9B5914708
:1047900063E3870297D501009385458617C501001D
:1047A0001305050A97B00100E78020A917C501008D
:1047B0001305C55ED9B49704002083C4E496970717
:1047C000002083C75796A204DD8C8E04B7770200C1
:1047D0006D14BE942286A68517C501001305455D9C
:1047E00097B00100E78060A5B7E70400FC47228688
:1047F000970500209385559328008297931604010E
:10480000C1823000A685094597E0FF1FE78060FD63
:104810002A8409C917C501001305455B97B001003B
:10482000E78080B9930770F81946970500209385B3
:10483000658F4A85170700202306F78E970700200B
:10484000A384878E97F0FFFFE780205E2A84E30E23
:1048500005B497C501009385657A17C50100130556
:1048600025FE97B00100E780409DA28517C5010095
:104870001305C55695B99947630BF41297C5010006
:104880009385C57717C50100130585FB97B0010017
:10489000E780A09A17C501001305C555F9BA9147DD
:1048A00063E3870297C501009385457517C501002D
:1048B000130505F997B00100E780209817C501009E
:1048C0001305C5545DBA9704002083C4E485970797
:1048D000002083C75785A204DD8C8E04B7770200C1
:1048E0006D14BE942286A68517C501001305455395
:1048F00097B00100E7806094B7E70400FC47228688
:10490000970500209385558228008297931604010D
:10491000C1823000A6850D4597E0FF1FE78060EC5F
:104920002A8409C917C501001305455197B0010034
:10493000E78080A8930780F8194697F5FF1F9385B5
:10494000657E4A8517F7FF1F230EF77C97F7FF1F39
:10495000A38C877C97F0FFFFE780204D2A84E30635
:1049600005A497C501009385656917C50100130566
:1049700025ED97B00100E780408CA28517C50100A6
:104980001305054D95B699476303F40297C50100D9
:104990009385C56617C50100130585EA97B0010028
:1049A000E780A08917C501001305054CF9B0B7E7EA
:1049B0000400FC4F9305000417F5FF1F034585EA2B
:1049C000829797500000E78060BA994579B18D478A
:1049D0006303F40297C501009385456217C5010082
:1049E000130505E697B00100E780208517C5010093
:1049F0001305054959B017C501001305654997B05E
:104A00000100E780609B1305C01297E0FF1FE7805D
:104A10004093014597E0FFFFE78000680D45971040
:104A20000000E780203E294597E0FF1FE780609166
:104A300097E0FF1FE780C0818DBA99476303F402B6
:104A400097C501009385855B17C50100130545DFF8
:104A500097A00100E780607E17C50100130505449B
:104A600029B817F7FF1F0347376C97F7FF1F83C756
:104A7000A76B22075D8F9166BA96C2061166C18246
:104A80001306F6EF8D476365D60297F7FF1F9387EE
:104A9000A7929C4B17F6FF1F0346F6689386C70044
:104AA0002DC203D6070069CA8907E39CD7FE894750
:104AB0001307A0F8114697F5FF1F9385A5664A8551
:104AC00097F6FF1F2380E66617F7FF1FA30DF76415
:104AD00097F0FFFFE78060352A84E308058C97C5CF
:104AE00001009385A55117C50100130565D597A051
:104AF0000100E7808074A28517C501001305453BBE
:104B0000E5B203D60700630EE60A8907E39BF6FECB
:104B10008D4779BF91476304F40297C501009385DF
:104B2000E54D17C501001305A5D197A00100E78049
:104B3000C07017C50100130525396FF00FF4B7E7F2
:104B40000400FC4F9305000817F5FF1F034585D1AE
:104B50008297C9B897C501009385454A17C50100DA
:104B6000130505CE97A00100E780206D17C5010051
:104B7000130505376FF06FF02390E70017F5FF1F5F
:104B80001305858397400100E780A09797C5010032
:104B90009385C54617C50100130585CA97A0010076
:104BA000E780A06917C501001305853497A00100AF
:104BB000E780A068294597A00100E780E06C814765
:104BC000C5BD2390070017E5FF1F1305E57E97403D
:104BD0000100E780009397C501009385254217C522
:104BE00001001305E5C597A00100E780006517C522
:104BF0000100130565315DBF011122CC06CE26CA26
:104C00004AC8834705002A849DC797C5010093853C
:104C1000A53A17C501001305A5C297A00100E780BA
:104C2000C0614C4017C501001305057197A0010034
:104C3000E780A060E1A05841B707CF009387777D58
:104C4000631DF7060359C500854704450356E50073
:104C50009716002083D6E6AC63FC270383C70400C5
:104C600003C71400A207D98FC2077177C187130742
:104C7000C755639FE7006305D60C6244F240CA85BE
:104C800026854249D244056117E3FFFF670043557B
:104C9000630AD600CA85268532C697E0FFFFE78003
:104CA000205432466244F240CA8526854249D244A5
:104CB000056117F3FFFF6700E354B707CC00938744
:104CC000777D6317F70497C501009385E52E17C517
:104CD00001001305E5B697A00100E78000561C44CB
:104CE0008356E4008355C40003C6070017C50100BE
:104CF0001305056697A00100E78020546244F24046
:104D0000D24442492945056117A301006700C357F2
:104D1000B707CE009387777D6304F70297C501003C
:104D20009385852917C50100130585B197A001005A
:104D3000E780A0504C4017C501001305E555FDB5AF
:104D4000F2406244D244424905618280B7E70400E0
:104D5000FC4741112E8606C622C426C24AC02E84B4
:104D60002A89AA8517F5FF1F1305C53B829797C5AA
:104D700001009385652A17C50100130565AC97A04E
:104D80000100E780804B97F5FF1F83C5A53917C544
:104D90000100130565D097A00100E780004A29456E
:104DA00097A00100E780404E97F4FF1F938484375B
:104DB00083C7040041479387070693F7F70F636F94
:104DC000F75A17C70100130727BB8A07BA979C43F6
:104DD000BA9782879D476307F40297C501009385C0
:104DE000A52317C501001305A5A597A00100E7801D
:104DF000C04417C501001305A5CA97A00100E780AC
:104E0000C04395A497F7FF1F83C7D731DDCB17F7B2
:104E1000FF1F0347573197F7FF1F83C7C73022078C
:104E20005D8F97F7FF1F83C72730C2075D8F97F706
:104E3000FF1F83C7772FE207D98F17F7FF1F23299B
:104E4000F72C83C7640097C501009385E51C17C53F
:104E500001001305E59E17F7FF1F230AF72A97A005
:104E60000100E780803D97F7FF1F9387672A8C43F7
:104E700017F6FF1F0346A62917C50100130505C431
:104E800097A00100E780603B294597A00100E780DB
:104E9000A03F97F7FF1FA38707282244B240924400
:104EA0000249930700F817F7FF1F230DF7269D45CA
:104EB00017F5FF1F13050527410117530000670071
:104EC000231597700000E780E0E497F7FF1F238C1D
:104ED000A7249357850017F7FF1FA306F7249357BE
:104EE00005012A8417F7FF1F2300F7249357850134
:104EF000014517F7FF1FA309F72297700000E7800D
:104F0000C0E597F7FF1F2382A72297C5010093856D
:104F1000A51017C501001305A59297A00100E78011
:104F2000C03117F6FF1F03464620A28517C50100B2
:104F3000130545BAB1B7CD476303F40297C5010025
:104F40009385850D17C501001305858F97A0010076
:104F5000E780A02E17C50100130545B979BD97F765
:104F6000FF1F83C7471D17F7FF1F0347B71CA20783
:104F7000D98FC207C18717F7FF1F2319F718634A94
:104F8000F00097F0FFFFE780401397F7FF1F239F84
:104F9000A716B7E7040003A387051306000A89458F
:104FA0002244B2409244024917F5FF1F0345858B06
:104FB000410102838D476303F40297C50100938585
:104FC000A50517C501001305A58797A00100E78077
:104FD000C02617C50100130525C105B517F4FF1F2D
:104FE0000344641497F7FF1F83C7D71397C50100C5
:104FF00093858502220417C50100130565845D8C25
:1050000097A00100E7806023A28517C50100130562
:1050100065AF97A00100E7804022294597A00100D5
:10502000E78080260D4697F5FF1F9385A50F228503
:1050300097F0FFFFE78060DFAA8421C197C50100D8
:10504000938585FD17B501001305857F97A00100A5
:10505000E780A01EA68517C501001305E5AB97A044
:105060000100E780801D2244B24092440249294554
:10507000410117A301006700232197F7FF1F239B1E
:105080008700B7E70400116603A38705130606E847
:10509000914539B78D476303F40297C501009385A5
:1050A000A5F717B501001305A57997A00100E780C2
:1050B000C01817C501001305E5C181B317F4FF1F20
:1050C0000344640697F7FF1F83C7D70597C5010000
:1050D000938585F4220417B50100130565765D8C70
:1050E00097A00100E7806015A28517C50100130590
:1050F000E5A397A00100E7804014294597A001008F
:10510000E78080180D4697F5FF1F9385A50122853E
:1051100097F0FFFFE78060D1AA841DC197C5010009
:10512000938585EF17B501001305857197A00100E0
:10513000E780A010A68517C50100130565A005B777
:1051400097F7FF1F239A87F2B7E70400116603A3BE
:105150008705130606E89305000299B5894763E3BE
:10516000870297C50100938525EB17B5010013054C
:10517000256D97A00100E780400C17C501001305BD
:1051800025B8A5B997F4FF1F83C4E4F997F7FF1F6B
:1051900083C757F997C50100938505E8A20417B5A1
:1051A00001001305E569DD8C97A00100E780E008A8
:1051B000A68517C501001305259A97A00100E78071
:1051C000C007294597A00100E780000C228697F5CB
:1051D000FF1F938525F5268597F0FFFFE780E0C444
:1051E0002A84630E051A97C501009385E5E217B579
:1051F00001001305E56497A00100E7800004A28583
:1052000017C501001305859699BD854763F9871871
:10521000834519002244B24092440249B335B0009C
:1052200097F7FF1F2382B7E817C5010013054595BF
:10523000410117A3010067004300A2852244B24048
:1052400092444A8502494101171300006700C3C117
:1052500099476303F40297C501009385E5DB17B511
:1052600001001305E55D97A00100E78000FD17C56B
:1052700001001305A5C251B617F4FF1F0344A4EAA9
:1052800097F7FF1F83C717EA97C501009385C5D815
:10529000220417B501001305A55A5D8C97A00100E3
:1052A000E780A0F9A28517C501001305E58E97A038
:1052B0000100E78080F8294597A00100E780C0FC45
:1052C000194697F5FF1F9385E5E5228597F0FFFFC7
:1052D000E780A0B5AA841DC197C501009385C5D3F9
:1052E00017B501001305C55597A00100E780E0F44C
:1052F000A68517C501001305258B95B397F7FF1FEA
:10530000239A87E0B7E70400116603A38705130615
:1053100006E89305000869B1854797C501009385A4
:10532000A5CF17B501001305A551630BF40097A095
:105330000100E78080F017C501001305258875BCC2
:1053400097A00100E78060EF17C50100130585886D
:1053500097A00100E78060EE294597A00100E78053
:10536000A0F22244B2409244024997F7FF1F239FC4
:1053700007D84101177300006700438A97C50100F1
:10538000938585C917B501001305854B97A00100CA
:10539000E780A0EA17C50100130585B4B9BCB24087
:1053A00022449244024941018280411106C622C42E
:1053B00026C239C12A8497F00000E780400EAA84F3
:1053C00011EDB7E70400BC4741468145228582972D
:1053D000B2402244268592444101828041657D1578
:1053E00097F00000E780800CB7E7040001E9BC47B4
:1053F00041468145228582978144D9BF0347E50113
:10540000FC479305900819E393050003AA954146CC
:105410002285829785446DBF411106C622C426C2EB
:105420004AC097F00000E780800755CD97700000D4
:10543000E780008F2A8497100000E780804EAA84BE
:105440002285637394002685B7D7B0009387F75EF3
:1054500063F3A702B7E7B000130514009387F74F73
:1054600063E3A7082244B240924402494101177302
:1054700000006700A38B8567938707F13E956364FF
:10548000A4003305F40097700000E780208A97702D
:105490000000E780E0882A8963F6A40097100000E6
:1054A000E780E04A97C50100938585B817B50100EC
:1054B0001305053997A00100E78020D8A6864A8603
:1054C000A28517B501001305654F97A00100E7807D
:1054D000C0D62244B240924402492945410117A353
:1054E0000100670063DAB24022449244024941015C
:1054F0008280797122D437E404005C5C06D626D21F
:10550000354697C501009385E5BB17D50100130506
:10551000A592829711E917B501001305253897A0C8
:105520000100E78060E901A097E7FF1F93874734F8
:105530003ECCB7F50700856793870780814617E65D
:10554000FF1F13066632E10519453ECE97D0FF1FB7
:10555000E78020297C44194697E5FF1F9385C530D5
:1055600017F5FF1F130545B38297340817E6FF1F91
:105570001306862F97C501009385050117C5010005
:105580001305050297600000E780602EAA8421C100
:1055900097C50100938545A417B501001305452A59
:1055A00097A00100E78060C9A68517C50100130513
:1055B00065B297A00100E78040C8294597A0010087
:1055C000E78080CCB250225492544561828097E0AB
:1055D0000000E780809317C501001305A5A697502A
:1055E0000000E780802297500100E780C04C17E55B
:1055F000FF1F1305E5D897500100E780603517C5F8
:105600000100130525A597500100E780404DAA84AD
:1056100097600000E780408997000100E780A024A0
:1056200097800100E780C0BD97700000E78020E50B
:1056300097600000E78040FF97300100E78000E6B8
:1056400097C501009385459917B501001305451FBE
:1056500099C897A00100E78040BEA68517C5010044
:10566000130585A9B9B797A00100E78000BD17C54C
:1056700001001305A5AA97A00100E78000BC2945F9
:1056800097A00100E78040C097300100E780E0C1AB
:1056900097F00000E780A0E06300051497F0FFFF9B
:1056A000E780A0A197E7FF1F83D787C017070020D7
:1056B0002319F7062A8699C36302F50897C50100E6
:1056C0009385859117B501001305851732C697A0FC
:1056D0000100E78080B632469705002083D5650437
:1056E00017C50100130505A597A00100E780E0B4E8
:1056F000294597A00100E78020B997070020238F54
:1057000007F097070020239E070097600000E780BE
:10571000E05097C501009385258C17B5010013054E
:10572000251297A00100E78040B117C501001305BD
:1057300025A997A00100E78040B041B58545370510
:10574000040097200000E780402397C5010093855F
:10575000A58817B501001305A50E97A00100E780E5
:10576000C0AD17C50100130525A097A00100E78073
:10577000C0AC294597A00100E78000B18547170715
:105780000020230DF7E897E7FF1F9387E7C2DC4768
:1057900003D70700C167FD176316F70097E0FFFF07
:1057A000E780406997000000E78040C7971000003D
:1057B000E78040EB170500200355A5F69740000051
:1057C000E780805A054597500000E780608D97502C
:1057D0000000E780E0B235BF97F0FFFFE780E08D83
:1057E00097F7FF1F2394A79297B501009385C57E75
:1057F00017B501001305C50497A00100E780E0A3D9
:1058000017C601001306869897F5FF1F83D50590EC
:1058100017C501001305059897A00100E780E0A1D6
:10582000294597A00100E78020A63C4C1306000AFA
:10583000894517E5FF1F0345E5028297014597500B
:105840000000E780E085F1B5411122C437E404008F
:105850008327041A06C6829797400000E780805489
:10586000832704081705000013050503829797E7AF
:10587000FF1F2389A7FE17E5FF1F1305E5B3974018
:105880000000E78060052244B24041011703000098
:10589000670063C6011122CC06CE26CA4AC84EC68E
:1058A00093F715002E84B5CB97E0FFFFE780805873
:1058B000930710F817F7FF1F2306F78697E7FF1FD8
:1058C00083D7077B17F7FF1FA30EF7849145A183AA
:1058D00017F5FF1F1305058517F7FF1F2305F7842D
:1058E00097F7FF1FA381078497400000E78040726D
:1058F000B7E70400BC4F130600149305001017E52A
:10590000FF1F034525F6829713451400F2406244B9
:10591000D2444249B2490561828093F70510B1C76C
:10592000054597400000E780A07717050020035544
:1059300045DF97400000E780204397000000E780A4
:10594000E0AD97100000E780E0D197F7FF1F83C715
:10595000B78C89E797500000E780C0989750000007
:10596000E780009A1345041055B793F72500E9CF57
:1059700017E7FF1F0357877969C7AD64B719004060
:105980009384A4AA23A0990097E6FF1F93864678E4
:10599000944297C701009387279817E6FF1F034695
:1059A0000677814517C5010013050598976000002B
:1059B000E780E01623A0990097E7FF1F2392A790A6
:1059C0002A8941C197B501009385056217B5010089
:1059D000130505E797A00100E7802086CA8517B563
:1059E00001001305650097A00100E78000852945A7
:1059F00097A00100E780408997E7FF1F2398077071
:105A0000930710F817E7FF1F230EF77097E7FF1FA4
:105A100083D7076617E7FF1FA306F770A18317E771
:105A2000FF1F2302F77091458D4717E5FF1F1305F0
:105A3000656F17E7FF1FA308F76E97400000E78028
:105A4000205D13452400D9B593F74500D1C397B520
:105A500001009385655917B50100130565DE979020
:105A60000100E780807D17B501001305A5F9979027
:105A70000100E780807C294597A00100E780C08075
:105A8000930720F817E7FF1F230EF76897E7FF1F1C
:105A900083D7476017E7FF1FA306F768A18317E7BF
:105AA000FF1F2302F768854717E7FF1FA30DF7665F
:105AB00097400000E78080AB17E5FF1F1305856660
:105AC000914597400000E780A054134544003DBD38
:105AD00093F78500A9C797B501009385E55017B5E1
:105AE00001001305E5D597900100E780007517B513
:105AF0000100130565F297900100E78000742945C5
:105B000097900100E780407897E7FF1F2390076098
:105B100097600000E780801013458400C5BB93F7B1
:105B20000501D1C3854517E5FF1F0355A5569750BD
:105B30000100E78080C597B501009385E54A17B558
:105B400001001305E5CF97900100E780006F17B5BE
:105B500001001305A5ED97900100E780006E29452F
:105B600097900100E7804072930730F817E7FF1F16
:105B7000230AF75A97E7FF1F83D7C75117E7FF1F7D
:105B8000A302F75A17E5FF1F1305C559A1838D45D9
:105B900017E7FF1F2309F75897400000E7804047A9
:105BA00013450401A5B393F70502D1C797B50100CA
:105BB0009385854317B50100130585C897900100AB
:105BC000E780A06717B50100130585E897900100ED
:105BD000E780A066294597900100E780E06A930777
:105BE00040F817E7FF1F230FF75297E7FF1F83D7F0
:105BF000A74817E7FF1FA307F752A18317E7FF1F67
:105C00002303F752854717E7FF1FA30EF75097E7C7
:105C1000FF1F2393074697400000E780209517E574
:105C2000FF1F13052550914597400000E780403E37
:105C300013450402E1B993F70504FDC397B50100CC
:105C40009385853A17B50100130585BF979001002C
:105C5000E780A05E17B50100130505E197900100EC
:105C6000E780A05D294597900100E780E06197E714
:105C7000FF1F83C7274B1307700A6386E7061307C6
:105C8000800A638CE7081307600A6393E7049307AD
:105C900060F817E7FF1F2307F74897E7FF1F83D731
:105CA000C74617E7FF1FA30FF746A18317E7FF1F9C
:105CB000230BF746854717E7FF1FA30AF746B145B1
:105CC00017E5FF1F1305054697400000E7804034A5
:105CD00097400000E78080891345040497E7FF1F81
:105CE0002395074225B1930770F817E7FF1F230B91
:105CF000F74297E7FF1F83D7474117E7FF1FA3032B
:105D0000F742A18317E7FF1F230FF740854717E7E7
:105D1000FF1FA30BF740994565B7930780F8F1B7CC
:105D200093F705080145E38307BE97B50100938506
:105D3000A52B17B501001305A5B097900100E780CA
:105D4000C04F17B501001305A5D397900100E78058
:105D5000C04E294597900100E78000539307A0F8B3
:105D600017E7FF1F2300F73C97E7FF1F83D7873A0A
:105D700017E7FF1FA308F73AA18317E7FF1F2304C4
:105D8000F73A854717E7FF1FA30FF73897E7FF1F7D
:105D90002392073897300000E780407D17E5FF1F0A
:105DA00013054538914597400000E780602613456C
:105DB0000408A9BE411106C697E0FFFFE780C0FFB7
:105DC0000DC197E7FF1F83D7472E850717E7FF1FF2
:105DD000231DF72C97E7FF1F239AA72CB240410100
:105DE000828097E7FF1F83D7872C850717E7FF1F60
:105DF000231FF72AE5B78546170300006700C3FB9A
:105E0000411122C491462A8417E6FF1F1306863FDC
:105E10009D652D4506C697D0FF1FE780809CB7F78C
:105E2000070003C70701A5476313F70001A0930606
:105E3000001001469D65254597D0FF1FE780609AB9
:105E400097E7FF1F2380873C2244B240914617E624
:105E5000FF1F1306263B9D652945410117D3FF1FF0
:105E6000670023981171CED7B7E9040083A7C9044E
:105E7000CAD917E9FF1F1309E92AA2DD2E8686DF9A
:105E8000A6DB2E84AA854A85829797E7FF1F83C7E2
:105E900067291307700A6385E710636DF70013071E
:105EA000600A6385E704FE506E54DE544E59BE59B5
:105EB000116182801307800A6385E7161307900A31
:105EC000E393E7FE8D476306F41C97B501009385C5
:105ED000A55317B501001305A59697900100E7801B
:105EE000C03517B501001305654F25A08D47630C1C
:105EF000F40297B501009385255117B501001305EC
:105F0000259497900100E780403317B501001305F1
:105F1000254697900100E78040322945979001007F
:105F2000E780803649B7854717B501001305054658
:105F300017E7FF1F230AF71697900100E780C04775
:105F4000B7750200B76602000146054597D0FF1FEE
:105F5000E7802089930760F817E7FF1F2304F71CE9
:105F600097E7FF1FA381071C9307002617E7FF1F72
:105F7000232CF71AE5779387072117E7FF1F2317CD
:105F8000F71AB14597E7FF1F2383071A97E7FF1F0B
:105F9000A38FA7184A8597000000E780E01621B775
:105FA000914763E3870297B501009385E54517B5EF
:105FB00001001305E58897900100E780002817B5D8
:105FC00001001305A53EB1B797E4FF1F83C4C415B4
:105FD00097E7FF1F83C73715A204DD8C83A7C90489
:105FE0006D14228697E5FF1F93851514280082976C
:105FF0008E0493160401B7750200C1823000A69585
:10600000094597C0FF1FE780C07D930770F817E729
:10601000FF1F2309F710994597E7FF1FA386A710D5
:1060200095BF914763E3870297B501009385C53D0E
:1060300017B501001305C58097900100E780E01FA8
:1060400017B5010013050538E9B597E4FF1F83C4B0
:10605000A40D97E7FF1F83C7170DA204DD8C83A74C
:10606000C9046D14228697E5FF1F9385F50B280060
:1060700082978E0493160401B7750200C182300026
:10608000A6950D4597C0FF1FE780A075930780F880
:10609000BDBF17B501001305A53597900100E78036
:1060A000A031930790F82304F100834719008D4530
:1060B0002800A304F100834729002305F10097007D
:1060C0000000E78060041305C01297C0FF1FE7803F
:1060D0004027014597D0FFFFE78000FC0D45970062
:1060E0000000E78020D2294597C0FF1FE780602588
:1060F00097C0FF1FE780C0157DB397E7FF1F23AB55
:10610000A710828097E7FF1F9387C71003A307009C
:1061100063030300028317430000670063EF41112C
:106120004AC097F6FF1F83D6C65F328917D6FF1F76
:106130000356A62A22C426C206C62A84AE84970025
:106140000000E780606929C921C8994763F6970470
:106150008347140003470400A207D98F13978700D1
:10616000A183D98FC2073167C1831307C7556395D0
:10617000E70297D7FF1F83D74726A301F400A18327
:106180002302F40097F7FF1F83D7A75991C7A302F3
:10619000F400A1832303F40097F7FF1F83C7074888
:1061A000A1CB2686A28517D5FF1F0355052397008F
:1061B0000000E78080C4630F090297F7FF1F83C7C1
:1061C000E7458DEB97E7FF1F83C7070585C79DC090
:1061D00097E7FF1F83C747ED91EF22852244B24026
:1061E0000249A6859244410117430000670043E23B
:1061F000E31A09FCB24022449244024941018280E0
:106200000145828097A70100938707549C430111A1
:106210006800914506CE3EC697000000E780C0EEBC
:10622000F240056182808D4763F6B708011126CAE6
:1062300006CE22CC0344350097E4FF1F83C4D4FD6F
:1062400097B501009385051EB337800017E7FF1F40
:10625000A304F7FC09C497B501009385651D17B524
:1062600001001305651D97900100E78000FD97E789
:10627000FF1F83C777FA6386970097000000E780C7
:10628000C04597400000E780A0079967938757EEC5
:106290002316F100680085479145A3078100230775
:1062A000F10097000000E78020E6F2406244D2440B
:1062B000056182808280894763F7B708011122CC8B
:1062C00006CE26CA8344250085472A84639DF404AC
:1062D000914763F5B7040345450083473400220521
:1062E0005D8D97D7FF1F239AA70E97000000E780C8
:1062F00080579967938767EE2314F1008347340032
:1063000023059100A305F10083474400954528002B
:106310002306F10097000000E78000DFF2406244AE
:10632000D24405618280FDF89967938767EE231454
:10633000F10097D7FF1F83D7470AA305F100230574
:106340000100A183E1B782800111996722CCD517A2
:1063500017F4FF1F1304842C2314F1008347040057
:1063600026CA97F4FF1F9384C43B2305F10083D70B
:10637000040028009545A305F100A18306CE23065D
:10638000F10097000000E78020D803D60400834581
:10639000040017B501001305250B97900100E78055
:1063A000C0E9F2406244D244056182809D67797100
:1063B000D9172316F10097F7FF1F9387272683C766
:1063C00007001305F10006D62307F10097F0FFFF41
:1063D000E780E0FD09E9B7E70400BC474146814595
:1063E0001305F10082976800CD4597000000E78013
:1063F000A0D197F5FF1F83C5652217B501001305CE
:10640000A50797900100E78040E3B2504561828084
:1064100063060516411126C206C622C44AC097E784
:10642000FF1F83C777DF97F4FF1F83C4241F99C31F
:1064300093E424002A8497100000E780400119C1EA
:1064400093E4040137E904008327890422851306B5
:10645000200381458297930750FA2300F4009307A5
:10646000A005A300F400A302F40097F7FF1F83D751
:10647000472B2304F400A1830D47A304F40097D70E
:10648000FF1F83D787F52301E400230394001147FE
:106490002305F4009304C400A183A301E4002302B4
:1064A0000400A305F400268597F0FFFFE78020F0A5
:1064B00019E583278904414681452685829797D728
:1064C000FF1F83D727EF230EF400A183A30EF40050
:1064D00093070002230FF400930710FAA30FF400B0
:1064E0009D472300F402A3000402B7E70400FC4721
:1064F00013052402194697D5FF1F9385E536829729
:1065000097E7FF1F83D7A7BA2304F402A183A3044C
:10651000F40297E7FF1F83D747B92305F402A1834D
:10652000A305F40297E7FF1F938747B883970700F7
:106530002285930500032306F402C207C183A183C9
:10654000A306F40297D7FF1F938787D78397070087
:106550002307F402C207C183A183A307F4029700B3
:106560000000E78060232308A4022181A308A4027D
:10657000B2402244924402494101828082805D718E
:10658000E17793C777FF1305E10086C62316F10074
:1065900097000000E78000E868009305400397003B
:1065A0000000E78060B6B640616182804DC941114C
:1065B00022C426C206C6930750FA2300F5009307AB
:1065C000A005A300F500A302F50097F7FF1F93872E
:1065D000E70483C7070009472301E5002303F5000B
:1065E00097E7FF1F938757C383C70700114793049B
:1065F000C500A303F50097F7FF1F83D78712230475
:10660000F500A183A304F50097D7FF1F83D7E7DC2C
:106610002305F500A1832A84A301E50023020500D8
:10662000A305F500268597F0FFFFE78040D801E934
:10663000B7E70400BC4741468145268582972285FD
:10664000F14597000000E7802015230EA40021816A
:10665000A30EA400B2402244924441018280828071
:106660005D710A8586C6A2C497000000E78040F4E9
:1066700037E404007C448A850810794682973C44BC
:106680001305E10309468145829710109305000226
:10669000014597D0FFFFE7806006B6402644616160
:1066A0008280411122C426C22A84AE848566AA85CE
:1066B0000146254506C697C0FF1FE7808012A285C8
:1066C0002244B24026869244A1462945410117C37F
:1066D000FF1F670003110111B7C7A55A22CC93878A
:1066E000C73317E4FF1F130434B33EC483470400C9
:1066F0002C00196506CE3EC697000000E780A0FA80
:106700008345040017B50100130585E1979001004A
:10671000E780A0B2F2406244056182800111A14687
:10672000300099652D4522CC06CE97C0FF1FE7802B
:10673000400BA24737C4A55A1304C433639587029C
:10674000B24517B50100130565D5B335B00097E71D
:10675000FF1FA383B7AC97900100E78000AEF24023
:106760006244056182809165A1463000938505F001
:106770002D4597C0FF1FE780C006A247E38287FC34
:1067800097E7FF1FA38A07A8814517B501001305E6
:1067900025D3D1B7C16769768146FD1705061397E2
:1067A000060141836364B7003E8582803307D500CC
:1067B00003470700B98F214713F817008583630546
:1067C0000800B18FC207C1837D171377F70F6DF7EC
:1067D0008506F1B741C5A547054763F2B70883476A
:1067E0001500034705003168A207D98F139787006A
:1067F000A183D98FC207C1831308C8550547639089
:106800000707411106C622C426C20344250091474A
:1068100063F087049307540063ECF502A301C500FD
:1068200021822302C5009304340091C6A302D5003F
:10683000A1822303D5002A84A68597000000E78063
:10684000A0F526942300A4002181A300A400014701
:10685000B240224492443A854101828005473A85FC
:1068600082800111B7C7A55A22CC9387E7342A84C6
:106870002AC62C00156506CE3EC497000000E780AE
:1068800080E2A28517B50100130585CB9790010022
:10689000E780A09A97000000E780C0DCF2406244E5
:1068A000056182800111A146300095652D4522CCFD
:1068B00006CE97C0FF1FE780C0F2A24737C4A55A93
:1068C0001304E43463958702B24517B5010013053C
:1068D00025C197D7FF1F2392B7B0C205C1819790FA
:1068E0000100E7808095F2406244056182809165F5
:1068F000A1463000938505EE2D4597C0FF1FE78028
:1069000040EEA247E38287FCD14717D7FF1F23162B
:10691000F7ACD14517B50100130585BEC9B7011104
:10692000A146300091652D4506CE97C0FF1FE78038
:1069300040EB2247B7C7A55A938707350145631334
:10694000F7003245F240056182800111B7C7A55AB0
:106950002AC6938707352C00116506CE3EC49700E2
:106960000000E78040D4F240056182804DC54111AE
:1069700026C206C622C4AE84D1C92A84971000005C
:10698000E78080AD97E7FF1F83C7078999C7A68572
:10699000228597300000E780A06797F7FF1F83C725
:1069A000E7C7ADC7954763F397068347040013070E
:1069B0003005639DE7048346140013075004639772
:1069C000E60483462400130710046391E60403479A
:1069D0003400631DF702034744009307B0046317B4
:1069E000F70203475400930790056311F702A2854D
:1069F0002244B2402686924417D5FF1F0355E59DD9
:106A00008D46410117F3FFFF6700033BB24022446C
:106A1000924441018280828001114EC606CE22CC72
:106A200026CA4AC893F71500AE899DCBAD673717C4
:106A300000409387A7AA1CC3B7E70400BC4F130606
:106A40000019854517D5FF1F03450599829713C582
:106A50001900F2406244D2444249B2490561828041
:106A600093F725000145F5D717F7FF1F035747CBCD
:106A7000954763F9E70C014417F6FF1F130646BA62
:106A80009306300513055004130810049308B0044E
:106A900013039005930764006374F7043A847D59E7
:106AA00097F4FF1F83C4C4B797F7FF1F83C757B777
:106AB000A204DD8CAD679387B755638BF41463E351
:106AC000970AA9679387A755638EF414A28517F5D3
:106AD000FF1F1305E5B497000000E78060E9E9A017
:106AE000B307860083C50700639AD50483C51700E2
:106AF0006396A50483C527006392050583C5370007
:106B0000639ED50283C54700639A150383C7570068
:106B10006396670222890DE897F5FF1F83D545C06C
:106B2000B3852541C20517F5FF1F130565AFC18168
:106B30004A9597000000E780A0E3E1A00504420425
:106B4000418089BF3A847D598547E3EB87F45DC472
:106B5000854517F5FF1F1305A5AC97000000E780DA
:106B600020E169A8B1679387C7556389F404B567C5
:106B70009387D755E39CF4F4A28517F5FF1F1305FF
:106B800025AA97300000E780A0488947630EF400EB
:106B90009305E4FFC205C18117F5FF1F130565A822
:106BA00097100000E780408BA68517B501001305FC
:106BB000E59A97800100E780406889A0972000004F
:106BC000E780603A97100000E780608811C9A285CD
:106BD00017F5FF1F1305C5A497100000E780C087B5
:106BE0000546A28517F5FF1F130585A397F0FFFF44
:106BF000E780205397200000E780E036FD57E31D33
:106C0000F9F097F7FF1F239D07B013C5290091B531
:106C1000A28517F5FF1F1305A5A097F0FFFFE780DA
:106C2000605E59B7A28517F5FF1F1305659F97F0A2
:106C3000FFFFE780605D8DBF411122C437E404008F
:106C40005C5C06C6354697A501009385A54717B538
:106C500001001305651E829711E917B501001305A0
:106C6000259197800100E780207501A08327041CEF
:106C700082972A84054597C00000E78060289770B6
:106C80000100E78080AD97700100E780808297B0B7
:106C90000000E780E0392285B24022444101828031
:106CA0004111054506C622C426C297C0FFFFE780F2
:106CB00080281305A00497B0FF1FE780403F75753B
:106CC00085457D1597C0FFFFE78020127D758545BE
:106CD0001305F53697C0FFFFE780801B371400408F
:106CE0008327840A8D451305002093E7072023247A
:106CF000F40A97C0FFFFE780400FB7E4040097C095
:106D0000FFFFE7806054C85897800100E780C06AA1
:106D100017B501001305451297800100E780C0698F
:106D20008327840C8545414593E707082324F40C09
:106D300097C0FFFFE780C0158D451305000897C079
:106D4000FFFFE780E01497C0FFFFE780C04137A551
:106D500007001305051297C0FFFFE780603D01455E
:106D600097C0FFFFE780804395450545894717F7A2
:106D7000FF1F2309F79A97C0FFFFE780C043B7E7DB
:106D800000E013070006238DE7403707000423A027
:106D9000E71097D0FFFFE78040C597D0FFFFE7805F
:106DA00040D797000000E78060E997000000E78087
:106DB000209797000000E78020AF97F0FFFFE78063
:106DC000E0A897000000E780606A97000000E78075
:106DD000801083A7040817050000130525C48297B7
:106DE00097C7FF1F238AA75EBC4C13060064854526
:106DF000829797B0FF1FE780A05F01458280AD6753
:106E0000371700409387A7AA1CC3B7E700E03707EE
:106E1000400023A0E71801000100B7F7070003C7EF
:106E20000701A5476316F7009397450191C301A099
:106E30004111AE860146AA85254506C697C0FF1FAB
:106E4000E780209AB240B7E700E03707400023A070
:106E5000E710410182804111B2862E86AA852D4518
:106E600006C697C0FF1FE780C097B24001454101A9
:106E700082809307000463ECC7041D71A2CC2A84AE
:106E80000808A6CACAC886CE32C697800100E78025
:106E9000602FAD67371700409387A7AA1CC3B7E4DC
:106EA00000E03709400023A0241901000100B24688
:106EB0001008A285294597C0FF1FE7808092F64001
:106EC000664423A02411D644464925618280395561
:106ED000828041110D658D4506C697C0FFFFE78092
:106EE000C0F0B71700408D6623A6D70A17F5FF1F1D
:106EF000130585831387C70A9387870A1CC15CC55E
:106F0000856689675CC958C114C518C9B7E704000C
:106F1000B24003A3871E410102838145B307B50038
:106F20008387070089E7172300006700630A850548
:106F3000C205C181E5B7411106C6B94763EEB70086
:106F400017A501001305457B97000000E78020FD91
:106F5000B2400545410182808347E50013071003D5
:106F60006390E702854717F7FF1F2301F78C17A5EA
:106F700001001305A57A97F7FF1F2398078AE9B741
:106F800013070003E39EE7FA97F7FF1F2380078AA2
:106F900097F7FF1F239B078817A501001305857925
:106FA00065B7411126C2E97797F4FF1F938444889F
:106FB00022C49387A7552E842381B4002E86AA85E8
:106FC00017F5FF1F1305058706C62390F400A3815C
:106FD000040097800100E780E01A93052400C205B1
:106FE000C18117F5FF1F1305C58497F0FFFFE780E8
:106FF000A07AB38784002382A7002181A382A700FF
:10700000930564002244B24026859244C205C181A2
:107010004101172300006700A3FB09C9930700047F
:1070200063E6B700170300006700E3F7828093066A
:10703000F00F0307060019E79307F00F63F0B7029C
:107040002E85828093871500C207C183E3E6F6FE92
:10705000AA952380E5000506BE85E1BF2E95230095
:107060000500F9BF01111C08B69706CE238A07FE5A
:107070005C00BE9617A801001308C8771377F600C6
:10708000429703470700FD1611822380E600E3972D
:10709000D7FE3E8697000000E780A0F9F240056128
:1070A00082800111580006CE23070100A947BA8843
:1070B00029482543B3760603FD1793F7F70F938608
:1070C0000603A304D700B35606036375C3007D17F8
:1070D0003686EDF33386F80097000000E78060F510
:1070E000F24005618280397117A601001306066916
:1070F00006DE22DC26DA2A844AD84ED69700000023
:10710000E78020F3AA8517E6FF1F035686619146A4
:10711000228597000000E78020F597E7FF1F83C7CF
:10712000E74FAA8517A601001306C66289C717A6EE
:1071300001001306A661228597000000E78060EF3A
:10714000AA8517A601001306A663228597000000F2
:10715000E78020EEAA8517A601001306E6622285C5
:1071600097000000E780E0ECAA8511462285970091
:107170000000E78040F3AA8517B601001306C6BFDA
:10718000228597000000E780C0EAAA8517A60100C3
:1071900013060660228597000000E78080E9AA8533
:1071A00017B60100130646BD228597000000E78050
:1071B00040E8AA851306A005228597000000E78015
:1071C00080EE97D7FF1F83C73705AA8517A6010052
:1071D0001306C65889E717A601001306A65822858C
:1071E00097000000E780E0E4AA8517A601001306D7
:1071F000665A228597000000E780A0E337A60700C3
:10720000AA8513060612228597000000E780A0E9F0
:10721000AA8517A60100130666582285970000006C
:10722000E78020E197E7FF1F83C78751AA8517A64C
:1072300001001306A65389E717A60100130686531B
:10724000228597000000E780C0DEAA8517A601000E
:1072500013068655228597000000E78080DDAA8509
:1072600017A601001306C654228597000000E78088
:1072700040DCAA8517A60100130606542285970054
:107280000000E78000DB9146AA8517C6FF1F035662
:107290006612228597000000E78000DD2AC697501D
:1072A0000000E780E0A7B245AA8417A601001306F4
:1072B000E650228597000000E780A0D713D604018E
:1072C000AA8589461376F60F228597000000E7808D
:1072D000A0D9139604019146AA8541822285970080
:1072E0000000E78060D8AA8517A601001306864D26
:1072F000228597000000E780C0D39146AA8517C673
:10730000FF1F0356860D228597000000E780C0D539
:10731000AA8517A601001306664B22859700000078
:10732000E78020D19146AA8517D6FF1F035626D89D
:10733000228597000000E78020D3AA8517A60100C8
:1073400013064649228597000000E78080CE9146CB
:10735000AA8517D6FF1F035646D522859700000041
:10736000E78080D0AA8517A601001306264722854C
:1073700097000000E780E0CB9146AA8517D6FF1F53
:107380000356C6D2228597000000E780E0CDAA858B
:1073900017A601001306C644228597000000E78067
:1073A00040C9AA85914617C6FF1F035666F122857C
:1073B00097000000E78040CBAA8517A601001306BE
:1073C000A642228597000000E780A0C6AA858144D6
:1073D00097C9FF1F938949491949B387340103C6E7
:1073E00007008946228597000000E780E0C78504F2
:1073F000AA85E39424FF17A601001306663F2285A1
:1074000097000000E780E0C22AC6080897E0FFFF67
:10741000E780E0F9B24504081309010283C70400BC
:1074200003C614009146A2075D8E228597000000D6
:10743000E78080C38904AA85E31299FEF250625462
:10744000D2544259B2592161828017E5FF1F03458A
:10745000252F828097E7FF1F83C7473D89E71723C2
:1074600000006700E3B6828097E7FF1F83C7A7404D
:1074700099EF411106C697200000E78040ADB24069
:10748000854717E7FF1F2308F73E4101828082806E
:107490006302054E6380054E2971B7064000232E16
:1074A0001112232C8112232A91122328211323261F
:1074B0003113232441132322511323206113232E3C
:1074C0007111232C8111232A91112328A111232624
:1074D000B11101475948A5069319070193D909012C
:1074E00063F1B902B307E50083C70700D91793F723
:1074F000F70F6368F800B3D7F600858B1306170003
:10750000A1E3B3893541C20993D90901B9472E894D
:10751000AA8463F937033304E500394697A50100CF
:107520009385C50B228597800100E78040C319E948
:10753000CE85228597000000E78020A025E5F1A4F4
:10754000328759BF97E7FF1F83C7472E638F0724F2
:10755000BD6A396C014A17EBFF1F130BAB1E938BEF
:10756000FA55938CFA66130DEC5505A8B3874401C0
:1075700083C6070097E7FF1F83D7272BA5E3930751
:10758000A005639BF600854717E7FF1F231FF72819
:1075900097E7FF1F2388D71A050A93170A01C183AB
:1075A000E3E627FD8320C1130324811383244113C1
:1075B000032901138329C112032A8112832A41124C
:1075C000032B0112832BC111032C8111832C411138
:1075D000032D0111832DC11031618280854D639B84
:1075E000B7039307500A639EF600894717E7FF1F0A
:1075F000231DF722930750FA17E7FF1FA304F71480
:1076000061BF9307A005E389F6F897E7FF1F239E64
:10761000072059B7138717004207DA974183238061
:10762000D70017E6FF1F2312E6208D47E3F6E7F6A3
:1076300017E4FF1F0344341197E7FF1F83C7A71008
:1076400022045D8C9307F4FFC207C1839306F00DFB
:10765000E3EDF6FA93076400C207C183E31EF7F275
:1076600093052400C205C18117E5FF1F1305A50D71
:1076700097F0FFFFE780401233078B0083475700E6
:1076800003474700A207D98F17E7FF1F231F0718DB
:107690006312F5108149630DB40197E9FF1F83C997
:1076A000A90AA20997E7FF1F83C7170AB3E9F900E0
:1076B000170500001305A59697F0FFFFE78020A4AB
:1076C0006385790963EF3B036388A9059307EC653C
:1076D0006383F90697E7FF1F83C7070705476380A2
:1076E000E70881CB1387A7051377F70F8D4663F95A
:1076F000E6081307F0072300E100A300F100894525
:1077000095A8638999059387FA77E395F9FC97F033
:10771000FFFFE78000E711A8A28517E5FF1F13050B
:10772000A50297F0FFFFE78040B0014597F0FFFF0B
:10773000E780E09C95B5A28517E5FF1F1305C500FE
:1077400097F0FFFFE78060B7CDB797F0FFFFE780C6
:10775000E0BFE1BF97F0FFFFE78080C5F9B793076F
:1077600010F8130511002300F10097F0FFFFE780E8
:1077700020E4FD450A8597000000E780C08275B7C8
:10778000A28517E5FF1F130525FC97E0FFFFE780A3
:10779000A06D61BF9307F00789450A852310F100AA
:1077A00097000000E7802080C5BB1547637527055B
:1077B00003C604009306500B0147631FD60203C69D
:1077C00014009306B0053E876318D602CA85268545
:1077D00097F0FFFFE78000A311C917A5010013056B
:1077E000E5E097F0FFFFE78080736DBB17A5010010
:1077F000130505E1FDB70147B70640005946A50648
:1078000013140701418063692401CA85268597C046
:10781000FFFFE780E09C79B3B389E40083C70900E8
:10782000D91793F7F70F6367F600B3D7F600858B88
:107830000507F9F73304894042044180BD4763FDE1
:107840008706414697A50100938585DD4E85978083
:107850000100E780C09017A601001306A6DD05C150
:107860003D4697A50100938525DE4E859780010052
:10787000E780E08E21E917A601001306E6DD8145C9
:107880000A8597F0FFFFE780C07AAA850A859700EE
:107890000000E7808085AA85179601001306C65967
:1078A0000A8597F0FFFFE780C078AA850A859710C0
:1078B0000000E780E071FDB1E304F4FAB547E3F6B8
:1078C00087F439A8C147E3FB87FE454697A5010029
:1078D0009385C5D94E8597800100E780408815D5EE
:1078E000394697A50100938565CF4E8597800100A5
:1078F000E780E08601E5A2854E852DB9394697A53A
:1079000001009385E5D74E8597800100E7802085AB
:10791000E30D05EEC147E3FA87EE414697A5010066
:10792000938505D74E8597800100E7804083E31E4D
:1079300005EC83C7090113071003639CE700854723
:1079400017E7FF1F230EF7DE17A50100130585D5E6
:1079500049BD1307000317A501001305A5D7E3923E
:10796000E7E897E7FF1F238D07DC17A50100130544
:10797000E5D485BD8280411126C2AE848D4522C4E6
:1079800006C62A8497B0FFFFE7808050B7170040F3
:1079900099C803A5C70C418D23A6A70CB240224469
:1079A00092444101828003A5870C418D23A4A70C3A
:1079B000F5B78347050003471500A207D98FC20713
:1079C0006177C18713072720639AE7008345250065
:1079D0003705040017030000670023FA828017E6CA
:1079E000FF1F1306A6E98147B2861303F00FA948CB
:1079F0003308F6000348080013F7F70F6307A80CD5
:107A0000630668008507E39517FF2947B387E600FB
:107A10002380A70097E7FF1F938707E75DA8411121
:107A200013D765001347170006C693F63500058B7C
:107A3000954791CA054699476387C60009469D4701
:107A40006383C600A14713F645003336C00093F6A2
:107A50008503050685C2A145638BB604E145638AAB
:107A6000B604930580026388B6049305800363938C
:107A7000B600914697E5FF1F238DF50697E5FF1F9A
:107A80002388C50697E5FF1FA384D506BE8517A5E5
:107A90000100130525DA97700100E780007AB240F3
:107AA000854717E7FF1FA306F7044101828085463B
:107AB000D1B78946C1B78D4675BF17A5010013051B
:107AC000E5D9177301006700437717E7FF1F130716
:107AD000A7DBBA972380B700E147E302F5F49307E9
:107AE0007002E30CF5FC82802A8723800500814721
:107AF00017E5FF1F130585D81308F00F2946B306B5
:107B0000F50083C606006396E60297E6FF1F93869C
:107B1000A6D7B69783C7070005452380F500994788
:107B2000636EF7029D4763FDE700E147630DF700D1
:107B30008280638506018507E393C7FC0145C5B7CD
:107B4000238005008280B737004003C7370083C712
:107B5000050093F70704D98F2380F50082805D71BB
:107B600052DC56DA5ED6716A97EBFF1F938B8B0956
:107B70008D6AA6C24EDE62D486C6A2C4CAC05AD8D6
:107B800066D26AD06ECEC1495E8C97E4FF1F9384A3
:107B900064D0130A0A20938A7ADC17E9FF1F03498D
:107BA0006909B3872B0183C7070093F7F70FC9EF64
:107BB000B787004003C76700058BE310077C03C746
:107BC0006700118BE30D077E83C75700918B99E304
:107BD0006F10200317E7FF1F0347E705854763047E
:107BE000F7006F10400197E7FF1FA384E7F097E7C6
:107BF000FF1F238107D697E7FF1F238F07E097E733
:107C0000FF1F238D07EC97E7FF1F238A07EC97E7F9
:107C1000FF1FA38107D497E7FF1FA38F07DE97E716
:107C2000FF1FA38D07EA97E7FF1FA38A07EA97E7DD
:107C3000FF1FA38107EC97E7FF1FA38E07FEB787FF
:107C4000004011476F0070779307190093F7F70F03
:107C50003D476364F70617E7FF1F230DF7FC97E71F
:107C6000FF1F938727FCCA9783C7070013071002DB
:107C700093F7F703638EE71E6366F7040544638595
:107C8000871CE38C07620947638EE7101307000225
:107C9000E384E74EB7E700E03707400023A0E7188A
:107CA00001000100629923000900FD1923A0E710DB
:107CB00093F9F90FE39309EEE5BD97E7FF1F238BD7
:107CC00007F671BF130730026388E70C63E8E71615
:107CD00013074002638CE70A13070003E39CE7FAEB
:107CE00097E7FF1F938707F3CA9703C70700A147CA
:107CF0001377F70FE31BF71483C7640097E6FF1FA2
:107D00002380F6DE97E7FF1F83C737B991C7FD577A
:107D100097E6FF1F2386F6DC97E5FF1F83C595B71F
:107D200097E7FF1FA38EB7DA97E7FF1F83C787B6D2
:107D300013FB07089306000493F70706639FD74CCD
:107D40009307A009638DF51663EAB7129307F00550
:107D50006386F54A930750096384F52A014497E73F
:107D6000FF1F83C7F7D71547E392E736B7E700E071
:107D70003707400023A0E71801000100B786004044
:107D800023808602130680FC6F00500EFD5717E714
:107D9000FF1F2306F7D4FDBDFD5717E7FF1F230F75
:107DA000F7D2CDBD17A501001305C5BC9770010022
:107DB000E780806097E7FF1F9387C7E5CA9703C4F2
:107DC0000700014B97ECFF1F938C4CC51374F40F05
:107DD00017AD0100130D8DBA63478B0429459770C9
:107DE0000100E780604A854717E7FF1FA306F7C237
:107DF00017E7FF1F230387C217E7FF1F230CF7CEE8
:107E000037E700E0B70640002320D7180100010043
:107E1000378600408347A60293F7370F2305F60203
:107E20002320D71085BDB3876C0183C507006A8501
:107E3000050B97700100E780404079BF854717E741
:107E4000FF1F230BF7BCB9B517E7FF1F130787DC2C
:107E50004A970347070097E6FF1FA38DF6AE97E604
:107E6000FF1F238AE6AE17E7FF1F2305F7C81DB5DE
:107E7000854717E7FF1F230FF7AC29BD9307400A7B
:107E80006389F5349307200B6384F5369307100A52
:107E9000E396F5EC838724000144E3D207EC97E7EF
:107EA000FF1F83C7579F93F63700638A061A05465C
:107EB000638AC62209466395C61A1D4755A217E56F
:107EC000FF1F0345459DC94797ECFF1F83CCBC9C12
:107ED00097E5FF1F83C5459C17E4FF1F0344D49B10
:107EE0006315F510CD476392FC1093077008639CEF
:107EF000F5021307300FB7170E006308E4001307ED
:107F0000900DB7B704006314E40817E7FF1F232F91
:107F1000F7BCBE8517A501001305C5A69770010023
:107F2000E780A03125BD93078008639DF500B30766
:107F3000804013F4F70FB7774600938787CDB3D708
:107F40008702E1B793079008639AF500B307804072
:107F500013F4F70F91679387C766D5B79307A00807
:107F6000639BF500B307804013F4F70FB7173D008C
:107F700093870790E9B79307B008639AF500B307B2
:107F8000804013F4F70F9167938797D04DBF93F517
:107F9000F5078D47639BF500B307804013F4F70F97
:107FA000B7975B00938707D859BF8947639BF50054
:107FB000B307804013F4F70FB7770B009387071BC5
:107FC000BDBF8547639AF500B307804013F4F70FF0
:107FD000DD67938767E3A5B7D28785F9B30780404C
:107FE00093F7F70FB3D7FA020DB797000000E780B9
:107FF000409FA285668597000000E780809EB9BB00
:108000009305610017E5FF1F0345E58817E4FF1F8F
:108010000344748897000000E78040AD9305710029
:10802000228597000000E78060AC3C0017E7FF1F47
:108030002328F7BC834761002304F10083477100C4
:10804000A304F100894717E7FF1F230BF7A8835705
:10805000810017E7FF1F231FF782094409B3154763
:1080600093F64700B336D00093F78703850685C3A0
:108070002146638BC7066146638AC70613068002E2
:108080006388C706130680036393C700914717E60A
:10809000FF1F230FD6A497E6FF1FA38BF6A497E735
:1080A000FF1F2388E7A417D7FF1F0347E77E9376B8
:1080B000070497D7FF1F83C7377E8DEE1377770CA2
:1080C00093067008630CD7021377F7078D46631287
:1080D000D70CB307F040B7955B0093F7F70F938584
:1080E00005D849A81947ADBF854755B7894745B752
:1080F0008D4771BF930670086311D7021307300FC5
:10810000B7150E006389E7021307900DB7B5040099
:108110006383E7021307700845BF9306800C631161
:10812000D702B307F040B775460013F7F70F9387F0
:1081300085CDB3D5E70297E7FF1F23A9B79AD9BB2F
:108140009306900C631CD700B307F04093F5F70F2C
:1081500091679387C766B3D5B702F1BF9306A00CAA
:10816000631DD700B307F040B7153D0093F7F70F35
:1081700093850590B3D5F5027DBF9306B00CE3154A
:10818000D7F4B307F04093F5F70F9167938797D033
:10819000D9B78946631BD700B307F040B7750B000A
:1081A00093F7F70F9385051BF1B78546631AD70040
:1081B000B307F040DD6593F7F70F938565E35DBF87
:1081C000D28535FBB305F04093F5F50FB3D5BA0270
:1081D0009DB783C72400C18B99C7854717E7FF1F49
:1081E0002303F790A5BE97E7FF1F238E078EBDB62A
:1081F000854717E7FF1FA30EF78E8DB63C0017E7E4
:10820000FF1F232FF79E0947930700032314F10054
:1082100097E6FF1F2386E68C2DBD63940756A9477A
:1082200063E5B742179701001307075E8A05BA9501
:108230009C41BA97828717D4FF1F0344D465894CA9
:108240006306940D63E68C0685476303F408930781
:10825000F00F17E7FF1F0347A78863F6E70017E74C
:10826000FF1F230FF78697ECFF1F83CC6C879307C4
:10827000000413F4FC0F63F497011304000497E760
:10828000FF1F9387E79703AD070022862685EA85BF
:10829000B38C8C40229D97700100E780A0EE97E799
:1082A000FF1F238F978397E7FF1F23ABA79545BC3D
:1082B0008D47630CF40A9947E31BF4F89797010084
:1082C0009387075B17E7FF1F232CF792A94751B746
:1082D00017E7FF1F0347279697E7FF1F93874782FC
:1082E0004946979501009385A56163068700979598
:1082F00001009385E55C3E8597700100E78080E88A
:1083000017E7FF1F232EA78EC947A1B797E6FF1FC8
:1083100083C66692054797D7FF1F9387677E63944E
:10832000E6023E8513067002979501009385C55AB3
:1083300097700100E78000E517E7FF1F2322A78C55
:108340009307700239B73E851306300497950100F4
:108350009385C55297700100E780C0E217E7FF1FC1
:108360002320A78A93073004EDB597D5FF1F83C557
:108370008552179501001305256297700100E7806B
:10838000C0EB054D97EDFF1F83CDED8A97D5FF1FFD
:1083900083C5655017950100130505606398AD0B03
:1083A00097700100E78060E997D7FF1F83C7A74E4A
:1083B000B5CBE36EF4E8179401001304A458638C62
:1083C000B70117940100130464586386970117944A
:1083D000010013042459228597700100E78000FFF3
:1083E0001375F50F93071500860717D7FF1F23098D
:1083F000F7708D4717D7FF1FA304F77097D7FF1F9C
:10840000938707700147BE861376F70F8907636568
:10841000A60297D7FF1F23A5D77E97D7FF1F83C735
:10842000276E05BD979701009387C74A17D7FF1F8F
:108430002328F77C914731BD3306E400034606004C
:10844000A380070005072380C7007DBF9770010048
:10845000E780A0DE97D7FF1F83C7E743E1D7E36834
:10846000F4DE179401001304E44A638CA701179407
:1084700001001304A44A63869701179401001304B2
:10848000644B228597700100E78040F41375F50F67
:1084900093071500860717D7FF1F2303F7668D473D
:1084A00017D7FF1FA30EF76497D7FF1F9387476562
:1084B0000147BE861376F70F8907E37CA6F43306DF
:1084C000E40003460600A380070005072380C700D9
:1084D000D5B797D5FF1F83C5053C17950100130538
:1084E000654C97700100E78040D597D7FF1F83C781
:1084F000F76093E7470017D7FF1FA301F76083C713
:10850000240017D7FF1FA309F75E89B8179501004C
:108510001305854A97700100E78000EA97D7FF1F8F
:108520009387875D83C7070017D7FF1F2304F7369C
:1085300017D4FF1F0344C45A333480000DB017957D
:1085400001001305A54897700100E780E0E697D782
:10855000FF1F83C7B75A93E7070117D7FF1FA30F62
:10856000F75883C7240017D7FF1F2307F7586FF06A
:10857000EFFE179501001305A54697700100E780EF
:10858000A0E303C704007D8B51EFB787004003C70A
:1085900067021377C70B136727002383E70203C71C
:1085A000A7021377C70B136727002385E70203C7CA
:1085B000E7021377C70B136727002387E70203C778
:1085C00027031377C70B136727002389E702854723
:1085D00017D7FF1F2300F73817D7FF1F230EF742C7
:1085E00017D7FF1F230CF74E17D7FF1F2309F74E8E
:1085F00097D7FF1FA380073697D7FF1FA38E07408B
:1086000097D7FF1FA38C074C97D7FF1FA389074C51
:1086100097D7FF1FA380074E97D7FF1FA38D076033
:108620006FF0CFF389476312F70297D7FF1F83C715
:10863000A7269146638CD70863E0F604638EE70CA7
:108640006369F70A05476380E70EFD5717D7FF1FD9
:10865000A308F74837074000B7E700E023A0E71872
:1086600001000100B78600401306F0FC2381C6021A
:1086700023A0E7106FF00FE2130720086382E708DA
:108680006362F70213071008E391E7FC37870040A5
:108690008347670293F7C70B93E727002303F7028B
:1086A0006FF0CFEB130730086389E7021307400828
:1086B000E39DE7F8378700408347270393F7C70B0D
:1086C00093E727002309F7026FF04FE9378700404F
:1086D0008347270393F73707F5B73787004083476A
:1086E000E70293F7C70B93E727002307F7026FF022
:1086F000EFE6378700408347E70293F73707F5B780
:10870000378700408347A70293F7C70B93E72700FB
:108710002305F7026FF08FE4378700408347A702F5
:1087200093F73707F5B7378700408347670293F71A
:108730003707ADB7179501001305852B977001001A
:10874000E78080C797D7FF1F23860714D5B31795F7
:1087500001001305E52A97700100E780E0C597D76F
:10876000FF1F2399071297D7FF1F9387673703C40B
:108770000700894763F3870009441374F40F6FF00F
:108780000FDE13070002E392E7EC631B0B0A638F13
:10879000F500930720026383F50817950100130580
:1087A000A52997700100E78040A945B517950100FC
:1087B0001305C52597700100E78000C00144179D8F
:1087C0000100130DED25A14CB387840083C507007C
:1087D0006A85050497700100E78020A6E31694FFE0
:1087E000178501001305456B97700100E780C0BC39
:1087F00017D4FF1F0344440A01E897D7FF1F238DB6
:108800000706014B6FF0AFD58947E310F4E48547C5
:1088100017D7FF1F2302F7066FF04FD417D6FF1F9D
:108820000346760797D5FF1F83C5E5061795010018
:108830001305851F97700100E78020A06FF00FD20D
:108840006380F50693071002E399F5F497D5FF1FAF
:1088500083C58504179501001305051F9770010056
:10886000E780A09D97D7FF1F23AC973897D7FF1FAE
:108870009387C727944383D7470017D7FF1F034722
:10888000472717D6FF1F2327D6001D4497D6FF1F63
:108890002394F60097D7FF1F2381E7006FF02FCCBA
:1088A00097D5FF1F83C545FF179501001305451B8D
:1088B00097700100E780609897D7FF1F238E07FA13
:1088C00097D7FF1F239807FC6FF02FF92547638F79
:1088D000E7C89946378700406394D7022300870290
:1088E000B7E700E0B706400023A0D7180100010059
:1088F000130600FC2301C70223A0D7106FF08FB925
:108900009306100A639FD70023008702B7E700E0B1
:10891000B706400023A0D71801000100130680FC11
:10892000D1BF9306A009E381D7FE9306400AE38DE9
:10893000D7FC93062002639DD700B7E700E0B70697
:10894000400023A0D7180100010023008702F9B7D7
:108950008546E384D7FE93070008E300FBFEB7E7F4
:1089600000E0B706400023A0D7180100010013065D
:1089700020FC23008702BDBF17D7FF1F03475716F0
:108980006302F71E63E7E70295476300F710994714
:10899000630AF704B786004023800602B7E700E0C9
:1089A0003707400023A0E718010001001306A0FCD0
:1089B00075B99307F005630AF7009307500963063A
:1089C000F70093071002E317F7FCB7E700E037075B
:1089D000400023A0E71801000100B78600401306FD
:1089E00020FC69B117DBFF1F034B8B0F93070004BB
:1089F0005A8D63F46701130D000497D7FF1F938707
:108A0000272083AC07001374FD0F2286E685268598
:108A100097600100E7800077B3078B40669417D713
:108A2000FF1F230FF70A97D7FF1F23AB871CB787BA
:108A30000040630C0B022380A703B7E600E0370673
:108A4000400023A0C6180100010003C727021347F6
:108A500007042381E70203C727021377C70F238187
:108A6000E70223A0C6106FF0EFA22380070237E7CA
:108A700000E0B70640002320D718010001001306CC
:108A800020FC2381C7026FF0AFB9378700408347CE
:108A9000370097D6FF1F83C6360693F70708D58F92
:108AA000A301F700B7064000B7E700E023A0D718FE
:108AB000010001001306A0FC35BD97D7FF1F938767
:108AC0006715CA9783C7070093F7F70FC1CF97D7EA
:108AD000FF1F83C74716D9E717D7FF1F0347570064
:108AE000930700026310F70883AD040017DDFF1F32
:108AF000034D8DDA97DCFF1F83CC1CDA17DBFF1FD9
:108B0000034BABD9E6876A87DA866E8697D5FF1F57
:108B100083C585D617950100130505F697600100FA
:108B2000E780A07197D7FF1F23A2B7FD97D7FF1F3C
:108B30002380A7FD97D7FF1FA38C97FB97D7FF1F15
:108B4000238967FB97D7FF1FA38787D2B7E700E08A
:108B50003707400023A0E71801000100B786004056
:108B60006FF04FA2B7E700E03707400023A0E718F7
:108B700001000100B786004015BD97D6FF1F83C6D0
:108B8000860B0547639CE60429472381E7020947D2
:108B90002383E7022385E70297D7FF1FA38C07F4FF
:108BA00097D7FF1FA3890708B7870040A381070055
:108BB00017D7FF1FA30207F405472383E700B6403A
:108BC000264496440649F259625AD25A425BB25B35
:108BD000225C925C025DF24D6161828029472381B3
:108BE000E70209472383E7022385E7022387E70299
:108BF0002389E70255B717D7FF1FA30EF7C66FE00B
:108C00001FFF854717D7FF1F2306F7D417D7FF1F6E
:108C10002304F7E017D7FF1F2302F7EC17D7FF1F36
:108C2000230FF7EA6FE0BFFE854717D7FF1F230327
:108C3000F7D217D7FF1F2301F7DE17D7FF1F230F28
:108C4000F7E817D7FF1F230CF7E817D7FF1FA30379
:108C500007D017D7FF1FA30107DC17D7FF1FA30FEC
:108C600007E697D7FF1FA38C07E68280411106C64F
:108C700097000000E78080FBB78700402380070053
:108C8000130740FC2386E7001307C004A386E70010
:108C900017D7FF1F130707C02398E70017D7FF1F39
:108CA000130747C3239AE70017D7FF1F1307C7CE41
:108CB000239CE70017D7FF1F130747DA239EE7001F
:108CC00029472381E70209472383E7022385E70237
:108CD0002387E7022389E702A3810700930600F8B0
:108CE000A380D700930690022380D700FD562383EC
:108CF000D7002381E7009306000537E700E0230B48
:108D0000D740B70640002320D71003C717001367CA
:108D10001700A380E700B24097D7FF1F239E07DC10
:108D200041018280411106C697000000E78000F0F3
:108D3000B787004023800700130700FC2386E70065
:108D40003147A386E70017D7FF1F1307A7B423985F
:108D5000E70017D7FF1F1307E7B7239AE70017D7D6
:108D6000FF1F130767C3239CE70029472381E702FE
:108D700009472383E7022385E702A38107009306BF
:108D800000F8A380D700930690022380D700FD56F9
:108D90002383D7002381E7009306000537E700E02F
:108DA000230BD740B70640002320D71003C7170076
:108DB00013671700A380E700B24097D7FF1F239DDA
:108DC00007D241018280F1679387072017D7FF1FE1
:108DD000232EF7D0854717D7FF1F231BF7D0A147B6
:108DE00017D7FF1F2307F7D097D7FF1FA38307D0FD
:108DF00097D7FF1F238007D097D7FF1F238E07A683
:108E000097D7FF1FA38907A6814717D5FF1F130513
:108E1000E5A6FD5517D6FF1F130606A72947B3067B
:108E2000F5002380B600B306F60023800600850710
:108E3000E397E7FE97D7FF1FA38507CA97D7FF1FC2
:108E4000A38307CA97D7FF1F238E07C897D7FF1F93
:108E5000238907C897D7FF1F238807C897D7FF1F05
:108E6000A38207C897D7FF1F238F07C6814717D64E
:108E7000FF1F130626D94147B306F60023800600DC
:108E80008507E39BE7FE828017D7FF1F0347A7DA1A
:108E900085476316F700170300006700E3E8170330
:108EA00000006700E3DC411122C406C617D7FF1F8C
:108EB000034767D885472E8613F4F50FAA856317F5
:108EC000F70417D5FF1F130525B197600100E78050
:108ED000602B97D7FF1F238107B4B78700402384F7
:108EE0008702B7E600E03706400023A0C61801005D
:108EF000010003C7A7021377C70F2385E702B2401B
:108F0000224423A0C61001454101828017D5FF1FCE
:108F1000130545A097600100E780C02697D7FF1F83
:108F2000238A07A2B787004023828702B7E600E0C2
:108F30003706400023A0C6180100010003C76702DE
:108F40001377C70F2383E7025DBF411106C6970061
:108F50000000E78080E7B24041011703000067008E
:108F6000E3F2411106C697F0FFFFE78080BF97D775
:108F7000FF1F83C7379EA1CB97D5FF1F83C5A59D34
:108F800089C917D5FF1F1305259D97E0FFFFE780CF
:108F9000605097D7FF1FA38F079A97D7FF1F238B88
:108FA00007B437E700E0B70640002320D7180100D8
:108FB0000100378600408347660293F7370F23038B
:108FC000F6022320D710B2404101828041C9D9C5A1
:108FD00097D7FF1F83C747B2D1C3011122CC4AC81C
:108FE0004EC656C25AC006CE26CA52C42E89AA8977
:108FF0000144930A0004371B030063772403B3077B
:109000008940C207C183BE8463F4FA00930400045C
:10901000C204C180130A1BD497D7FF1F83C787934D
:109020009DE37D1A631C0A00F2406244D244424927
:10903000B249224A924A024B0561828097F0FFFFB3
:10904000E78020B2D1BF338589002694A6854204EB
:1090500097000000E78060E5418045B7828097D7A0
:10906000FF1F9387A7CF18429C4383D64500034533
:10907000070083C5C700035646006396A50083D545
:10908000E700638DD502011106CE2386A700239742
:10909000D700B705CF00DC4B9385757D05077D169E
:1090A0002EC2230001003AC42316C1002317D100A9
:1090B00099C30A858297F2400561828082804111BE
:1090C00022C417A4FF1F1304A4335C4C06C691CB23
:1090D000C84B01C9B7E70400BC5782975C4C23AA70
:1090E0000700B240224441018280DC4DDC4B81CF3D
:1090F000B7E70400904503A38705914517D5FF1FE7
:10910000034505C602838280B7E7040003A3070571
:10911000A14517D5FF1F0345A5C402836D713C0807
:109120003EC6B707E500232291103EC8AA843C083A
:109130003285232611103ECA2324811023202111B9
:109140002E8997300000E780605A2A8497950100A5
:1091500093850596177501001305856E97600100CC
:10916000E780A00DA28517950100130525A1976042
:109170000100E780800C294597600100E780C0105E
:10918000B705CB009385757D680097100000E780D8
:10919000E05FA285680097300000E78080470147C4
:1091A00081467000CA85268597200000E78060838D
:1091B00005CD2A84979501009385858F1775010049
:1091C0001305056897600100E7802007A2851795C1
:1091D00001001305659B97600100E78000062945A3
:1091E00097600100E780400A8320C11003248110AA
:1091F00083244110032901105161828097D7FF1FFA
:109200009387C7B518429C43797122D406D6034888
:10921000070083C807012A8483D64500035546000A
:109220006396080183D82701638DD802238807013C
:1092300005072399D7003708CC00DC4B1308787D4D
:109240003ACC1307F5FF42CA23080100231EE100B0
:10925000231FD10099C7080832C62EC48297324610
:10926000A245228597000000E78080EBB25022548F
:109270004561828079713146977501009385054D6E
:10928000280006D697600100E780C0EF97A7FF1F70
:1092900083D70717231B0100231C0100231D010096
:1092A000231E0100231F010099E3C167FD17231A44
:1092B000F10097A7FF1F83D7C71491EB97D7FF1F24
:1092C0009387C7A99C439C43DC4783D7070097A695
:1092D000FF1F9386E612231BF100D84E83D746006A
:1092E000231CF1005C4B91CB97A7FF1F83C7B711DD
:1092F00081EB97000000E780C0DCB25045618280BE
:10930000FD1717A6FF1FA300F6100356070183C71A
:1093100006014C472800230FF10097300000E7803A
:10932000602C97D7FF1F938767A39C4301479796AD
:10933000010093866681884330004C089710000036
:10934000E780206A5DD975B799C9B7E7040003A320
:109350000705A14517D5FF1F034585A0028382801D
:109360005C4EDC4BB9CFB1CD411122C41775010061
:109370001305054D2E84978501009385A57806C6B3
:1093800097600100E78060EBA28517850100130557
:10939000A57997600100E78040EA294597600100C0
:1093A000E78080EEB7E704002244B24003A38705BC
:1093B00017D5FF1F0345C59A130640069145410185
:1093C00002838280411122C417A4FF1F13040401E9
:1093D0001C4C06C689C7DC4399C34C488297584C3D
:1093E000B7E70400BC57484B82975C4CB24022441C
:1093F00023AA07004101828017A7FF1F1307070058
:10940000834707009306F00B850793F7F70F63E98F
:10941000F60097A6FF1F2383F6FE03450700828010
:10942000930700F8FDB78357450099E37D55828087
:10943000011122CC17A4FF1F130484FC5C4C4AC802
:109440004EC6DC4B52C406CE26CA56C2B2892E8AFC
:109450002A898DC7B7E70400FC5F829797D7FF1F63
:109460009387C78D9C431307301FB307F540715591
:109470006375F70697000000E780A0C49307D00D3E
:109480007D5563EC3705B7E4040093878900B8582D
:10949000832AC401139507014181029723AAAA00D8
:1094A000484C584921E7978501009385A5631775B6
:1094B00001001305E53897600100E78000D81785A3
:1094C00001001305256F97600100E78000D729454B
:1094D00097600100E78040DB5D55F2406244D24472
:1094E0004249B249224A924A056182801387490063
:1094F000B705CF002319E5009385757D31059710D9
:109500000000E780A028484C83456900310597306A
:109510000000E7800010484C4E86D2853105973018
:109520000000E780200C7146CA8517A5FF1F1305B0
:1095300025ED97600100E780E0C4FC5C829703267C
:10954000C90097C7FF1F23ABA77E11CABC4C854536
:1095500017D5FF1F0345C58082970145BDBF970002
:109560000000E78060D1D5BF411106C622C426C2E3
:1095700017C4FF1F1304C47E97000000E78060B487
:10958000B7E40400FC4C034504008545829703457D
:109590000400224403A3C405B2409244A145410102
:1095A0000283411126C297C4FF1F9384247B9C40F1
:1095B00006C622C44AC0D5C3DC43C5C35CC1230070
:1095C000B5002A84978501009385054D1775010024
:1095D0001305052797600100E78020C6294597609D
:1095E0000100E78060CA9C4023A4070023A2070073
:1095F00097A7FF1F938787DEDC4FDC4B91C7295568
:1096000097000000E78040DC97A7FF1F938747DFA4
:10961000DC4FDC4B89C797000000E78020F537E975
:1096200004008327C905894517C5FF1F03454573F6
:1096300082978327C905914517C5FF1F03454572CA
:1096400082979C4003A347016309030022852244BB
:10965000B2409244024941010283B2402244924402
:109660000249410182800111328506CE22CC26CAF0
:109670002E8497300000E7806007AA849785010058
:109680009385C544177501001305851B976001007C
:10969000E780A0BA030784000356640083554400A2
:1096A000A686178501001305A54A97600100E7808B
:1096B000C0B8294597600100E78000BD97A7FF1F4C
:1096C00083C727D2639D9700014597000000E7807C
:1096D000A0CF81450A8597000000E780C0ECF240EA
:1096E0006244D244056182806D7123248110232657
:1096F00011102322911093F745002E8463870714DD
:109700003C083EC0B707E5003EC23C083EC42317F4
:1097100001002318010023190100231A0100231B53
:10972000010097A7FF1F83D767CB99E3C167FD1798
:109730002316F10097A7FF1F83D767CA91EB97C73E
:10974000FF1F9387A7619C439C43DC4783D7070097
:1097500017A7FF1F130787C82317F100544F83571C
:1097600047002318F100DC4AA1E7978501009385A3
:10977000253A177501001305A50C97600100E780D5
:10978000C0AB178501001305654997600100E780AC
:10979000C0AA294597600100E78000AF1345440047
:1097A0008320C110032481108324411051618280E1
:1097B00097A7FF1F83C7F7C22555D9C3FD1717A663
:1097C000FF1FA300F6C203D6060183470701CC465C
:1097D0000A85230BF10097300000E780A0E097C7CF
:1097E000FF1F9387A7579C4317A7FF1F130707BFA8
:1097F000978601009386C63288430A866C009710CC
:109800000000E780001EAA8451D997850100938546
:109810002530177501001305A50297600100E78048
:10982000C0A1A685178501001305054097600100BA
:10983000E780A0A0294597600100E780E0A4268585
:1098400097000000E78040B891BF93F725009DC7BF
:10985000B7E70400BC474146814528088297255553
:1098600097000000E78040B628089305F00F9700A6
:109870000000E78040D3134524001DB793F715007F
:1098800081CB97000000E780209F1345140009BF9B
:1098900093F78500014589D717A7FF1F0347B7B680
:1098A00097A7FF1F9387C7B50DC3D84F584B11CF4C
:1098B00037E70400384F9047854517C5FF1F03451C
:1098C000254A029713458400E1BD97F0FFFFE7802A
:1098D000407FCDBF5C4D411106C688C317C7FF1F2F
:1098E000232EF746B7E7040083A7070817050000F3
:1098F0001305C5DF8297B24097C7FF1F2382A74693
:1099000001454101828001113335A000A307A10068
:10991000B7E7040083A7471706CE1306F100854575
:10992000130550308297F240056182808280411198
:1099300022C406C697B7FF1F83C7178E054489EF59
:1099400097C7FF1F83C787CD014499E717B4FF1F4F
:109950000344848C13441400228597000000E780A0
:10996000C0FA178501001305E53209E417850100E7
:10997000130545332244B2404101176301006700DB
:10998000C38B797122D4A30F010037E4040083272D
:10999000841726D24AD006D6AA842E8913055030C1
:1099A0009305F10132C6829732468347F101931540
:1099B0000601C18185CB01452EC697000000E780D6
:1099C000C0F483274417B2454A8626858297054509
:1099D00097000000E78060F3B2502254925402597D
:1099E00045618280832744174A8626858297EDB792
:1099F00041119397050122C406C626C2C1872E8451
:109A000063D40702B7E40400FC5417A5FF1F034505
:109A100025A2829719C1BC5482972165218DB2403D
:109A2000224492444101828093F715008DC7B7E725
:109A3000040083A7471A17A6FF1F1306669E97C543
:109A4000FF1F9385A53217A5FF1F0345659E8297CB
:109A500013451400E9B793F725000145E9D397C7EB
:109A6000FF1F83C7273285E7B7E7040003A8871ADB
:109A70001307401F97A7FF1F83C7879B81461306C5
:109A80004006994517C5FF1F0355452F02981345FA
:109A9000240071B797C7FF1F83D7472E6398A7028B
:109AA00017C7FF1F231DB72C17C7FF1F231AC72C6B
:109AB00017C7FF1F2317D72C2E8617850100130504
:109AC000E524BE8517530100670023771785010041
:109AD00013054525176301006700038E03574500F2
:109AE00097C7FF1F83D787296318F702C167F91744
:109AF00017C7FF1F2324F72897C7FF1F23A2072894
:109B000097C7FF1F238A072697C7FF1F238C0726A7
:109B1000170300006700E3E11785010013058520A6
:109B200017630100670043897D15954763E2A71C11
:109B300017870100130787140A053A951C41011184
:109B400022CC06CEBA972E84828717850100130592
:109B5000E51D97600100E7802086A1A203C72500CC
:109B600099476311F7022E8597000000E78040F7C0
:109B700083456400178501001305451C97500100BB
:109B8000E780A06B97A7FF1F238807681785010050
:109B90001305851C7DBF03C7250095476319F70290
:109BA000C16717C7FF1F0357671DF91703D5A50026
:109BB0006309F702B7E7040083A7C71782971785E1
:109BC00001001305651A97500100E780E07E854784
:109BD00017A7FF1F2302F764178501001305451B14
:109BE0008DBF97C7FF1F239BA71883D7E50097C694
:109BF000FF1F2396F61883D7050197C6FF1F2391F1
:109C0000F61883D7250197C6FF1F239CF61697C722
:109C1000FF1F23830716631BE502B7E70400BC4F51
:109C2000096613060690894517A5FF1F0345458061
:109C300082970356E4008355A4001785010013059D
:109C4000E51397500100E780405F51B79307700F0D
:109C50002316F100B7E7040083A7870D1796FF1FAF
:109C60000346067D6C0082974DF9854717C7FF1F95
:109C70002304F7105DB71785010013052512D1BD28
:109C800083C5250091476392F502178501001305EE
:109C9000651297500100E780207297000000E7806E
:109CA00040C9F24062440561828099476392F5029F
:109CB000228597000000E780A0E2834564001785B5
:109CC00001001305A50797500100E7800057D1BF99
:109CD0009547639AF50083471400E1F31785010067
:109CE0001305850FBDB5178501001305650FE1BF8D
:109CF00082803757315F9797FF1F9387A7741307A9
:109D000077D598C39356C500178701001307C7FC82
:109D1000BA9683C5060093568500BD8ABA9603C6D7
:109D2000060093564500BD8A3D89BA962A9783C698
:109D3000060003470700238407002383D700A3837B
:109D4000E7002382B700A382C7009797FF1F93877E
:109D500067702383B700A383C7002384D700A3843D
:109D6000E7008280411106C697000000E780A0F856
:109D7000B7E7040083A787141796FF1F1306866CA6
:109D8000D54501458297B2404D469795FF1F938573
:109D9000656C130570304101170300006700A3BE16
:109DA00061712324811A37E40400832704082326E1
:109DB000111A2322911A2320211B232E3119170552
:109DC0000000130525C382971799FF1F13094966E1
:109DD000994785442300A900231CF10097850100C1
:109DE000938585EE9307400617750100130545A579
:109DF000231CF1082308910097C9FF1F93896992DA
:109E000097500100E780604383D509001785010062
:109E1000130585EA97500100E780204229459750B5
:109E20000100E780604603D5090097000000E78045
:109E300080EC83274417100885451305503082971E
:109E4000832744171796FF1F1306C660CD451305D9
:109E500070308297832744171796FF1F1306865D7D
:109E6000B54513056030829783274417300889452C
:109E7000130510318297832744173009894513054C
:109E800020318297832744159305000A0D45829758
:109E9000832744159305000A11458297A305910075
:109EA0002306910002CD23080100230C0100832723
:109EB00084163009914513057040829783278416D4
:109EC0001306B10085451305004082978327841649
:109ED000700085451305104082978327841630084B
:109EE00085451305204082978327841610088545F1
:109EF000130550408297832704157D558297832749
:109F000044137D5582977D559790FFFFE780E0775A
:109F10008327440C82979790FFFFE7804053832765
:109F200084141796FF1F1306E651D5450145829705
:109F300089471306700F814528092306F100978091
:109F4000FFFFE780C01C8D471306000881452808E5
:109F5000230CF1089780FFFFE780601B9147230CDB
:109F6000F100976701009387277F984383C74700D5
:109F70003AC8230AF10097C0FFFFE780A06E700087
:109F8000854505459790FFFFE780407730099305A9
:109F9000700F09459790FFFFE780407630089305E2
:109FA00000080D459790FFFFE78040751008954524
:109FB00011459790FFFFE7806074C16717C7FF1FC7
:109FC0001307C7DBF9171CC3232207001795FF1FD0
:109FD0001305C5459790FFFFE78020718327C41DB7
:109FE00017C5FF1F130505D882973C480345090094
:109FF000854582978320C11A0324811A8324411A3C
:10A000000329011A8329C1195D618280C16717C8BC
:10A01000FF1F0358A8D6F9176301F8083DCDB5CD49
:10A02000011126CAB7E4040083A7841222CC2E862D
:10A030002315B10006CE2A8401478146ED454285AD
:10A0400082972AC611ED17850100130525CA97507E
:10A050000100E7806036F2406244D24405618280AC
:10A06000FC440356A100A28582972C0017C5FF1F50
:10A070000355C5D09790FFFFE780E07369DD178532
:10A0800001001305E5C797500100E780E03283A780
:10A09000C412ED45280082977DBF82800DC585479B
:10A0A0001797FF1FA30DF7389797FF1F238A0738CD
:10A0B00035469795FF1F9385E537130560301703E5
:10A0C00000006700438C9797FF1FA38A0736E9BFFC
:10A0D00097C7FF1F83C707CBA9EFC16717C7FF1F2C
:10A0E0000357C7C9F9176306F7044111854722C40E
:10A0F00017C7FF1F2308F7C837E404007C4C06C6C7
:10A1000089451795FF1F0345A53282970323841ABB
:10A110002244B2409797FF1F83C7873117C5FF1F9F
:10A120000355C5C51307401F814631469945410176
:10A13000028382806D712324811023261110232233
:10A140009110328401CD8947630AF5028320C11042
:10A1500003248110832441105161828017850100FE
:10A160001305C5C8AE8497500100E780E024A2859E
:10A17000268597B0FFFFE780A0BDC9BFB7E7040001
:10A18000FC4728008297178501001305E5C6975004
:10A190000100E78060228347810039C41307000B68
:10A1A0006380E7021387A7051377F70F8D4663EDEA
:10A1B000E602A285280097C0FFFFE780E0CA79B7D2
:10A1C0008547E3F587F8834591001775010013056E
:10A1D000259BB335B00097A7FF1F2387B7EC975097
:10A1E0000100E78080059DB703479100A207B9668B
:10A1F000D98F1387E6556384E70C636DF7042D67E9
:10A200001307B755638FE708636AF70029671307D9
:10A21000A755638FE708A2852800A1BF3167130700
:10A22000C7556388E70635671307D755E395E7FEFB
:10A230008947E3FD87F097000000E780A0E99305D8
:10A24000E4FFC205C1811305A1009790FFFFE780DD
:10A2500020F9EDBD3D671306F7556389C706636DA9
:10A26000F6009386E665E398D7FAA285280097C0A2
:10A27000FFFFE7808004D9BD9306F766638DD7049E
:10A280001307F777E399E7F897C0FFFFE780602FA0
:10A2900075BD0146A285280097C0FFFFE78060E8F2
:10A2A00075B5A285280097C0FFFFE780A0F579BDAE
:10A2B000A285280097C0FFFFE78000F541BDA28579
:10A2C000280097C0FFFFE78040F649B597C0FFFF21
:10A2D000E780C007A5BD97C0FFFFE780600DBDB553
:10A2E000C16717C5FF1F035565A9F9176307F50077
:10A2F000B7E7040003A3C7170283828017F3FFFFA9
:10A30000670023631783FFFFE702C3DB2A84084546
:10A310002E89B28919C900C1971500009385A586B9
:10A32000610597300100E780600481447D5A9710F1
:10A330000000E780E03963C7A4048144971000005F
:10A34000E780003A63C8A40497C7FF1F9387C7A399
:10A350009C43DC47B307F94091872302F4006383F1
:10A3600009048327C900B307F4409587A302F400CA
:10A370001C4C89C79C4799C3228582971783FFFF8E
:10A38000670083D75C44139714008504BA97239021
:10A39000470171BF1C48139714008504BA97239096
:10A3A000070069BF832789000547B307F4409587F5
:10A3B000A302F40083570400638EE7028DC30947AC
:10A3C0006384E7040D47E395E7FA978701009387D5
:10A3D00067F51CCC978701009387C7F511A897876D
:10A3E00001009387A7BB1CCC97870100938707BC0C
:10A3F0005CC8BDBF97870100938747A71CCC978790
:10A4000001009387A7A7EDB797870100938747F6C9
:10A410001CCC978701009387A7F6D9BF95E51783D2
:10A42000FFFFE702C3CB00461844834794007583BF
:10A430009D8B6317F70097100000E78060B448C455
:10A440001783FFFF6700E3CB82801783FFFFE702DC
:10A4500063C713893500C16442094111AA890144C7
:10A46000F11413590901054A2EC697100000E78020
:10A470002026B2456348A400014541011783FFFF30
:10A48000670083C783A7090013171400BA9783D7FF
:10A4900007006388B7006394970063742A0105047A
:10A4A000E1B70545D9BF1783FFFFE702C3C0AA89FB
:10A4B0002E89328BB6843A8ABE8A97A00000E78044
:10A4C00000FE71C9268597200000E780C00C8D47EB
:10A4D00063E7A7007D551783FFFF670043C183DB58
:10A4E000440097100000E780A0242A849710000001
:10A4F000E78040259307740031443305850263CD1E
:10A50000A70297100000E780A02297100000E780C4
:10A5100020222A8497100000E780C022930774004D
:10A5200031443305850263C3A70497100000E78018
:10A5300020209307450029A897100000E78080207D
:10A54000330585021307F0179307C017E35FA7FAD7
:10A550002D55E3C277F963040B02D6865286A68591
:10A560004A8597200100E78000BDB5B7971000002D
:10A57000E780401D330585029307C5FFD1BF8327C0
:10A5800049001385C90083D5270097000000E780A4
:10A5900000EC61F581B769553DBF97B7FF1F239761
:10A5A000A77E97B7FF1F9387277E904381470C466E
:10A5B0003307F500420741836393B7008280544616
:10A5C000139847008507C2962390E600D5B797B742
:10A5D000FF1F9387677B9C4303C58700828017B565
:10A5E000FF1F0355A57A82801783FFFFE70223AF81
:10A5F000C1671387D7FF630BE502636AA700F117F2
:10A600006300F50201451783FFFF670083AF1387DF
:10A61000E7FF6302E502FD171D8D13351500E5B751
:10A6200097500000E780A0297D15C5BF9750000016
:10A63000E78020FED5BF97500000E78040FCEDB7D3
:10A640001783FFFFE702A3A94111AA8401442EC684
:10A6500097100000E780C008B2456348A400014598
:10A6600041011783FFFF6700C3A99C48131514001D
:10A670003E9583570500E385B7FE0504C9BF03482F
:10A680005500814693F7F60F63E5070181473E8544
:10A690008280584593975600BA9703D727006316D0
:10A6A000B70003D70700E304C7FE8506E1BF834672
:10A6B000450001479377F70F63E4D700814711A85E
:10A6C0001C45131657000507B29703D60700E3137E
:10A6D000B6FE3E8582801783FFFFE702A39E931795
:10A6E0000501C18797BAFF1F938A0A6A635BF00866
:10A6F00083A70A00C0479C4703570400198D4205F1
:10A7000041816368F500014422851783FFFF6700DC
:10A71000A39E12052A94CDBFDC4713944900014A39
:10A720003E94834744006341FA02014A8347540040
:10A730006349FA028509C20993D9090183A70A006E
:10A740009847E3EBE9FCC1B71C4413195A00A685EE
:10A750003E994A8597000000E780C0EE05E1050AB2
:10A76000C9B75C4413195A00A6853E994A859700DB
:10A770000000E78020ED19E1050A4DBFE30C09FA5E
:10A7800061B7AA8481495DBF1783FFFFE702239564
:10A790001C452A8481E79307C5001CC51C4423126D
:10A7A00004001CC09307F00F63EDB70093F5F50F9D
:10A7B000228597200000E780C0E51783FFFF670030
:10A7C000439493940501C167C18063F9F500A685A0
:10A7D000228597200000E780E0E8C5B7C18193F5A6
:10A7E000F50F228597200000E780A0E2A68522854C
:10A7F00097200000E780E0E3C9B797B7FF1F938772
:10A80000A758884382801C4599C797B7FF1F23AD7F
:10A81000A756014582807D55828097B7FF1F938799
:10A82000A756984383474500484792073E95828044
:10A830001783FFFFE702A38A617100451C183EC61B
:10A84000B70780013EC81C183ECA8357440002CE99
:10A8500002D002CC231EF100834784002A8902D251
:10A860002301F1023C083ED402D697000000E780A5
:10A8700000FB835705002316F10297500000E78084
:10A8800040C72307A1025C4003556400F18313F71E
:10A8900017008347F10252055181F99BD98FA30715
:10A8A000F10297100100E780607839CDAA84035542
:10A8B000050097A00000E78060BF83D704002AD27C
:10A8C0006800231CF10083D72400231DF1001C48DD
:10A8D00003D647008C4397200000E780A0D0834731
:10A8E000B400CA86177601001306C6518117A30566
:10A8F000F4006C00481097200100E780C0835D6180
:10A900001773FFFF6700E37F2155D5BF1C45B1CF0B
:10A9100003C5A700894613576500630BD7028D4610
:10A92000630ED70285466300D7021307400633053E
:10A93000E50203C7B700418B15CB83C7B700BD8BBA
:10A940003355F54082801375F5031307803EC5B774
:10A9500009671375F50313070771D1BF372709007E
:10A960001375F5031307077CD9B701458280177368
:10A97000FFFFE702C37603A98500630C0904834740
:10A98000B900AE8493F7070E85C30345990093057C
:10A9900020030D810505B305B50288446105973094
:10A9A0000100E780C0AC35A02E8597000000E7804D
:10A9B00020F62A8419CD97000000E780605C83258B
:10A9C000C900B307B54063FA87002E94B305A440CD
:10A9D000E9F51773FFFF6700C37285457DBF1773E5
:10A9E000FFFFE702C36F2A8403D50500011132C6B9
:10A9F00036C43AC22EC002CA02CC02CE97A00000D2
:10AA0000E780C0AA82452ACA22852ECC9700000082
:10AA1000E780E0E003570500231EE10097500000A7
:10AA2000E78020ADA24632469247230FA100368729
:10AA30004C08B2862285014697000000E780E0A618
:10AA400005611773FFFF6700C36B1773FFFFE70212
:10AA5000036961711C183EC6B70780013EC81C1807
:10AA60003ECA3C0800453ED4AA8402CC02CE02D0A5
:10AA700002D202D697000000E78060DA8357050013
:10AA800035592316F10297500000E78080A623076E
:10AA9000A10209C48357440081EB21594A855D61B5
:10AAA0001773FFFF6700E36503556400520551818A
:10AAB00097100100E78080572A8965D18347B40049
:10AAC00093F7070E99C71305840197300100E780BB
:10AAD000409C83574400231EF100834784002301D8
:10AAE000F1025C4003550900D98313F70708834737
:10AAF0001102231CA10093F7F707D98FA300F102DD
:10AB000083572900231DF1005C40F18313F71700E0
:10AB10008347F102F99BD98FA307F10297A00000A8
:10AB2000E780C0982AD235D98347940068001397EC
:10AB300057008347B400FD8BD98FA305F4001C4850
:10AB400003D647008C4397200000E780A0A9A68782
:10AB5000177701001307072B740005464C10268554
:10AB600097000000E78060942A890DD98347B400DC
:10AB7000A685FD8BA305F40097000000E78060DF49
:10AB800031BF1773FFFFE7028355832485FE2A84B4
:10AB90004111268597000000E78080D7834734FF66
:10ABA00093F7070E8DCB2AC6268597000000E78015
:10ABB00060C809CD834734FFB245FD8BA309F4FE7D
:10ABC00091C5228597300100E780608A41011773A3
:10ABD000FFFF670003537DD98327C4FF2685829733
:10ABE00075F5834734FF93F7070E91C72285973099
:10ABF0000100E780008A032584FE97000000E780BB
:10AC000000E5E9B71773FFFFE702634A9C41411172
:10AC10002A8903C7070089472E84935667006380FB
:10AC2000F6040D466388C6049307F0076304F70231
:10AC30002E8597200000E78060ABAA848149C16B14
:10AC4000130C490097B7FF1F938707149C4398473D
:10AC500063E4E90441011773FFFF6700034903D769
:10AC600045008547E3F8E7FE2E8597200000E78042
:10AC700040ADE1B703D74500E3FEE7FC2E85972002
:10AC80000000E780A0A6AA84228597200000E78024
:10AC900000A8C204C98C5DB7DC470355A900139A0C
:10ACA00049003E9A93170501C187635DF000835701
:10ACB0000A006397A70263E774038327CA00034D62
:10ACC0005A002DA0A1672167A98F1307F7EFE3743E
:10ACD000F7FE6397090097000000E780209161FD6F
:10ACE00085098DB783278A00034D4A00835DA9003B
:10ACF00003576900216A138BC7003AC6814A33CAD9
:10AD00004D01631E5D0197B7FF1F938767089C4342
:10AD1000E1DBA2866286814526858297D1B7A1674D
:10AD20009387F7EF930C4BFF63F24703B2455A85C5
:10AD300097F0FFFFE780A0710DC103278B0010473C
:10AD400009CE10436382C4023107D5BFEE85668504
:10AD500097000000E780008F71F993861A0093FA3C
:10AD6000F60F130B0B0271BF835644005C43E3E9FB
:10AD7000F6F622853AC697200000E7802081A16779
:10AD80009387D7042A8A035D4400324763E897001B
:10AD90008347D90093E707F8A306F9001C476685A7
:10ADA0002286E2858297C1670844FD17337AFA004C
:10ADB000529508C02312A40125B797B7FF1F9387A8
:10ADC000A7FC9843814715C31447814763FFD5000B
:10ADD000939745004C47BE9519C903C75500814755
:10ADE0006375E600DC451606B2973E85828003C790
:10ADF00045008147E37BE6FE16069C45F5B71773D1
:10AE0000FFFFE702232CAA892E8A814497BAFF1FED
:10AE1000938A8AF783A70A00984763E6E4001773CA
:10AE2000FFFF6700632DDC471394440001493E9403
:10AE300013BB140083474400634BF900014913BB63
:10AE4000140083475400634FF9008504E1B70844B8
:10AE5000931759005287DA860146A2853E9582995A
:10AE60000509C9BF4844931759005287DA86054639
:10AE7000A2853E9582990509E9B71773FFFFE7029E
:10AE80000326814517F5FFFF1305054897B7FF1FF8
:10AE9000239E07EE97000000E780A0F61773FFFFE0
:10AEA0006700232697B7FF1F938707EE9C4395C340
:10AEB0001773FFFFE702A322814517F5FFFF130574
:10AEC000A54497000000E780C0F31773FFFF6700F9
:10AED000432382801773FFFFE702C31E37E4040099
:10AEE0008327841241112315E100AE893289368A05
:10AEF0003A8681460147ED45AA8482972AC621C930
:10AF00000356A100D28597400100E780A027832740
:10AF1000C413CE8526858297058905C98327440DEC
:10AF20002314210101462C00268582972A8401C919
:10AF3000B7E7040083A7C712ED4528008297228552
:10AF400041011773FFFF6700231B4944D5B76554C0
:10AF5000FDB75C41FD175CC182801773FFFFE702FC
:10AF60000318B7E70400FC5F829795473305F502A5
:10AF700081450D811773FFFF6700A3181773FFFF4B
:10AF8000E702E315B7E70400FC5F829795473305B6
:10AF9000F5020D811773FFFF6700A3161773FFFFFC
:10AFA000E702E313B7E7040083A7870B0355050007
:10AFB00082971773FFFF6700C3141773FFFFE70241
:10AFC0000312035505003287AE861786FF1F03560E
:10AFD000864E97B5FF1F9385E5DB97000000E7805D
:10AFE000A0EF1773FFFF6700C3111773FFFFE7029E
:10AFF000030FB7E7040083A7C71782971773FFFFF4
:10B00000670023101773FFFFE702630DB7E7040023
:10B0100083A7871397B5FF1F9385C5D782970145EF
:10B020001773FFFF6700E30D1773FFFFE702230BA2
:10B03000B7E7040083A7C71F81451785FF1F035586
:10B04000854382971773FFFF6700A30B1773FFFFFA
:10B05000E702E308B7E7040083A7871397B5FF1F4C
:10B06000938545D4829701451773FFFF67006309F5
:10B070001773FFFFE702A306B7E7040083A7C71F04
:10B0800081451785FF1F0355054582971773FFFFFD
:10B09000670023071773FFFFE70263042E8597807D
:10B0A0000000E780C0B297800000E780C0EF177310
:10B0B000FFFF670003051773FFFFE7024302978056
:10B0C0000000E780C0F91773FFFF670083035C4946
:10B0D000E1175CC95CC583572501A1072319F50059
:10B0E00083570501A1072318F5008280F147330536
:10B0F000F50297B7FF1F9387E7CC9C433E9582806C
:10B100008D476315F60803D74600854763F0E708C7
:10B110001773FFFFE702A3FC368536842E8997104C
:10B120000000E780A05C29C98357440093140501FF
:10B13000C18063E39704228597100000E780005BDD
:10B14000FD14231294009307A0026300F5029307F5
:10B15000B0026307F50293079002631FF500228592
:10B1600097000100E780A08801A80146CA852285D2
:10B1700097A00000E78040B31773FFFF670063F8F4
:10B18000228597100000E7806007FDB7828097B6A0
:10B19000FF1F938666C39C42014599CF9843D442D2
:10B1A00017B6FF1F2322E6C26396D70097B6FF1F8C
:10B1B00023AEE6C01385C7FE82801773FFFFE70248
:10B1C00003F297000000E780A04B7144330585022D
:10B1D000914597900000E78000EC11E565551773E5
:10B1E000FFFF670003F297B7FF1F23ABA7BC9700D1
:10B1F0000000E780E0483305850291459790000004
:10B20000E78060E961DD97B7FF1F23ADA7BA97001C
:10B210000000E780E04697B7FF1F239DA7B897007F
:10B220000000E780E04597B7FF1F2396A7B8977700
:10B230000100938767C217B7FF1F2321F7B897074D
:10B240000000938707E917B7FF1F2327F7B60145CB
:10B2500079B71773FFFFE70283E8AA8517B5FF1FC9
:10B26000130545B597100000E780605F1773FFFF77
:10B27000670023E91773FFFFE70263E6970000000A
:10B28000E78060FD97100000E780E05E97B7FF1F42
:10B29000938787B39C4391CF1387C7FE19CB83D580
:10B2A000C7FF17B5FF1F1305A5B297200100E78060
:10B2B000001C1773FFFF6700C3E41773FFFFE7026B
:10B2C00003E297000000E780C0EC09CD83478500CA
:10B2D0002A8493F7070499EB0355E50097000000D3
:10B2E000E78080F91773FFFF6700A3E18347C5007C
:10B2F0009304450117B9FF1F130909AD85E383279F
:10B3000009005CC997B7FF1F23A097AC83274900AA
:10B31000F1FB97B7FF1F23AB97AAE9B7FD172306E9
:10B32000F500610597800000E780A0D983078400BD
:10B3300063CB07048347840093E707F82304F400F2
:10B34000B7E704009C5F82974205A94741813375A6
:10B35000F5028347840093F707FCC98F2304F400A8
:10B360008347D4003E951C402318A40089CF9843FE
:10B3700019CB8347C4005040814585073305F5024A
:10B38000420541810297832709005CC897B7FF1FD8
:10B3900023AC97A28327490089E797B7FF1F23A70C
:10B3A00097A28347C4009DDF8355040117B5FF1F93
:10B3B000130505A297200100E780600B25B71773DE
:10B3C000FFFFE702C3D197B7FF1F9387A7C59C472D
:10B3D00001448583858B85E3AE84B2853A869710D8
:10B3E0000000E780204F2A8419C597100000E780ED
:10B3F0006045829408CC22851773FFFF670063D0F5
:10B400001773FFFFE70203CC41112E8932C6AA89C8
:10B4100097000000E780C031324713060502CA8654
:10B42000970500009385C5CC17B5FF1F13058598B8
:10B4300097000000E780E0F82A8425C99304C5003E
:10B4400097000000E780E0411946AA8526859710FD
:10B450000000E78020198545268597100000E780C9
:10B460000015177501001305E59C4E9583450500F1
:10B47000268597100000E780C0195C483146814559
:10B48000A1075CC85CC483572401E1172319F400A9
:10B4900083570401E1172318F4001C4C3E85977074
:10B4A000FFFFE780C0C6A304250122854101177371
:10B4B000FFFF670063C41773FFFFE70243C2411138
:10B4C000AA842EC632C497100000E780003A004DCF
:10B4D000B2452246834784000CC050C093F7F7035F
:10B4E00093E707042304F40023180400268597102B
:10B4F0000000E780203583479400A9462317A40065
:10B5000013D7370005073307D7029D8B850723061E
:10B51000F400A306E40083C70401D8488507230F7D
:10B52000F7FE17B7FF1F1307278A5843232A040083
:10B530009307440129E317B7FF1F2329F78817B79B
:10B54000FF1F2323F78817B4FF1F13046488228585
:10B5500097200100E780E0E31C44858B5D8D19E5B1
:10B560008145228597200100E78060F04101177333
:10B57000FFFF670003B91CC317B7FF1F2328F78419
:10B58000D9B71773FFFFE70283B5970500009385CE
:10B5900065B7014597000000E78000B001451773CB
:10B5A000FFFF670003B61773FFFFE70243B397007F
:10B5B0000000E78080B01773FFFF670083B4834704
:10B5C000C500A5E31773FFFFE70263B12A840355A3
:10B5D000E50097000000E78000C821C18347840090
:10B5E00093F7F7FB2304F4001C4091C7DC4381C7A9
:10B5F0004C400145829797000000E78080B917A56D
:10B60000FF1F1305E57C97200100E78080E80355C4
:10B61000E40097000000E78020C61773FFFF670073
:10B6200043AE82801773FFFFE70263AB97A7FF1F4C
:10B630009387877997050000938565C817A5FF1F35
:10B640001305057923A0070023A207009720010016
:10B65000E780C0D11773FFFF6700A3AA1C4D91CFED
:10B66000DC4381CF1773FFFFE70263A78345070021
:10B6700082971773FFFF6700C3A8828097A7FF1FF9
:10B68000938747779C4303C50700828097A7FF1FD6
:10B69000938747769C4303C51700828097A7FF1FB7
:10B6A000938747759C4303C52700828097A7FF1F98
:10B6B000938747749C4303C54700828097A7FF1F69
:10B6C000938747739C4303C53700828097A7FF1F6A
:10B6D000938747729C4303C55700828097A7FF1F3B
:10B6E000938747719C4303C56700828097A7FF1F1C
:10B6F000938747709C4303C57700828097A7FF1FFD
:10B700009387476F9C4303C58700828097A7FF1FDD
:10B710009387476E9C4303C59700828097A7FF1FBE
:10B720009387476D9C4303C5A700828097A7FF1F9F
:10B730009387476C9C4303C5B70011E11D45828088
:10B7400097A7FF1F9387076B9C4303C5C7008280A1
:10B7500097A7FF1F9387076A9C4303C5D700828082
:10B7600097A7FF1F938707699C4303C5E700828063
:10B7700097A7FF1F938707689C4303D50701828023
:10B7800097A7FF1F938707679C4303C52701828004
:10B7900097A7FF1F938707669C4303D547018280C5
:10B7A00097A7FF1F938707659C4303D56701828096
:10B7B00097A7FF1F938707649C4303D58701828067
:10B7C00097A7FF1F938707639C4303C5A701828048
:10B7D00097A7FF1F938707629C4303C5B701828029
:10B7E00097A7FF1F938707619C4303C5C70182800A
:10B7F00097A7FF1F938707609C4303C5D7018280EB
:10B8000097A7FF1F9387075F9C438857828097A75E
:10B81000FF1F9387275E9C4303D5C702828097A7AB
:10B82000FF1F9387275D9C4303D5E70219E11305AA
:10B83000800C828097A7FF1F9387C75B9C4303C53B
:10B840000703828097A7FF1F9387C75A9C43C85B53
:10B85000828097A7FF1F938767598843828097A7A5
:10B86000FF1F9387E7588843828019E17D558280C6
:10B87000F5DE984265DFFDD917A7FF1F1307877A0A
:10B880001847AA877155058B631D072403C5070058
:10B890001547E37DA7FC03C737001305F0057D17A7
:10B8A0001377F70FE364E5FC03C35700E30003FCE1
:10B8B00083C86700E38C08FA03C777004945791706
:10B8C0001377F70FE364E5FA03C7A70011481305E0
:10B8D000F7FF1375F50FE36BA8F803CE97000D483B
:10B8E0001305FEFF1375F50FE362A8F803C8B70050
:10B8F0006309080065181378F80F1305600DE367F6
:10B9000005F703C5C700794879151375F50FE36F7F
:10B91000A8F403C8D7000D457D181378F80FE36726
:10B9200005F503D80701930E401751184208135824
:10B930000801E3ED0EF303C8E7007D181378F80F54
:10B94000E36605F303C827017D181378F80FE36F4A
:10B9500005F103C88700C54E75181378F80FE3E7A3
:10B960000EF103D86701856E938EBEE06D18420814
:10B9700013580801E3EC0EEF03D847016D18420895
:10B9800013580801E3E40EEF03D887017918420841
:10B9900013580801E36C05ED03C8A7017D1813785F
:10B9A000F80FE36505ED03C5B7011D487D15137557
:10B9B000F50FE36DA8EA03C5D70171487915137532
:10B9C000F50FE365A8EA03D5E7011308E00F7D153D
:10B9D00042054181E36CA8E803C50702494879158F
:10B9E0001375F50FE364A8E8C85301C937C83400DC
:10B9F0005915130858BFE36BA8E603A8870237C59B
:10BA00003400130555BF5918E36205E717A5FF1F5A
:10BA10002320C53E03C6050117A5FF1F232CF53CB7
:10BA20000545E375C5E403D82501D04933760603FF
:10BA3000E31E06E203C61501E30A06E217A6FF1F8E
:10BA40002326B63A83C5270001466387A50003C6AF
:10BA50001700F1453306B60283C707039305C002FA
:10BA600072971A071307C70516031A979608469781
:10BA7000B387B70241553E973297420741836362CD
:10BA8000E8061763FFFFE7028365368597800000AD
:10BA9000E780806B97000100E780004B2A8497A025
:10BAA0000000E780605D2A9497F00000E78040295D
:10BAB0002A9497900000E78080842A9497F0FFFFF3
:10BAC000E780E06F2A9497400000E78000972A946F
:10BAD00097700000E780809F22951763FFFF670043
:10BAE000436282801763FFFFE702635F4111A30790
:10BAF000A10097A00000E78080C89305F10017051A
:10BB000000001305E5B597F0FFFFE780802F0145A2
:10BB100041011763FFFF6700C35E1763FFFFE70282
:10BB2000835917A4FF1F1304E44F03288400795995
:10BB30009368180097A4FF1F23AA144F13781800C6
:10BB400063100802BA84BE89368B328A2E89AA8A8B
:10BB500097F0FFFFE780E0A77D15269519E531599D
:10BB60004A851763FFFF6700835897F0FFFFE78060
:10BB700040A67D152695A167E353F5FE97B7FF1FF5
:10BB80009387478198433E8C814B01CB014597F0C9
:10BB90000000E7800047933B15004A85DA86568609
:10BBA000D28597900000E780A0502A8911CD1C44CF
:10BBB000F99B17A7FF1F232BF74683270C00CDD334
:10BBC000E3800BFA829769BF268597A7FF1F23ADF5
:10BBD000074497F0FFFFE780809C4146CE8517A57C
:10BBE000FF1F1305A54D97300100E780A05997D09E
:10BBF0000000E780209C0325040B97D00000E7801D
:10BC0000E09F054597D00000E780E0A60545970036
:10BC10000000E78060EDA9B797A7FF1F93878740D3
:10BC20009C47858BEDC71763FFFFE702434B17A5C2
:10BC3000FF1F1305E54697A7FF1F23A5073E97A7FC
:10BC4000FF1F23A3073E97A7FF1F23A1073E9720AF
:10BC50000100E780008497500000E780C0F897104B
:10BC60000100E780804F97100100E780805597A77B
:10BC7000FF1F9387A7399C4391C705459780000014
:10BC8000E780202397A7FF1F938707229C4399C72C
:10BC900041657D1597700000E78020A597F00000B2
:10BCA000E780C04097D00000E780609297A7FF1F11
:10BCB0009387474C9C43139717016356070097F0EF
:10BCC0000000E780E0AF97A7FF1F23A9073E97A7D3
:10BCD000FF1F23A7073E97A7FF1F23A5073E97A790
:10BCE000FF1F23A3073E97000000E780008C97000A
:10BCF0000000E780A07597F0FFFFE780401897F0FD
:10BD00000000E78020D91763FFFF6700833F828030
:10BD100097A7FF1F938707318843828097A7FF1F4C
:10BD200093874730C8438280B7E7B00093870750B6
:10BD300063E1A70297A7FF1F9387C72ED843FD573C
:10BD40006367E50097A7FF1F23A0A72E81473E85C5
:10BD50008280B957EDBF1763FFFFE7024338978032
:10BD60000000E780A07497800000E78000771763E9
:10BD7000FFFF670003391763FFFFE702A3342A843C
:10BD80009304140201112E85B289A685214636C678
:10BD90003A8997300100E780803C0DE9B2463808C7
:10BDA0002686CE851305940497500000E780A040B6
:10BDB00021462C084A8597300100E780403A133528
:10BDC000150005611763FFFF670003330145D5BF09
:10BDD0001763FFFFE702A3309305450617A5FF1F72
:10BDE0001305850197100100E78060681763FFFF66
:10BDF000670023311763FFFFE702632E41112EC650
:10BE000097F0FFFFE780C017B24588C14101176373
:10BE1000FFFF6700032F1763FFFFE702A32AAA842F
:10BE20002E8497800000E780406BAA898545228593
:10BE300097000000E780E07D83C7E4011389940840
:10BE400099E313890403CE85228597000000E780DB
:10BE5000407C214693051902228597000000E78067
:10BE6000607897A7FF1F9387E71B8C432285971065
:10BE70000000E780C08221469385840222859700D6
:10BE80000000E78020761763FFFF6700E326176353
:10BE9000FFFFE7024322397197F00000E78020B4EA
:10BEA0009305400661E997800000E780405F6302E8
:10BEB000051497A7FF1F83C7E7F513B7170097A6C9
:10BEC000FF1F2389E6F4014499CFC16417A9FF1F1E
:10BED000130949159309400EFD1497000000E780EF
:10BEE00020836342A40A97F0FFFFE780600941695D
:10BEF000B7290900096AFD7A2A8B81447D19938943
:10BF0000F97B130A0A71938A8AC797000000E780B9
:10BF1000208063D7A4041304400EB387840217A7BC
:10BF2000FF1F130727100324070B3E948357C401F8
:10BF30006382270B18403307EB4063EAE90083472D
:10BF400044008507B3874703D6976365F708014622
:10BF50008145094597F0FFFFE780C04AAA8B29E594
:10BF600097400000E780C08285476317F506896522
:10BF70009385057117A5FF1F130505E897100100AC
:10BF8000E780E04E95A0B30734030327090BBA9767
:10BF900003D7C7016308970003C75700A3820700B0
:10BFA0002382E700050415BF9305C500228597008D
:10BFB0000000E78080E65E85228697650100938514
:10BFC000A5E897F0FFFFE780404F5E8597100000DF
:10BFD000E780608A850415BF97A7FF1F93878704B2
:10BFE0009C478D83858BC1F721611763FFFF670035
:10BFF000031001468545094502D002D202D402D67B
:10C0000097F0FFFFE7800040AA8479DD97F00000F9
:10C01000E780209C1389C4002A8481454A859700C3
:10C020000000E780005F0C4041464A859700000011
:10C03000E780405B832944006385090C4E8502D864
:10C0400002DA02DC02DE97300100E78020382ACED7
:10C05000141005462C0808184ECC97500000E780B5
:10C06000200A1375F50F51ED8355840093E52500E3
:10C070004A8597000000E780E05E11460C104A8573
:10C0800097000000E7800056014697650100938500
:10C0900025DC268597F0FFFFE78020422685970064
:10C0A0000000E780407D5C40A1D3014685450D45F9
:10C0B00097F0FFFFE7800035AA841DD5484013891B
:10C0C000C40097300100E78060302AC64A85970097
:10C0D0000000E780404C3246636FC5004C404A8503
:10C0E00097000000E780005001468145268597F0C3
:10C0F000FFFFE780803C268597000000E780A0775F
:10C10000E5B583558400ADB71763FFFFE70223FD54
:10C1100097A7FF1F938707F19C471DC193E78700EF
:10C1200017A5FF1F130545CD17A7FF1F2320F7F005
:10C1300097100100E78080311763FFFF670063FC01
:10C14000DD9B17A7FF1F2323F7EE97300000E78042
:10C1500020647DF117A5FF1F130505CA9710010084
:10C16000E7802033D1BF1763FFFFE702C3F44169C3
:10C17000AA892E8AB28A368BBA8B814417ACFF1FEC
:10C18000130C4CEA930C400E7D1997F0FFFFE780EB
:10C19000205863C4A40001443DA033849403832742
:10C1A0000C0B3E948357C401638627055A87D686B5
:10C1B0005286CE851305040397000000E780E0BB9C
:10C1C00001C923800B0022851763FFFF670023F25C
:10C1D0008347F40185C35A87D6865286CE851305D8
:10C1E000940897000000E78040B909C5854723807F
:10C1F000FB00D1BF850451BF835745006380071EF4
:10C200001763FFFFE70203EC01112A849700000087
:10C21000E780C04D09C985476309F50605611763C5
:10C22000FFFF670063ED97E00000E780407B7DF54E
:10C23000835744004947ED9BE392E7FEC1452285C1
:10C2400097000000E7804033AA8422859700000011
:10C25000E780204F0357440002CE91472A89631A92
:10C26000F700228597000000E780A0513C082ACC07
:10C270003ECE97E00000E780C0755C55C5D37408DA
:10C280004A86A6850545829751BF03574400D1478A
:10C29000E3F6E7F8032A0400C169014997AAFF1FE2
:10C2A000938A4AD8130B400EFD1997F0FFFFE780E1
:10C2B0002046634FA90E2285032A04009700000040
:10C2C000E780C042A1452A89228597000000E780C7
:10C2D000A02AAA84228597000000E780804A1440A3
:10C2E0002A86AA8978082685CA8597000000E780F3
:10C2F000C0E7AA8405D503C7F40189476315F70091
:10C300008347C10181DF5546D2851385640097308C
:10C310000100E78020E7014597800000E7800019D1
:10C3200001C583D7C401A5E797A7FF1F938787CFD0
:10C330009C4793551900858913D73700058B01CF8A
:10C340008983858B6399B70001452EC6970000004D
:10C35000E780C0DBB2454E8597800000E780A01ED5
:10C360000346C1012A849375190026859790000021
:10C37000E780203935C1268597800000E7802018A6
:10C38000268511C0014597800000E780404B97301B
:10C390000000E780E03F8547E312F5E883C75400DB
:10C3A0001307F00FE38CE7E68507A382F400BDB521
:10C3B000B304690383A70A0BBE9483D7C401638BBC
:10C3C00037015546D2851385640097300100E78018
:10C3D00000D955DD0509D1BD5DD86DB782801763E1
:10C3E000FFFFE70223CE97800000E780400B05C1E6
:10C3F000C164014417A9FF1F1309C9C29309400E64
:10C40000FD1497F0FFFFE780A030634EA40017A54E
:10C41000FF1F1305659E97100100E7802003176337
:10C42000FFFF670063CD330534038327090B3E9577
:10C430008357C50163889700231205009780000089
:10C44000E780E00B050475BF97A7FF1F938787BDA3
:10C450009C478D83858B8DE31763FFFFE70223C81D
:10C4600017A5FF1F1305459997100100E78060028B
:10C470001763FFFF6700E3C882801763FFFFE702CF
:10C4800003C6970500009385C5A017A5FF1F1305D8
:10C49000A59697100100E78060ED1763FFFF670026
:10C4A00043C61763FFFFE70283C38841B7E7040071
:10C4B000BC5B050542054181829709C5854723007C
:10C4C000F50005051763FFFF6700A3C383C7F5FFEA
:10C4D0002E858507A38FF5FE828083C7F5FFFD17A4
:10C4E00093F7F70FA38FF5FE99EF1763FFFFE702AE
:10C4F00003BFB7E70400BC571385F5FF82971763A6
:10C50000FFFF670003C082801C41035745008D8FE9
:10C51000BA951CC12312B5003E85828093D7850051
:10C52000A2051441DD8D835745001387E6FF18C12E
:10C5300089072312F50013D685004111238FB6FE1B
:10C54000A38FC6FE4101828018419307F7FF1CC1EB
:10C550008357450085072312F500A30FB7FE82809D
:10C56000835745008D8F2312F5001C41BE950CC1E9
:10C570002E858280AA8703D7470008410D8FAA9590
:10C580002392E7008CC38280184108453305A740F9
:10C59000828083574500035765001D8F1C41084565
:10C5A0003385A7403305A74082801763FFFFE7026A
:10C5B00003B341112EC62A8497000000E780A0FD36
:10C5C000B2456373B50001A0835744000840BE958F
:10C5D0002312B4003E9541011763FFFF670063B269
:10C5E0001763FFFFE702A3AF41112E84B28532C665
:10C5F00097000000E780A0FB3246A285973001003B
:10C60000E78040B841011763FFFF670083AF1763FE
:10C61000FFFFE702C3AC2E84854597000000E7804A
:10C6200000F9230085001763FFFF670083AD1763E0
:10C63000FFFFE702C3AA41112317B1008945970004
:10C640000000E780C0F68347E1002300F500834740
:10C65000F100A300F50041011763FFFF670063AA23
:10C660001763FFFFE702A3A793D78500A205411137
:10C67000DD8D2317B100894597000000E78020F386
:10C680008347E1002300F5008347F100A300F50094
:10C6900041011763FFFF6700C3A61763FFFFE702AF
:10C6A00003A41397850193D78501C166938606F08D
:10C6B000D98F13D78500758FD98FA2053707FF0053
:10C6C000F98D4111DD8D2EC6914597000000E78060
:10C6D00000EE6C00114697300100E780A0AA4101EE
:10C6E0001763FFFF6700E3A11763FFFFE702239FC4
:10C6F0001C41854503C4070097000000E78080E6E1
:10C7000022851763FFFF6700C39F1763FFFFE702E0
:10C71000039D1C414111894503C7070083C71700CA
:10C720002307E100A307F10097000000E78080E302
:10C730000355E10041011763FFFF6700839C176306
:10C74000FFFFE702C3991C414111894503C7070058
:10C7500083C717002307E100A307F100970000003B
:10C76000E78040E08357E100410113D58700A2072D
:10C770005D8D420541811763FFFF67008398176352
:10C78000FFFFE702C3950C4141112A84114668005E
:10C7900097300100E780009F9145228597000000B7
:10C7A000E78040DCB247C166938606F013978701A5
:10C7B00013D58701598D13D78700758F598DA2071F
:10C7C0003707FF00F98F5D8D41011763FFFF670099
:10C7D00043931C45BE950CC18280AE87944391E67D
:10C7E000584101EF0CC15CC1828003C75700136739
:10C7F0001700A382E700B687D5B70CC3EDB7AA87A9
:10C80000084119CD1841D44398C36313D500D8C348
:10C810002A87034657009376160081E623200700F7
:10C820008280944381CA8C4203A847008CC36393DF
:10C830000601CCC3799A14C3A302C7003687D1BFBF
:10C840001C45DC471D8DB777DBB6938777DB098501
:10C850003305F502420541818280F147B385F50237
:10C8600048452E9582808347450085072302F500C1
:10C8700082801763FFFFE70283862A8409E4176337
:10C88000FFFF6700038883474400F5DBFD1793F73C
:10C89000F70F2302F400E5F71C4403D72700050730
:10C8A0002391E700DC4399C3228582974C4889CDC8
:10C8B00083475400898B99E71C4422859C479C43FD
:10C8C0009C478297232A04000040232004007DB760
:10C8D0001763FFFFE702A3808357250041112EC68F
:10C8E00081EB0144228541011763FFFF67006381EB
:10C8F000035705008147F146E305F7FEB385D702EC
:10C90000404585072E948345440008C4F5F5B24799
:10C91000AA8481E7232A040009A81C456C0022850B
:10C920009C439C43829748C84DDD85472312F40001
:10C93000B24723200400231804002319F4005C48A4
:10C940005CC483D72400FD172391F40061BF175303
:10C95000FFFFE702C3789797FF1F9387E74B884352
:10C960002326050023240500410597100100E780D8
:10C9700040B21753FFFF6700C3781753FFFFE7026A
:10C9800003761794FF1F130424491C40411199CFCB
:10C990009C472300B5002AC65CC197000000E780D1
:10C9A00040FB1C40DC4399C3324582974101175339
:10C9B000FFFF670003750347450029E3584DAA8729
:10C9C0007D551DCF1753FFFFE70263711CC3DC4782
:10C9D0009796FF1F23A2E644F15613050701239003
:10C9E000D700970500009385050297100100E780A6
:10C9F000E09701451753FFFF6700A3707D558280C4
:10CA000082801753FFFFE702836D01116146814564
:10CA100028009750FFFFE780806F9797FF1F93874D
:10CA2000A73F9C4328009305F00FDC473EC69700C4
:10CA30000000E780C0F405611753FFFF6700636CD7
:10CA40009797FF1F9387473D9C43D847A1679387DC
:10CA5000C702631EF70A397106DE22DC26DA80007F
:10CA60004AD84ED652D456D23285B28497000000AE
:10CA7000E780C0C7AA89268597000000E78020C903
:10CA80002318A4FC268597000000E78040C82319DE
:10CA9000A4FC268597000000E78060C783D7440088
:10CAA0000A8A231AA4FC858393F7F70F230EF4FC5C
:10CAB0008607BD0793F7073F3301F1408A8A014992
:10CAC0008347C4FD6367F902CE85130584FC232CDC
:10CAD00054FD97000000E78080EA5281130104FCB6
:10CAE000F2506254D2544259B259225A925A216198
:10CAF0008280268597000000E78060C193171900A7
:10CB0000D69705092390A7001379F90F55BF8280A6
:10CB10009797FF1F938747309C43D847A167938718
:10CB2000A702631AF70A397106DE22DC26DA8000D2
:10CB30004AD84ED652D456D23285B28497000000DD
:10CB4000E780C0BAAA89268597000000E78020BC4C
:10CB5000FD572318A4FC26852319F4FC9700000038
:10CB6000E780E0BA83D744000A8A231AA4FC8583AD
:10CB700093F7F70F230EF4FC8607BD0793F7073FE3
:10CB80003301F1408A8A01498347C4FD6367F90292
:10CB9000CE85130584FC232C54FD97000000E7800C
:10CBA00000DE5281130104FCF2506254D254425907
:10CBB000B259225A925A216182802685970000003C
:10CBC000E780E0B493171900D69705092390A700D2
:10CBD0001379F90F55BF82809797FF1F9387C7235B
:10CBE0009C43D847A16789076310F70A397106DEAD
:10CBF00022DC26DA80004AD84ED652D456D232856C
:10CC0000328997000000E78060AEAA894A859700C4
:10CC10000000E780C0AF835749000A8A2318A4FCAC
:10CC2000858393F7F70F230CF4FC8607BD0793F772
:10CC3000073F3301F1408A8A8144834784FD63E7DB
:10CC4000F402CE85130584FC232A54FD97000000CE
:10CC5000E780E0D25281130104FCF2506254D254B6
:10CC60004259B259225A925A216182804A859700CC
:10CC70000000E780C0A993971400D69785042390FD
:10CC8000A70093F4F40F55BF82809797FF1F9387F7
:10CC9000A7189C43D847A1679387E704631EF70A48
:10CCA000397106DE22DC26DA80004AD84ED652D40C
:10CCB00056D23285B28497000000E78020A3AA896B
:10CCC000268597000000E78080A42318A4FC268511
:10CCD00097000000E780A0A3231AA4FC26859700F4
:10CCE0000000E780C0A283D744000A8A2319A4FC6D
:10CCF000858393F7F70F230EF4FC8607BD0793F7A0
:10CD0000073F3301F1408A8A01498347C4FD6367C5
:10CD1000F902CE85130584FC232C54FD97000000F6
:10CD2000E780E0C55281130104FCF2506254D254F2
:10CD30004259B259225A925A21618280268597001F
:10CD40000000E780C09C93171900D697050923902F
:10CD5000A7001379F90F55BF82809797FF1F93871C
:10CD6000A70B9C43D847A1679387C704631AF70AA8
:10CD7000397106DE22DC26DA80004AD84ED652D43B
:10CD800056D23285B28497000000E7802096AA89A7
:10CD9000268597000000E7808097FD572318A4FCA4
:10CDA0002685231AF4FC97000000E780409683D77D
:10CDB00044000A8A2319A4FC858393F7F70F230EF6
:10CDC000F4FC8607BD0793F7073F3301F1408A8AD9
:10CDD00001498347C4FD6367F902CE85130584FCCE
:10CDE000232C54FD97000000E78060B952811301A5
:10CDF00004FCF2506254D2544259B259225A925A07
:10CE000021618280268597000000E780409093177B
:10CE10001900D69705092390A7001379F90F55BF7C
:10CE200082809797FF1F938727FF9C43D847A1676E
:10CE3000DD076317F7041753FFFFE702432A7971F1
:10CE40003285328497000000E780408A2AC6228516
:10CE500097000000E780A08B2311A1022285970094
:10CE60000000E780A088B2452300A10228089700AF
:10CE70000000E780C0B045611753FFFF67006328DB
:10CE800082809797FF1F938727F99C43D847A16714
:10CE9000938787046317F7041753FFFFE7022324E0
:10CEA00079713285328497000000E78020842AC699
:10CEB000228597000000E78080852311A10222854A
:10CEC00097000000E7808082B2452300A102280875
:10CED00097000000E780A0AA45611753FFFF670095
:10CEE000432282809797FF1F938707F39C43D8477D
:10CEF000A1679387A7046312F7021753FFFFE702A6
:10CF0000031E01112800814597000000E78020A73B
:10CF100005611753FFFF6700C31E82809797FF1FAD
:10CF2000938787EF9C43D847A1679387570263197C
:10CF3000F7021753FFFFE702831A0111328597F0BA
:10CF4000FFFFE780A07A2308A10081452800970011
:10CF50000000E780C0A205611753FFFF6700631A56
:10CF600082809797FF1F938727EB9C43D847A16741
:10CF70009387E702631BF7041753FFFFE7022316AB
:10CF800001113285328497F0FFFFE7804078AA8450
:10CF9000228597F0FFFFE7808077854709E92285A2
:10CFA00097F0FFFFE78080744205B337A0002800A8
:10CFB0008145231891003ECA97000000E780209C1D
:10CFC00005611753FFFF6700C31382809797FF1F08
:10CFD000938787E49C43D84799476313F70817530F
:10CFE000FFFFE702C30F79713285328497F0FFFFAC
:10CFF000E780C06F2AC6228597F0FFFFE780207187
:10D000002310A102228597F0FFFFE780206E230105
:10D01000A102228597F0FFFFE780406DA301A102E6
:10D02000228597F0FFFFE780606C2302A102228532
:10D0300097F0FFFFE780806B2313A102228597F012
:10D04000FFFFE780A06AB2452314A10228089700D9
:10D050000000E780C09245611753FFFF6700630A35
:10D0600082809797FF1F938727DB9C43D847A16750
:10D070009387C7036313F7081753FFFFE7022306DD
:10D0800079713285328497F0FFFFE78020662AC6E7
:10D09000228597F0FFFFE78080672310A102228599
:10D0A00097F0FFFFE780A0662311A102228597F089
:10D0B000FFFFE780A0632302A102228597F0FFFF14
:10D0C000E780C062A302A102228597F0FFFFE780FC
:10D0D000E0612303A102228597F0FFFFE780006152
:10D0E000B245A303A102280897000000E780208929
:10D0F00045611753FFFF6700C30082801753FFFF8E
:10D10000E702E3FD01112A8497F0FFFFE780005E4C
:10D11000AA84228597F0FFFFE780605F228597F061
:10D12000FFFFE780C05E035744008D4763F7E700C9
:10D13000228597F0FFFFE780805D228597F0FFFF53
:10D14000E780E05C2800A68597000000E780208348
:10D1500005611753FFFF6700C3FA9797FF1F938777
:10D16000A7CB9C43D847A167FD07631FF700175360
:10D17000FFFFE702C3F6328597000000E78040F822
:10D180001753FFFF6700E3F782809797FF1F93878E
:10D19000A7C89C43D847A167E5076315F70817534D
:10D1A000FFFFE702C3F379713285328497F0FFFF06
:10D1B000E780C0532AC6228597F0FFFFE7802055FD
:10D1C000228597F0FFFFE78080542310A10222857B
:10D1D00097F0FFFFE780A053520551812311A10270
:10D1E00022852302010297F0FFFFE7802050A3026F
:10D1F000A102228597F0FFFFE780404F2303A102A1
:10D20000228597F0FFFFE780604EB245A303A1029D
:10D21000280897F0FFFFE780807645611753FFFFEE
:10D22000670023EE82809797FF1F9387E7BE9C439A
:10D23000D847A1679387E703631FF7001753FFFFE2
:10D24000E702E3E9328597000000E78060EB1753BF
:10D25000FFFF670003EB82809797FF1F9387C7BB91
:10D260009C43D847A16793874704631EF70217536F
:10D27000FFFFE702C3E679713285328497F0FFFF42
:10D28000E780C0462AC6228597F0FFFFE780204846
:10D29000B245280897F0FFFFE780606E456117539D
:10D2A000FFFF670003E682809797FF1F9387C7B64B
:10D2B0009C43D847A167938787026310F7041753ED
:10D2C000FFFFE702C3E179713285328497F0FFFFF7
:10D2D000E780C0412AC6228597F0FFFFE780004122
:10D2E000B2452300A102280897F0FFFFE7802069DC
:10D2F00045611753FFFF6700C3E082801753FFFFAC
:10D30000E702E3DD011197F0FFFFE780203EAA85E9
:10D31000280097F0FFFFE780806605611753FFFF45
:10D32000670023DE9797FF1F938707AF9C43D8477B
:10D33000A167D107631FF7001753FFFFE70223DA46
:10D34000328597000000E780A0FB1753FFFF6700BE
:10D3500043DB82809797FF1F938707AC9C43D84796
:10D36000A167C507631FF7001753FFFFE70223D725
:10D37000328597000000E780A0F81753FFFF670091
:10D3800043D882809797FF1F938707A99C43D8476C
:10D39000A167B907631FF7001753FFFFE70223D404
:10D3A000328597000000E780A0F51753FFFF670064
:10D3B00043D582809797FF1F938707A69C43D84742
:10D3C000A167AD07631FF7001753FFFFE70223D1E3
:10D3D000328597000000E780A0F21753FFFF670037
:10D3E00043D282809797FF1F938707A39C43D84718
:10D3F00089476318F7021753FFFFE70243CE011175
:10D40000328532C897F0FFFFE780402EAA852800BA
:10D4100097F0FFFFE780A05605611753FFFF6700F5
:10D4200043CE82809797FF1F9387079F9C43D847DF
:10D43000A1678D076311F7041753FFFFE70223CAA3
:10D4400001113285328497F0FFFFE780202A13060E
:10D450006100AA844C00228597300000E7800023F9
:10D460002800A68597F0FFFFE780605105611753FC
:10D47000FFFF670003C982809797FF1F9387079A72
:10D480009C4381CFDC4391CB1753FFFFE70223C5B9
:10D4900082971753FFFF6700C3C682801753FFFFB1
:10D4A000E702E3C379713C08AE843ED2A165B707B9
:10D4B0000A002A843ED448103C08DD053ED636C416
:10D4C00032C63AC297D0FFFFE780402C124748107F
:10D4D000BA8597F0FFFFE780C01332464810B28547
:10D4E00097F0FFFFE780E014A2464810B68597F05A
:10D4F000FFFFE7800012501001478146A685228574
:10D5000097D0FFFFE780E04D45611753FFFF6700AD
:10D5100043BF1753FFFFE70283BC01117C000329BF
:10D52000C501AE843ECAA165B70707002A843ECC78
:10D5300048087C00C5053ECE97D0FFFFE780002558
:10D540008345D900480897F0FFFFE780800C50081A
:10D5500001478146A685228597D0FFFFE780604876
:10D5600005611753FFFF6700C3B91753FFFFE702B9
:10D5700003B783C7950093F7F707A384F5009700D7
:10D580000000E78040F91753FFFF670083B7175388
:10D59000FFFFE702C3B479713C08AE843ED2A165B7
:10D5A000B70709002A843ED448103C0893854504F7
:10D5B0003ED632C636C497D0FFFFE780201DA24674
:10D5C0004810B68597F0FFFFE780A0043246481068
:10D5D000B28597F0FFFFE780C005501001478146F4
:10D5E000A685228597D0FFFFE780A03F45611753AE
:10D5F000FFFF670003B11753FFFFE70243AE83C786
:10D60000950041112A8493F7F707A384F50032852A
:10D610002EC697F0FFFFE780800F85672AC46370EE
:10D62000F50297700000E78060E82246B24509EDF8
:10D6300011478146228597000000E78060E641019E
:10D640001753FFFF6700E3AB01478346F501DDB7E2
:10D650001753FFFFE70203A701113C003ECAB707BB
:10D660000A003ECC3C003ECE83C79500AA89328595
:10D6700093F7F707A384F5002E8497F0FFFFE78068
:10D6800000098567637DF504A165AA8493858504F7
:10D69000480897D0FFFFE780600F2685977000004D
:10D6A000E780C0E02A8929E19145480897F0FFFF0B
:10D6B000E78020F6A685480897F0FFFFE78060F72F
:10D6C000CA85480897F0FFFFE780A0F4014781462C
:10D6D0005008A2854E8597D0FFFFE7808030056116
:10D6E0001753FFFF670043A18145480897F0FFFFEC
:10D6F000E78020F20349090275BF1753FFFFE702D5
:10D70000639C79711C103ECAB7070F003ECC404D98
:10D710001C10AA84AE894808994532C636893ECE87
:10D7200097D0FFFFE780800632464808B28597F021
:10D73000FFFFE78000EE630C0902A545480897F05B
:10D74000FFFFE780C0E62546CA8597200100E780F5
:10D7500060A3500801478146CE85268597D0FFFFFC
:10D76000E780202845611753FFFF6700E398835542
:10D77000C402480897F0FFFFE780A0EB0355E402DE
:10D78000814505C5854785456301F502C167FD17DC
:10D790009305F00F630BF5007D1597700000E7808F
:10D7A000608D9305150093F5F50F480897F0FFFF7E
:10D7B000E78020E683450403480897F0FFFFE780F1
:10D7C00040E583451403480897F0FFFFE78060E4D5
:10D7D00083552403480897F0FFFFE78080E58355D1
:10D7E0004403480897F0FFFFE780A0E49DB7175374
:10D7F000FFFFE702C38E83C795008146014693F77A
:10D80000F707A384F50097000000E78040EF175367
:10D81000FFFF6700038F1753FFFFE702438C797107
:10D820003E841C103ECA2E89B7070F00A1653ECC6E
:10D83000FD051C10AA84480842C03AC23ECE36C438
:10D8400032C697D0FFFFE78060F432464808B285C1
:10D8500097F0FFFFE780E0DBA2464808B68597F027
:10D86000FFFFE78000DD12474808BA8597F0FFFF09
:10D87000E78020DC0248630C08029145480897F0D5
:10D88000FFFFE780C0D21146A28597200100E78004
:10D89000608F500801478146CA85268597D0FFFFD3
:10D8A000E780201445611753FFFF67008385894592
:10D8B000480897F0FFFFE78080CF834704002300EC
:10D8C000F50083471400A300F500E1B71743FFFFFD
:10D8D000E702437F83C7950001112A8A93F7F70770
:10D8E000A384F5003285AE8432C697F0FFFFE7804F
:10D8F00000E232462A89328597F0FFFFE78000DF99
:10D9000085676373F902AA894A8597700000E780EA
:10D91000E0B92A8419ED114781464A86A6855285C9
:10D9200097000000E780C0B705611743FFFF67005D
:10D93000A37C9387E9FF93F7F70F0547E366F7FEAC
:10D940008347F50195EB8947E380F9FE8346F401AF
:10D95000528501474A86A68597000000E78040B4BB
:10D96000A167D90748083ECC230A010002CE9700E0
:10D970000000E780A0B04DBF639EE7008947639E2B
:10D98000F90093071020231FF50097700000E7802F
:10D9900000B76DBF0947E39BE7FA8D47E398F9FAB3
:10D9A000228597700000E780C0DE9787FF1F93876E
:10D9B000E7659C4399E79787FF1F9387E74E9C4352
:10D9C00099C703D5040097800000E780E0CD231FAE
:10D9D000040022855DBF1743FFFFE702437001117A
:10D9E0003C003ECAB7070B003ECC3C003ECE83C78E
:10D9F00095002A89328593F7F707A384F500AE8452
:10DA000097F0FFFFE780A0D093170501C187635A05
:10DA1000F006A1652A849385E502480897D0FFFFA8
:10DA2000E780C0D6A285480897F0FFFFE78060C076
:10DA30009787FF1F938747479C43A9EB0144937542
:10DA4000F40F480897F0FFFFE780A0BC935584408F
:10DA500093F5F50F480897F0FFFFE78080BB9355DB
:10DA6000044193F5F50F480897F0FFFFE78060BA8F
:10DA7000014781465008A6854A8597D0FFFFE78079
:10DA800040F605611743FFFF6700A36741658546C0
:10DA90000546A2857D1597500000E780A0BC59DDA2
:10DAA000510597000100E780C08E130440063344FF
:10DAB000850271B71743FFFFE70263620111B707E1
:10DAC00006003EC683C7950021642A8993F7F707AD
:10DAD000A384F500AE8428009305A4040AC40AC8F0
:10DAE00097D0FFFFE78080CA300001478146A685B6
:10DAF0004A8597D0FFFFE780C0EE97E0FFFFE78001
:10DB0000E01113049404480822CC230A010002CE39
:10DB100097000000E780809605611743FFFF6700CC
:10DB2000435E1743FFFFE702E359C1642A890144BA
:10DB30009789FF1F9389094F130A8002FD1497E00C
:10DB4000FFFFE780E0BD6347A40001451743FFFFE7
:10DB50006700835AB307440303A7C90ABA9703D7D8
:10DB600007006306970083D7270063842701050415
:10DB7000F9B70545E1BF1743FFFFE702A3542A8A1F
:10DB80002E8999C123A0050081498144978AFF1FEE
:10DB9000938A0A29614B97E0FFFFE780A0BE63C725
:10DBA000A4004E851743FFFF6700035533846403C9
:10DBB00083A70A003E948357040099E76304090091
:10DBC000232089008504C1BF4146D2851305440046
:10DBD00097100100E780A05875F5A289E5B71743B3
:10DBE000FFFFE702234E39717C083ED4B7070A00D5
:10DBF0003ED67C083ED883C795002A8A328593F7A3
:10DC0000F707A384F5002E8932C697F0FFFFE7805F
:10DC100000B085676373F5083246AA84328597F0B1
:10DC2000FFFFE780A0AC8547AA8963E8A706A16546
:10DC300093858504281097D0FFFFE78020B52685BF
:10DC400097700000E78080862A8429ED914528108E
:10DC500097F0FFFFE780E09BA685281097F0FFFF75
:10DC6000E780209DCE85281097F0FFFFE780609A1F
:10DC7000014781463010CA85528597D0FFFFE78063
:10DC800040D6A1679387770448183EDC230A010237
:10DC900002DE97F0FFFFE780607E21611743FFFF00
:10DCA000670083458145281097F0FFFFE780609665
:10DCB000A685281097F0FFFFE780A0979787FF1FA2
:10DCC0009387076D9C4381CB22856389090097D098
:10DCD0000000E78080238345040271B797D00000DD
:10DCE000E7800022CDBF1743FFFFE702A33D83C7B4
:10DCF00095004111AA8993F7F707A384F5003285AF
:10DD0000AE84328A97F0FFFFE78060A08567637F6B
:10DD1000F5022A8997600000E78040792A849146BD
:10DD200031C58347F50105476387E70291C70D4772
:10DD30006366F704AD461DA89305050303250A0095
:10DD4000414697100100E78080410DE941011743EA
:10DD5000FFFF6700633A9305950803250A004146D3
:10DD600097100100E780A03F814669F54A86A685A5
:10DD70004E8597000000E780C081C9BF83250A0057
:10DD80001305940897700000E780E02819C1C14688
:10DD9000F1BF9787FF1F938767279C4399E7978772
:10DDA000FF1F938767109C4399C7228597800000C7
:10DDB000E780608969FD8547A30FF400228597B04D
:10DDC0000000E780A083228597600000E780207331
:10DDD0004E8581464A86A68597F0FFFFE780607BE7
:10DDE000A1679387570448003EC42302010002C67E
:10DDF00097F0FFFFE780806891BF1743FFFFE702BE
:10DE0000832B83C795004111AA8993F7F707A38451
:10DE1000F50032852E89B28A97F0FFFFE780208FC8
:10DE200085676374F50EAA8497600000E780006838
:10DE30002A840DED416B014A978BFF1F938B8B1E3C
:10DE4000130C400E7D1B19A833048A0383A70B0B08
:10DE50003E948357C40163836705050A97E0FFFF7B
:10DE6000E780008BE342AAFE95460DA08357C501CB
:10DE7000639697029305050303A50A004146971090
:10DE80000100E780C02D994611E181462686CA85AA
:10DE90004E8597F0FFFFE780C06F85A883A50A0035
:10DEA0001305040397700000E780E016C14679FD72
:10DEB0002285231E940097A00000E780207422850D
:10DEC00097600000E780A0639787FF1F9387474C08
:10DED0009C43A9C323000402228597D00000E78059
:10DEE00080EF4E8581462686CA8597F0FFFFE78042
:10DEF000406AA1679387070448003EC423020100DB
:10DF000002C697F0FFFFE780605741011743FFFF0C
:10DF10006700E31D89472300F402E1B7397106DE8B
:10DF200022DC4AD8800052D456D25AD026DA4ED6B5
:10DF30005ECE2E8A32892A8B97D0FFFFE780407A07
:10DF40000605710541998A8A3301A140232224FCE8
:10DF5000231404FC97D0FFFFE780807883479A0062
:10DF60000605350593F7F7072315A4FCA304FA006B
:10DF70004A85232624FC97E0FFFFE780407993172A
:10DF80000501C1876340F0025681130104FCF25081
:10DF90006254D2544259B259225A925A025BF24BFD
:10DFA00021618280AA844A8597E0FFFFE78020767E
:10DFB000AA894A8597E0FFFFE7806075A165938590
:10DFC000C5022A89130544FC97C0FFFFE780007C47
:10DFD000268597C0FFFFE7804070854511C94A86B6
:10DFE000CE8597C0FFFFE780C069AA8B21E98945EC
:10DFF000130544FC97E0FFFFE780A061A6851305A9
:10E0000044FC97E0FFFFE780C062CE85130544FC27
:10E0100097E0FFFFE780E061CA85130544FC97E0C5
:10E02000FFFFE780006101478146130644FCD2856B
:10E030005A8597D0FFFFE780C09AB9B7814513058D
:10E0400044FC97E0FFFFE780C05CA685130544FC15
:10E0500097E0FFFFE780E05DCE85130544FC97E085
:10E06000FFFFE780005DCA85130544FC97E0FFFFD2
:10E07000E780205C814497D0FFFFE7806066E3D4AF
:10E08000A4FA83A70B0113971400BA9783D507004E
:10E0900099C5130544FC97E0FFFFE780805985048C
:10E0A000D9BF797106D622D44AD000184ECE52CCB0
:10E0B00056CA26D25AC8AE893289AA8A97D0FFFF9B
:10E0C000E78000620605690541990A8A3301A1408B
:10E0D000232A24FC231C04FC97D0FFFFE780406028
:10E0E00083C7990006052D0593F7F707231DA4FCA8
:10E0F000A384F9004A85232E24FC97E0FFFFE780E4
:10E10000006193170501C187634FF000528113012D
:10E1100004FDB250225492540259F249624AD24A42
:10E12000424B45618280AA844A8597E0FFFFE780E1
:10E13000005EA1659385A5022A89130544FD97C059
:10E14000FFFFE780A064268597C0FFFFE780E058C7
:10E15000854509C9CA8597C0FFFFE78080552A8B8E
:10E1600029E18945130544FD97E0FFFFE780604AF8
:10E17000A685130544FD97E0FFFFE780804BCA8525
:10E18000130544FD97E0FFFFE780A04A0147814661
:10E19000130644FDCE85568597D0FFFFE780608447
:10E1A000B5B78145130544FD97E0FFFFE780604662
:10E1B000A685130544FD97E0FFFFE7808047CA85E9
:10E1C000130544FD97E0FFFFE780A046814497D008
:10E1D000FFFFE780E050E3DBA4FA83270B011397EE
:10E1E0001400BA9783D5070099C5130544FD97E03D
:10E1F000FFFFE78000448504D9BF1743FFFFE70214
:10E2000003EE83474500404DD5EFFD575DC483467F
:10E21000940009476363D70A0346B400854663EE5A
:10E22000C6088306E40063CA06085C45F9562390D5
:10E23000D7009787FF1F83C7E7BE99E3A304E400D5
:10E240009787FF1F938747C69C4381E78947A306AB
:10E25000F4009787FF1F9387A7139C4381E78947A3
:10E260002306F4009705000093854506AA8413054C
:10E27000040197F00000E780600FFD57231AF402B5
:10E2800081471CDC01489787FF1F23A987B8978720
:10E29000FF1F9387E7B8232E040304C0804397D061
:10E2A000FFFFE780204E61463306C5028145228587
:10E2B0009740FFFFE780A0E581473E851743FFFFBA
:10E2C000670023E4FD57D5BF1743FFFFE70223E1B3
:10E2D0002A840355450297600000E780201D19E558
:10E2E000231E04001743FFFF6700A3E18357E401E7
:10E2F000F5DB930504FF17450100130525EF97E0B3
:10E300000000E7802014F9BF1743FFFFE70223DD79
:10E310002E89A16541119385E5032A8436C432C64E
:10E32000BE843AC297C0FFFFE7804046124722856D
:10E33000BA8597E0FFFFE780C02D32462285B2857F
:10E3400097E0FFFFE780E02EA2462285B68597E0A2
:10E35000FFFFE780002E630309029145228597E0C5
:10E36000FFFFE780C0241146A68597100100E780D3
:10E3700060E141011743FFFF6700A3D8894522856B
:10E3800097E0FFFFE780A02283C704002300F50089
:10E3900083C71400A300F500E9BF1743FFFFE7029E
:10E3A00003D483C79500444D054793F7F707A3842B
:10E3B000F5001C42411183C707006367F7062E84EE
:10E3C0002A89B1C003C7D400630FF7021787FF1F64
:10E3D000130787AD184305C3A386F40097A0000078
:10E3E000E780804983C7D40099E741657D15974050
:10E3F0000000E780802F83D72403918B89C797E0A3
:10E400000000E78000134A85A28597F0FFFFE780B0
:10E410008010A167C10748003EC42302010002C664
:10E4200097F0FFFFE780800541011743FFFF67007A
:10E4300043CD1743FFFFE70283CA03D745008D474B
:10E44000AA8441112E8432892E8563E3E70297E086
:10E45000FFFFE780C02BAA8523000900268597C00F
:10E46000FFFFE780002541011743FFFF670063C9F5
:10E4700097E0FFFFE780A0292AC6228597E0FFFFEB
:10E48000E780E028B24585472A862300F9002685E3
:10E4900097C0FFFFE780E01EF9B7397106DE22DC86
:10E4A00026DA80004ED652D456D24AD85AD05ECE02
:10E4B000AE89B284AA8A97D0FFFFE7806021060563
:10E4C0001305250241990A8A3301A140232224FC25
:10E4D000231404FC97D0FFFFE780801F83C79900B7
:10E4E00006054D0593F7F7072315A4FCA384F9004F
:10E4F0002685232624FC97E0FFFFE7804021931721
:10E500000501C1876340F0025281130104FCF250FF
:10E510006254D2544259B259225A925A025BF24B77
:10E5200021618280AA8B03AB040097C0FFFFE780C4
:10E53000C01A51E583D7440001498544F11793B7C8
:10E540001700A301F4FC834734FCA165C9C7938578
:10E55000E504130544FC97C0FFFFE7802023A68550
:10E56000130544FC97E0FFFFE780A00ADE85130552
:10E5700044FC97E0FFFFE780C00B834734FC114663
:10E5800091E30946DA85130544FC97E0FFFFE78035
:10E5900060058144630A0900416B7D1B97D0FFFF32
:10E5A000E780001363CCA40201478146130644FCB4
:10E5B000CE85568597C0FFFFE780A042B1B7A685FC
:10E5C000130634FC97000000E780E0E69334150062
:10E5D0002A8986048DBF9385C504A5BF8327C900FA
:10E5E00013971400BA9783D5070063886501130554
:10E5F00044FC97E0FFFFE780C003850445B717435D
:10E60000FFFFE70243AB79711C103EC4B7070F0050
:10E610003EC61C103EC883C79500AA8A328593F770
:10E62000F707A384F500AE89328497E0FFFFE78007
:10E63000000E93170501C187635AF0062A8A2285C6
:10E6400097E0FFFFE780A00C2A895285032B040086
:10E6500097C0FFFFE780600839ED8357440081448D
:10E660000544F11793B71700A303F1008345710028
:10E67000DA872287CA865286280097000000E78042
:10E68000E0C8014781463000CE85568597C0FFFF20
:10E69000E7802035A1679387D70348083ECC230A3B
:10E6A000810026CE97F0FFFFE78040DD45611743EC
:10E6B000FFFF6700C3A3A285130671009700000047
:10E6C000E78060D7AA84094455D13544E30055FB5F
:10E6D0004A8597F0FFFFE78000450D4441D901448A
:10E6E00097D0FFFFE780C0FE634DA400C16B0144DB
:10E6F000FD1B97D0FFFFE780A0FD634EA4001544EB
:10E70000B5B7DC4413171400BA9783D707006383A7
:10E7100027030504F1B7D84493171400BA9703D719
:10E720000700631B770123902701268597A000002F
:10E73000E780C0DA01441DBF050465BF1743FFFF32
:10E74000E702439883C7950041112A8A93F7F70798
:10E75000A384F50032852E89328497E0FFFFE7809D
:10E7600000FB93170501C1876353F006AA89228530
:10E7700097E0FFFFE780A0F92311A1004E85832ACF
:10E78000040097C0FFFFE78040F539E58357440058
:10E7900085440144F11793B71700A300F100034823
:10E7A000110003572100D6875285CE862686CA855A
:10E7B00097F0FFFFE7806006A167F10748003EC4BD
:10E7C0002302910022C697F0FFFFE78020CB410192
:10E7D0001743FFFF67004392A285130611009700BD
:10E7E0000000E78040C52A84894455D98357210019
:10E7F00011678544BA97C2071167C1831307F7EF02
:10E80000E36FF7F89787FF1F938747809C4381CB7F
:10E8100085451305210097500000E78060748355FB
:10E8200021002285814497C0FFFFE780A0E125D920
:10E8300023100500228597A00000E78080CC85B7D3
:10E840001743FFFFE702238783C7950041112A8BF7
:10E8500093F7F707A384F50032852E8A328497E078
:10E86000FFFFE780C0EA93170501C1876351F006F7
:10E87000AA8A228597E0FFFFE78060E92A8956850A
:10E88000832B040097C0FFFFE78020E531E5835725
:10E89000440081440544F11793B71700A301F10028
:10E8A00003483100DE875A854A87D6862286D2857C
:10E8B00097F0FFFFE78060F6A167ED0748003EC4D0
:10E8C0002302810026C697F0FFFFE78020BB4101AD
:10E8D0001743FFFF6700A381A2851306310097004D
:10E8E0000000E78040B5AA8409445DD99167CA97C2
:10E8F000C2071167C1831307F7EF0544E362F7FA14
:10E90000CA8597C0FFFFE780E0D3014451F98149F0
:10E9100097D0FFFFE780C0DC63DBA900984893979E
:10E920001900BA9703D7070005EF2390270197D066
:10E93000FFFFE780E0DA1544E384A9F6268597A077
:10E940000000E78000BC9777FF1F9387276C9C43EC
:10E950000144B9D74A8597500000E780005889B72D
:10E9600085097DB71733FFFFE702C37579713E84D0
:10E970007C083EC82E8AB7071400A1653ECAE5058B
:10E980007C08AA89080836C4428932C6BA8AC68475
:10E990003ECC97C0FFFFE78060DFCA85080897E09C
:10E9A000FFFFE78000C732460808B28597E0FFFF07
:10E9B000E78020C8A246630A09049D45080897E03D
:10E9C000FFFFE780C0BE1D4681459730FFFFE7800F
:10E9D000007463890A089145080897E0FFFFE78003
:10E9E00000BD1146A68597000100E780A0791008B8
:10E9F00001478146D2854E8597C0FFFFE78060FEC4
:10EA000045611733FFFF6700236FB685080897E05D
:10EA1000FFFFE78000C21C400808D8439355C70198
:10EA2000858912075183B205D98D97E0FFFFE780F2
:10EA300040C01C40080883C5870097E0FFFFE780BF
:10EA400040BD1C40080883C5A70097E0FFFFE78092
:10EA500040BC1C40080883C5970097E0FFFFE78093
:10EA600040BB85BF8945080897E0FFFFE78020B4D9
:10EA700083C704002300F50083C71400A300F5003A
:10EA8000BDB71733FFFFE702E36383C7950041116A
:10EA9000AA8993F7F707A384F5003285AE84328400
:10EAA00097E0FFFFE780A0C693170501C187635D6C
:10EAB000F0042A89032A040097C0FFFFE780E0C121
:10EAC00019E9835744000548F11793B71700A307C6
:10EAD000F100814631A81306F100A28597000000DD
:10EAE000E78060951DC51C459DC783D6470001483A
:10EAF0000347F10093078500D2884A86A6854E8594
:10EB000097000000E78040E641011733FFFF6700F0
:10EB1000A35E09487DBF1D486DBF1733FFFFE702A5
:10EB2000635A65715C083EC4B7077B013EC65C084A
:10EB30003EC883C795002A8A328593F7F707A384D6
:10EB4000F500AE8997E0FFFFE78040BA8357E10008
:10EB5000E1C78945280097C0FFFFE78020C38145B2
:10EB6000280097E0FFFFE780C0AA97C0FFFFE7807B
:10EB700000C99787FF1F9387A7819C431774FF1FC6
:10EB80000344442AAA843334800099C313642400C4
:10EB90009777FF1F938747319C4399C313644400C1
:10EBA0009777FF1F938787469C4399C3136484001C
:10EBB00083D504002800014997E0FFFFE78060A7A4
:10EBC00083D52400280097E0FFFFE78080A683D547
:10EBD0004400280097E0FFFFE780A0A597D0FFFF43
:10EBE000E78000AB93150501C181280097E0FFFF86
:10EBF000E78020A4A285280097E0FFFFE78060A3BC
:10EC00009C446360F902014781463000CE855285FD
:10EC100097C0FFFFE780E0DC59611733FFFF670013
:10EC2000A34DDC441314490028003E9497E0FFFFF5
:10EC3000E78060968347440003475400890706072E
:10EC4000BA978607E36AF5FC835524002800814AB9
:10EC500097E0FFFFE780E09D83454400280097E0B0
:10EC6000FFFFE780009B83455400280097E0FFFFEB
:10EC7000E780209A8347440063C9FA00814A8347AA
:10EC8000540063C1FA020509A5BF1C4413975A003A
:10EC90002800BA9783D50700850A97E0FFFFE78031
:10ECA0004099C9BF032BC40093975A0028003E9B8C
:10ECB00083552B00850A97E0FFFFE78080978355F7
:10ECC0000B00280097E0FFFFE780A0964DBF1733A9
:10ECD000FFFFE702C3405C4993E717005CC997A0B8
:10ECE0000000E78060B51733FFFF670083411733EB
:10ECF000FFFFE702C33E2E84814597F0FFFFE780C8
:10ED0000C0E705C583570500FD172310F50009C4AA
:10ED1000835725002310F40097000000E78060FB74
:10ED200001451733FFFF6700C33D31457DD82310F0
:10ED30000400C5BF1733FFFFE702C33883C7950040
:10ED400041112A8A93F7F707A384F50032852E89AB
:10ED5000328497E0FFFFE780809B93170501C1870E
:10ED60006356F006AA89C145228597E0FFFFE78038
:10ED7000A0802A8B4E85832A040097C0FFFFE7807E
:10ED8000C09531E983574400231101000544F11770
:10ED900093B71700A300F100814403481100035703
:10EDA0002100D6875285CE862286CA8597F0FFFF3E
:10EDB000E780A0A6A1679387170248003EC42302FC
:10EDC000810026C697E0FFFFE780406B41011733C3
:10EDD000FFFF6700633213061100A28597F0FFFF63
:10EDE000E7806065AA8409E523110100094475B72D
:10EDF000930521005A8597000000E78080EF835734
:10EE000021002A84D9DB9777FF1F938727209C4313
:10EE100081CB85451305210097500000E780401401
:10EE2000835521002685314497C0FFFFE78080810C
:10EE30002DD523100500268597900000E780606C93
:10EE40000144A1BF1733FFFFE702632941112E8957
:10EE50006C00AA8402C697F0FFFFE78000D20DC1C4
:10EE60000357050005072310E50097000000E78021
:10EE700040E681473E8541011733FFFF6700632865
:10EE80003247954765DBCA85268597300000E780C5
:10EE9000800CC147E34005FE3244854741462310BC
:10EEA000F40083570900A685130544002311F400DC
:10EEB00097000100E780002D228545BF1733FFFF33
:10EEC000E702432083C795004111AA8A93F7F70709
:10EED000A384F5003285AE89328497E0FFFFE78096
:10EEE000008393170501C1876356F0062A8AC1453E
:10EEF000228597D0FFFFE7802068AA845285032BE4
:10EF0000040097B0FFFFE780407D31E9835744005C
:10EF1000231101008544F11793B71700A300F100F6
:10EF200001440348110003572100DA875685D28631
:10EF30002686CE8597F0FFFFE780208EA167938716
:10EF4000070248003EC42302910022C697E0FFFF5B
:10EF5000E780C05241011733FFFF6700E319A28524
:10EF60001306110097F0FFFFE780E04C2A8409E5C3
:10EF700023110100894475B7268593052100970068
:10EF80000000E78060ECAA8449FD835521002285BA
:10EF900097B0FFFFE780006B49F5014997C0FFFF7D
:10EFA000E7800074635DA900184893171900BA97A9
:10EFB00003D707000DEF035721002390E70097C008
:10EFC000FFFFE780E071630625039777FF1F9387B4
:10EFD000E7039C4399C70355210097500000E78041
:10EFE000C0EF228597900000E780A0511DBF050962
:10EFF00075B795443DB705C19307F00F630FF50052
:10F00000C547630CF5009307F5FF05453315F5007B
:10F010004205418182800145828041657D15828063
:10F02000B9E91733FFFFE702830B03450603328478
:10F0300097000000E78060FC9305803EB305B502B1
:10F04000C205C18181CD0357E402854763F8E7001B
:10F050001305040197E00000E78060418357E40254
:10F0600041677D176385E700FD172317F402173307
:10F07000FFFF6700030982801733FFFFE702A30346
:10F08000004283C79500444D0349140093F7F707E6
:10F09000A384F50083470400220911673369F9004E
:10F0A000A167B347F90041112A8BAE8A63ECE70EE2
:10F0B000834724001307C00EB91793F7F70F637344
:10F0C000F71003473400C14763EEE70E834744005F
:10F0D0001307E00793C707086371F70C834984009F
:10F0E00083477400A209B3E9F900856763F7F90A59
:10F0F000034A6400834754004E85220A336AFA00AB
:10F1000097500000E780803A61C123962403834B27
:10F110003400137AFA00239A340323887403239962
:10F12000440393890401631C090023A60402239865
:10F1300004024E8597E00000E780A0353DA003491A
:10F1400024004A8597000000E78020EB2397A40263
:10F15000834744004E85A388F402E38D0BFCE30B48
:10F1600009FC97E00000E780602E97900000E780A0
:10F17000407281460146D6855A8597E0FFFFE780B9
:10F180000058A167938797033EC4230201004800FB
:10F1900002C697E0FFFFE780602E41011733FFFFB3
:10F1A0006700E3F48544A2862686D6855A8597E0D3
:10F1B000FFFFE780C054A167938797033EC42302F3
:10F1C0009100F1B7BD44C5B79144F1BF1733FFFFBC
:10F1D000E70243EF01111C08404D3EC2B7070F0084
:10F1E0003EC41C083EC62A89AE8997C0FFFFE7804F
:10F1F00000D7585C1C5C6346B70E6394E50063E27D
:10F20000A70E3385A740B3B7A700B305B7401306D1
:10F21000803E81469D8D97000100E780C0B6931423
:10F220000501C180A1659385C503480097B0FFFF24
:10F23000E780C0558145480097D0FFFFE780603DDB
:10F2400083550404480097D0FFFFE780803E835534
:10F250002404480097D0FFFFE780A03D814589CC7A
:10F26000C167FD179305F00F6388F400268597505A
:10F270000000E78020E0AA85480097D0FFFFE780E4
:10F28000403903554404814501CDC167FD179305FD
:10F29000F00F6307F50097500000E780A0DDAA8516
:10F2A000480097D0FFFFE780C036834564044800DC
:10F2B00097D0FFFFE780E03583457404480097D07E
:10F2C000FFFFE7800035500001478146CE854A8523
:10F2D00097B0FFFFE780E07005611733FFFF67001D
:10F2E000A3E1814481B71733FFFFE70243DF83C700
:10F2F000950093F7F707A384F50097000000E780D7
:10F3000020ED1733FFFF6700C3DF1733FFFFE7026E
:10F3100063DB83C795004111404D93F7F707A38442
:10F32000F5002A8A3285B284AE8997D0FFFFE78044
:10F33000003E2A8B268597D0FFFFE780403D2A8933
:10F34000268597D0FFFFE780603A93170B0163CAC9
:10F350000702E177CA97C207C183116763E3E70237
:10F3600093070910C207C1831307B00F637BF7002F
:10F3700093170901C187AA8A634AF000C54763FE53
:10F38000570141011733FFFF670003D797B0FFFF15
:10F39000E7802025E31725FFD5B763080B02630636
:10F3A0000902814463890A02B7077F0023106405BC
:10F3B000231124057CC0568597000000E780E0C338
:10F3C0009304803EB304950239A0B7077F00232041
:10F3D00004047CC081440355240497E00000E780C6
:10F3E000E0A2A1C497C0FFFFE78060B7269593D73E
:10F3F000F44133379500AE97BA9708DC5CDCCE85D4
:10F40000528597000000E780A0DC99E023220404E5
:10F41000A1679387B70348003EC42302010002C6D8
:10F4200097E0FFFFE7808005A9BF814701481CDC0A
:10F43000232E0403E9B71733FFFFE70243CA97C03F
:10F44000FFFFE7802034E1473305F50291459750EF
:10F450000000E78040C4E55711C59777FF1F23A13F
:10F46000A79C81473E851733FFFF670083C9173389
:10F47000FFFFE702C3C69777FF1F9387279A804352
:10F480003DC0835704046390A70683572404639CFC
:10F49000B7043689B28497C0FFFFE78040AC5C5C5C
:10F4A00063C3B7046395B7001C5C63EEA702834790
:10F4B000640463F3F400A6872303F404834774040D
:10F4C00063F39700A687A303F404835744044167BA
:10F4D0007D176385E70085072312F4043C4481C748
:10F4E000CA85268582971733FFFF670083C1977708
:10F4F000FF1F9387A7929C43014599C303C58700CB
:10F5000082801733FFFFE70283BD0111B7070700B1
:10F510003EC683C79500584D0AC493F7F7070AC83B
:10F52000A384F5002A89AE8411CB1C4283C707004F
:10F530002304F70097900000E780003421649305CE
:10F540005402280097B0FFFFE78040249700000096
:10F55000E78020FAAA85280097D0FFFFE780600B9C
:10F56000300001478146A6854A8597B0FFFFE780B6
:10F57000404713044402480822CC230A010002CE6B
:10F5800097E0FFFFE78080EF05611733FFFF67001B
:10F5900043B71733FFFFE70283B401117C003ECA73
:10F5A000B70707003ECC7C003ECE83C795002E8473
:10F5B000AA8493F7F707A384F500A1659385550204
:10F5C000480897B0FFFFE780601C97000000E780C5
:10F5D00040F2AA85480897D0FFFFE78080035008D3
:10F5E00001478146A285268597B0FFFFE780603FEF
:10F5F00005611733FFFF6700C3B09777FF1F93873D
:10F60000E7819C43094599C303C59700828097779A
:10F61000FF1F9387A7809C43094599C303C5D70063
:10F6200082809767FF1F9387677F9C43014599C33B
:10F6300003C5A70082801733FFFFE702A3A80111CB
:10F64000B70708003EC683C79500404D0AC493F72C
:10F65000F7070AC8A384F5002A89AE8429C4144296
:10F66000854703C7060063E0E70A8347940009461D
:10F6700081496380C702B307F740A304E400B339AC
:10F68000F00083C716002305F40097900000E78080
:10F69000A01E03572403058B19C76386090097D062
:10F6A0000000E78000E9216493058402280097B0F8
:10F6B000FFFFE780A00D97000000E78040F4AA85D7
:10F6C000280097D0FFFFE780C0F497000000E78094
:10F6D00080F5AA85280097D0FFFFE78080F30147D7
:10F6E00081463000A6854A8597B0FFFFE780602FEE
:10F6F00013047402480822CC230A010002CE97E0CA
:10F70000FFFFE780A0D705611733FFFF6700C39EA7
:10F710001733FFFFE702A39C01117C003ECAB70725
:10F7200008003ECC7C003ECE83C795002E84AA8480
:10F7300093F7F707A384F500A16593858502480830
:10F7400097B0FFFFE780800497000000E78020EB80
:10F75000AA85480897D0FFFFE780A0EB970000003C
:10F76000E78060ECAA85480897D0FFFFE78060EA51
:10F77000500801478146A285268597B0FFFFE780A4
:10F78000402605611733FFFF6700A3979767FF1FA8
:10F790009387C7689C43014599C303C5B70082801E
:10F7A0001733FFFFE702A3930111B70707003EC617
:10F7B00083C79500404D0AC493F7F7070AC8A3848E
:10F7C000F5002A89AE8405C81C42054783C7070097
:10F7D0006368F7060347B400630FF700A305F4005E
:10F7E00097900000E78040098347B400B9CF97D0D5
:10F7F000FFFFE78000BF21649305B400280097B0A5
:10F80000FFFFE780A0F897000000E78060F8AA8576
:10F81000280097D0FFFFE780C0DF01478146300016
:10F82000A6854A8597B0FFFFE780A01B29044808FA
:10F8300022CC230A010002CE97E0FFFFE78000C43C
:10F8400005611733FFFF6700C38B97D0FFFFE78089
:10F85000E0BF55B71733FFFFE702638801117C0053
:10F860003ECAB70707003ECC7C003ECE83C795005A
:10F870002E84AA8493F7F707A384F500A165AD054C
:10F88000480897B0FFFFE78060F097000000E7802E
:10F8900020F0AA85480897D0FFFFE78080D750085E
:10F8A00001478146A285268597B0FFFFE780601358
:10F8B00005611733FFFF6700C3849767FF1F9387B6
:10F8C000E7559C43094599C303C5C7008280173398
:10F8D000FFFFE702C38001117C00AE843ECAA16530
:10F8E000B70707002A843ECCD1057C0048083ECEED
:10F8F00097B0FFFFE78080E997000000E78020FCD9
:10F90000AA85480897D0FFFFE780A0D0500801479C
:10F910008146A685228597B0FFFFE780800C0561B0
:10F920001723FFFF6700E37D1723FFFFE702237B19
:10F9300083C7950093F7F707A384F50097000000AD
:10F94000E78020F91723FFFF6700A37B1723FFFF42
:10F95000E702437783C795000329C501411193F757
:10F96000F707A384F5001C4283C90700854763E6B7
:10F9700037079777FF1F9387A7A19C432E84AA84FC
:10F9800085CF97000000E78080F389476306F50282
:10F99000630409028347C9006380370323063901E2
:10F9A00097900000E78040ED83572903898B89C732
:10F9B00097D00000E780E0B72685A2859700000079
:10F9C000E78020F1A167CD0748003EC42302010073
:10F9D00002C697E0FFFFE78060AA41011723FFFFFF
:10F9E000670083719767FF1F938747439C431D45BB
:10F9F00099C303C5E70082801723FFFFE702236E48
:10FA00000111B70707003EC683C79500584D0AC4C9
:10FA100093F7F7070AC8A384F5002A89AE8415C7AF
:10FA20001C4283C7070093968701E18663C40606DC
:10FA300085466381D7068346E7006388F60023077F
:10FA4000F70097900000E78020E321649305E4002D
:10FA5000280097B0FFFFE78060D397000000E780A1
:10FA6000A0F8AA85280097D0FFFFE78080BA014759
:10FA700081463000A6854A8597B0FFFFE78060F693
:10FA80003504480822CC230A010002CE97E0FFFF8C
:10FA9000E780C09E05611723FFFF67008366172379
:10FAA000FFFFE702C36301117C003ECAB7070700EE
:10FAB0003ECC7C003ECE83C795002E84AA8493F76B
:10FAC000F707A384F500A165B905480897B0FFFFC3
:10FAD000E780C0CB97000000E78000F1AA854808C6
:10FAE00097D0FFFFE780E0B2500801478146A2852A
:10FAF000268597B0FFFFE780C0EE05611723FFFF63
:10FB0000670023601723FFFFE702C35BAA84014459
:10FB10001769FF1F1309C930E14997C0FFFFE7804C
:10FB200060C66344A400014519A833053403832744
:10FB300009003E9583572500639797001105172309
:10FB4000FFFF6700635B0504C9BF032E8500630ADE
:10FB50000E121763FF1F1303634B03230300631588
:10FB6000030029436390061203234E01631503002B
:10FB70001D43639907101723FFFFE702C353C6898C
:10FB8000428A3E89BA8AB684328BAE8B2A84B5E12A
:10FB900003554E0019E501431A851723FFFF67003F
:10FBA0000355A167A98F116763FBE7009700000069
:10FBB000E78080F5814597F0FFFFE78080130844D8
:10FBC000B70700E05841F98F18455CC1B707001F1F
:10FBD000F98F1CC55C4991C7610597E00000E7807B
:10FBE000408BE38A09FA228597900000E78060C67F
:10FBF0005DB7328597C00000E78040430D4349DD83
:10FC00001C44116703D54700A167A98F63FBE70078
:10FC100097000000E78040EF814597F0FFFFE78005
:10FC2000400D0323840093164B01D1828347B30018
:10FC3000035663008588FD8BA305F300FD777D8E59
:10FC4000558EFD76FD16B204F18E83274301C58ED5
:10FC5000231273012313D30023045301230523012B
:10FC6000A3044301BDDF228597B0FFFFE78040CAB0
:10FC7000AA850844B5D1610597D00000E780207FB0
:10FC80008DB71D431A8582801723FFFFE702834348
:10FC90000569AA84AE89328A0144FD5A7D1997C04C
:10FCA000FFFFE780E0A26347A40001451723FFFFA1
:10FCB00067008344D84493171400BA9703D707000A
:10FCC000631F37032390570163070A002685979027
:10FCD0000000E780A0809C449DC383D76700B3F7F2
:10FCE0002701639E3701D288014881470147814639
:10FCF00001468145268597000000E78040E5050420
:10FD000079BF1723FFFFE702E33B79711C103EC464
:10FD1000B7070F003EC61C103EC883C79500AA8ACD
:10FD2000328593F7F707A384F5002E89328497D0A4
:10FD3000FFFFE780C09D93170501C187635AF00656
:10FD4000AA89228597D0FFFFE780609C2A8A4E858A
:10FD5000032B040097B0FFFFE780209839ED83570D
:10FD6000440081440544F11793B71700A303F10041
:10FD700083457100DA872287D2864E86280097E075
:10FD8000FFFFE780A058014781463000CA855685AD
:10FD900097B0FFFFE780E0C4A1679387F7034808A7
:10FDA0003ECC230A810026CE97D0FFFFE780006D6E
:10FDB00045611723FFFF67002334A28513067100F6
:10FDC00097E0FFFFE7802067AA84094455D1528558
:10FDD00097E0FFFFE78020D50D4459D90546D2852D
:10FDE000268597000000E78060EA2A8451B7172330
:10FDF000FFFFE702C32E835507000346270041118A
:10FE00002A842E8532C62EC497E0FFFFE780A0D15A
:10FE100001C93246A245228597000000E78000E72D
:10FE200041011723FFFF6700C32D1723FFFFE702E0
:10FE3000832883C795004111AA8A93F7F707A38403
:10FE4000F5003285AE89328497D0FFFFE780208CA1
:10FE500093170501C1876357F00AC1452A8A228595
:10FE600097C0FFFFE78040712A8D228597D0FFFF62
:10FE7000E780E0892A89228597D0FFFFE780008705
:10FE8000930705F893F7F70F1307E007AA8B637B37
:10FE9000F706228597D0FFFFE78040852A8C2285D0
:10FEA00097D0FFFFE7808084AA8C5285032B040043
:10FEB00097B0FFFFE780608239E983574400231140
:10FEC00001008144F11793B71700A300F100054426
:10FED0000347110083562100938784005685DA88F2
:10FEE00022885286CE8597F0FFFFE780E0A7A167C2
:10FEF000E90748003EC42302810026C697D0FFFFD1
:10FF0000E780C05741011723FFFF6700431E130618
:10FF10001100A28597E0FFFFE780E051AA8409E580
:10FF20002311010009446DB7930521006A8597F0FC
:10FF3000FFFFE78060F12A8441FD8355210093563D
:10FF4000C9001316490185486688E2875E87858A5D
:10FF50005182268597000000E78060BF2A848DBF0C
:10FF60001723FFFFE702231583C7950041112A8B52
:10FF700093F7F707A384F5003285AE89328497C0E2
:10FF8000FFFFE780C07893170501C1876352F00A2D
:10FF90002A8A228597C0FFFFE7806077AA8A228598
:10FFA00097C0FFFFE780A0762A89228597C0FFFFD0
:10FFB000E780C073930705F893F7F70F1307E0077F
:10FFC0002A8C6377F706228597C0FFFFE7800072CF
:10FFD000AA8C228597C0FFFFE78040712A8D528549
:10FFE000832B040097A0FFFFE780206F39E583573C
:10FFF000440085440144F11793B71700A301F100B1
:020000040001F9
:1000000003473100930784005A85DE882688D68608
:100010005286CE8597F0FFFFE78000958D47480018
:100020003EC42302910022C697D0FFFFE78000451F
:1000300041011723FFFF6700830BA28513063100E0
:1000400097E0FFFFE780203F2A84894455D99356E3
:10005000C9001316490185486A88E6876287858A40
:100060005182D68597000000E78060AEAA8449BF20
:100070001723FFFFE70203052A8981440144617ABF
:10008000916A176BFF1F130B6BF897B0FFFFE780A8
:10009000206563C7A40022851723FFFF6700C305FF
:1000A0008327090093991400CE9703D507003307DF
:1000B0004501420741836364570305C103270B00D1
:1000C00019C785453E8597400000E78060E9832792
:1000D00009000504CE972390070085047DB797009B
:1000E0000000E78060A2832709000504CE972390D3
:1000F000070065D5814597F0FFFFE78080BFF1BF1E
:100100001723FFFFE70203FC83C7950041112A8AEA
:1001100093F7F707A384F50032852E89328497C0C0
:10012000FFFFE780C05E93170501C187635AF004A3
:10013000AA89832A040097A0FFFFE780005A31E5CF
:100140008357440085440144F11793B71700A30176
:10015000F10003483100D68752850147CE862686B6
:10016000CA8597D0FFFFE780406BA167F50748007D
:100170003EC42302910022C697D0FFFFE7800030E3
:1001800041011723FFFF670023F7A2851306310003
:1001900097E0FFFFE780202A2A8489445DD997678A
:1001A000FF1F9387A7E69C4381CF044997B0FFFFC9
:1001B000E7800053AA85268597400000E78040DA53
:1001C0001305040197000000E780C0EA22859780AC
:1001D0000000E78000338144ADBF1723FFFFE70233
:1001E00083ED83C795004111AA8A93F7F707A3848B
:1001F000F5003285AE8932842311010097C0FFFFDC
:10020000E780E05093170501C1876354F0062A8AFE
:10021000C145228597C0FFFFE7800036AA8B528533
:10022000032B040097A0FFFFE780204B21E98357B1
:10023000440085440144F11793B71700A300F1006F
:100240000348110003572100DA875685D286268697
:10025000CE8597D0FFFFE780405CA1679387270298
:1002600048003EC42302910022C697D0FFFFE780DA
:10027000E02041011723FFFF670063E7A285130613
:10028000110097E0FFFFE780001B2A8489444DD9C5
:100290009767FF1F938787D798433E8901CF04490B
:1002A00097B0FFFFE780C043AA85268597400000EE
:1002B000E78000CB1305040197000000E78080DB96
:1002C00097B0FFFFE780C04195443DD993052100D9
:1002D0005E8597F0FFFFE78020B7AA8435F11C48C0
:1002E0000357210022852390E70097800000E780D4
:1002F000402183270900A9D703552100974000001A
:10030000E780A0BD35BF1723FFFFE702C3DA83C72D
:1003100095004111AA8A93F7F707A384F500328567
:10032000AE89328497C0FFFFE780603E93170501D6
:10033000C1876351F0062A8A228597C0FFFFE780B4
:10034000003D2A895285032B040097A0FFFFE78018
:10035000C03831E58357440085440144F11793B711
:100360001700A301F10003483100DA8756854A8758
:10037000D2862686CE8597D0FFFFE780004AA16708
:10038000F90748003EC42302910022C697D0FFFF20
:10039000E780C00E41011723FFFF670043D5A28508
:1003A0001306310097E0FFFFE780E0082A848944C4
:1003B0005DD99167CA97C2071167C1831307F7EF29
:1003C0008544E362F7FA9767FF1F938727C4984332
:1003D000BE8B01CF044997B0FFFFE7806030AA854C
:1003E000268597400000E780A0B713050401970019
:1003F0000000E78020C897B0FFFFE780602E95449B
:100400003DD11C482285814423902701978000001C
:10041000E780200F83A70B00B9D74A8597400000DB
:10042000E780A0AB89B71723FFFFE70243CB2A84FD
:100430004105B28497000000E780C0C311C5228542
:1004400097800000E780E00B81460146A685228563
:1004500097800000E780C04E1C4C89C7DC4799C3D9
:10046000228582971723FFFF6700A3C99767FF1FA5
:100470009387C79A9C43014599C3138507018280DE
:100480009767FF1F93878799884382801723FFFF11
:10049000E702E3C49317C600DD8DC2054111C18197
:1004A0002A8432C697C0FFFFE780A0183246228513
:1004B00011829375F60F97C0FFFFE7808015410109
:1004C0001723FFFF6700E3C31723FFFFE70283BF84
:1004D00079713C083ED2B7070C003ED43C083ED6AA
:1004E00083C79500AE842A8993F7F707A384F500A4
:1004F000A16593853504481097A0FFFFE780002988
:10050000C165FD150144176AFF1F130AAAB1930ABA
:10051000400EAE892E8B2EC697B0FFFFE780401F9E
:100520004205931704014181C183B24563E9A702E3
:10053000C167FD176387F500481097C0FFFFE7808C
:10054000400F501001478146A6854A8597A0FFFFBE
:10055000E780204945611723FFFF6700E3B93307B0
:10056000540383270A0BBA9703D6C701630A3601DF
:10057000638A3501481097000000E78060F1DA8552
:10058000050451BFB285EDBF1723FFFFE702A3B2F9
:1005900079717C083EC8B70711003ECA7C083ECC82
:1005A00083C79500AA89328593F7F707A384F500DE
:1005B0002E8997C0FFFFE780801585676378F50473
:1005C000A165AA848905080897A0FFFFE780001CA1
:1005D000268597400000E78060ED133415000A047B
:1005E000A285080897C0FFFFE780A002A68508083B
:1005F00097C0FFFFE780E00325CC01478146100844
:10060000CA854E8597A0FFFFE780A03D456117236F
:10061000FFFF6700C3ADB30754030327CA0ABA97A5
:1006200003D70700631C970003D627006380650586
:10063000080897000000E780A0E5DE8505042EC6C7
:1006400097B0FFFFE780C00D420593170401418179
:10065000C183B245E3E1A7FCC167FD17E38FF5F85D
:10066000080897C0FFFFE780C0FC41BFB285F9B71B
:10067000C165FD150144176AFF1F130AAA9A930A60
:1006800080022E8BAE8B65BF1723FFFFE70223A5E9
:1006900018418347170083460700A207D58FD2076A
:1006A000D1832390F50083472700034717008D452A
:1006B000A207D98F91832310F60097C0FFFFE78030
:1006C00060EA1723FFFF6700C3A31723FFFFE702BA
:1006D000639FC16401441769FF1F1309A99493091B
:1006E0008002FD1497B0FFFFE78080036347A400FA
:1006F00001451723FFFF670023A033053403832739
:10070000C90A3E9583570500E38597FE0504D9BFC6
:100710001723FFFFE702039B2A8AAE89B284B68AB9
:1007200097400000E78080D819E591473E85172360
:10073000FFFF6700639C2A894E8597C00000E78011
:10074000E08E2A84638E0A048D476DD1035705001D
:10075000C547E31D47FD0347F9018546AD47E3174C
:10076000D7FC8347450081CF4146A6855D0597F0BC
:100770000000E780C09E814755D9AD4745BF1309AA
:1007800065012302E500CA85268597100000E780F1
:10079000606231C1A547E38B0AF82302040079B7F0
:1007A00005C183570500E39247F94146A68519051F
:1007B00097F00000E780A09A81472DD99947BDB7EF
:1007C0004E8597000000E78080F02A84954739DD48
:1007D000130955004DBF4146A6852310440123113E
:1007E00034011305190097F00000E780A0992285D5
:1007F00097800000E780A0EA81470DBF1723FFFF25
:10080000E702E38D79717C003ECCB7070A003ECE4B
:100810007C003ED083C79500B2842E8493F7F707FF
:10082000A384F5001306A1002A892C0026859700D1
:100830000000E780A0E5A16528088D0597A0FFFFCF
:10084000E780C0F490408355A100035581008546A0
:1008500097000000E78000ECAA84AA85280897C0CA
:10086000FFFFE78000DB0356A100835581002808C5
:1008700097000000E780C0C1300801478146A2858B
:100880004A8597A0FFFFE780C015854748103ED4F2
:100890002302910202D697D0FFFFE78020BE456178
:1008A0001723FFFF6700E3851723FFFFE70223837A
:1008B00079717C003ECCB7070A003ECE7C003ED06A
:1008C00083C79500B2842E8493F7F707A384F500BD
:1008D0001306A1002A892C00268597000000E780D6
:1008E000E0DAA16528088D0597A0FFFFE78000EA00
:1008F00090408355A1000355810081469700000078
:10090000E78040E1AA84AA85280897C0FFFFE78016
:1009100040D00356A10083558100280897000000AD
:10092000E78000B7300801478146A2854A8597A035
:10093000FFFFE780000B48102302910202D402D689
:1009400097D0FFFFE78080B345611713FFFF670073
:10095000437B1713FFFFE702837897000000E780CF
:1009600060DB1713FFFF6700C3799757FF1F93875B
:10097000274B884382801713FFFFE7024376835794
:1009800025004111AE842A842307B10017F5FFFF2B
:10099000130525466C002316F10097A0FFFFE780A2
:1009A000404691C4228597800000E780E0D6FD573D
:1009B0002310F400130620028145130554009710FC
:1009C000FFFFE780C07441011713FFFF67006373E7
:1009D0001713FFFFE702036F79717C003ECCB70766
:1009E0000A003ECE7C003ED083C79500AA89AE8423
:1009F00093F7F7073285A384F5001306A1002C00B6
:100A000097000000E78080C803558100114497409B
:100A10000000E780A0A915C50355A100014497B0C7
:100A20000000E780A06011CD0357050083578100C7
:100A300045446318F700854597000000E780E0F320
:100A40000144216993053900280897A0FFFFE7803A
:100A5000E0D3A285280897C0FFFFE78080BB03563C
:100A6000A10083558100280897000000E78040A27C
:100A7000300801478146A6854E8597A0FFFFE78095
:100A800040F648104AD42302810202D697D0FFFFD5
:100A9000E780C09E45611713FFFF6700E3651713EA
:100AA000FFFFE70223629757FF1F938727372A84A8
:100AB00088432E8915C5035745038357C401631125
:100AC000F7022326050223180502410597D00000EE
:100AD000E780209C6306090097800000E78060DBC8
:100AE00081449759FF1F9389E953130A800297B0F5
:100AF000FFFFE780E0C263C4A4049757FF1F9387FA
:100B0000A73A9C4399C70355C40197200000E7808A
:100B1000C0BD63070900228597800000E780C0A060
:100B20001306400E814522859710FFFFE780205E67
:100B3000FD57231EF4001713FFFF6700E35B3385A7
:100B4000440383A7C90A3E95035705008357C40190
:100B50006317F700CA8597000000E78000E285046C
:100B600079B71713FFFFE702E35583C795004111DB
:100B7000AA8993F7F707A384F5003285AE8497C05E
:100B8000FFFFE780C0B885676378F5042A8997403E
:100B90000000E780A091014401CD83D704003144D7
:100BA00063882701854597000000E78080EF0144B6
:100BB0004E85A2864A86A68597D0FFFFE780609D76
:100BC000A1679387170448003EC42302810002C630
:100BD00097D0FFFFE780808A41011713FFFF67006E
:100BE000A3511713FFFFE702E34D9757FF1F9387AA
:100BF000E722804329C4014597C00000E780002117
:100C000081470148C1641CDC232E04032320040413
:100C10001759FF1F1309094101449309400EFD14A0
:100C200097B0FFFFE780C0AE634FA400814517F582
:100C3000FFFF1305857F97A0FFFFE780801C171338
:100C4000FFFF6700634B330534038327090B3E9591
:100C50008357C50163879700854597000000E780AB
:100C600040E4050475BF9357050113D78700A3809F
:100C7000F50093170501C183A1832380E50023813B
:100C8000F500A381A50082801713FFFFE70223452B
:100C90002300050083C71500A300F50083C72500C6
:100CA0002301F50083C73500A301F50083C7450084
:100CB0002302F50083C75500A302F50083C7650032
:100CC00093059500A30305002303F5002304050005
:100CD000328597000000E78040F91713FFFF670097
:100CE00043421713FFFFE702E33D4111E9540DCDE5
:100CF00085CD93F9C5FF2E842A89AA84338AA90059
:100D0000B7EA040063189A020D88854411CCB7E74E
:100D100004009C5F82972AC622866C003305390145
:100D200097E00000E7800046268541011713FFFF8A
:100D30006700833C83A78A03910482979317050178
:100D4000C183A183A38EF4FE93570501238FF4FE84
:100D5000A183238EA4FEA38FF4FE6DB763E6D502B4
:100D60001713FFFFE702A337B28741113686BE850E
:100D700036C697E00000E780E040B2464101368584
:100D80001713FFFF6700E33781463685828083872C
:100D900005001387F5003D05FD8793F77708834627
:100DA00007007D158606B58FA300F5006307B70021
:100DB0007D17834717009D83DDB782801713FFFFE0
:100DC000E702E331B7E7040083A7070932872A86E1
:100DD0003A858297133515001713FFFF67006332BA
:100DE00015C181478DC11713FFFFE702432F41460D
:100DF00097E00000E780003985473E851713FFFF25
:100E00006700233081473E8582801DCD1713FFFF89
:100E1000E702E32C414681452A849710FFFFE780D3
:100E2000002F41468145130504039710FFFFE7801B
:100E3000002E0147C1672322040438C87CC8054539
:100E40001713FFFF6700E32B0145828081473DCDEB
:100E5000B5CD1713FFFFE7028328B2842E8913064E
:100E6000800581452A849710FFFFE780402ACA85C4
:100E700024C4268597000000E780C0F641468145DE
:100E800022859710FFFFE78080283044A2852285C5
:100E900097000000E780C0F293040401A285268534
:100EA00097000000E780E0EEA68513050402970096
:100EB0000000E78000EE228597000000E78020F523
:100EC00085473E851713FFFF6700A3233E85828079
:100ED0001713FFFFE702031F4111E9540DCD85CD24
:100EE00093F9C5FF2E842A89AA84338AA900B7EA18
:100EF0000400639844030D88814411CCB7E70400D3
:100F00009C5F82972AC622866C003305390197E0E0
:100F10000000E7802027268541011713FFFF6700A7
:100F2000A31D83A78A039104829793170501C183A8
:100F3000A183A38EF4FE93570501238FF4FEA183B2
:100F4000238EA4FEA38FF4FE6DB765CD1713FFFFAC
:100F5000E7024317B28411E605451713FFFF670048
:100F6000A3192A842E890145EDD93C487848B3E677
:100F7000E700E5D69386F7FFB3B7F6007D17032A9F
:100F80004404BA9734C87CC863050A06C1491305EE
:100F90000A03B38949412295637D3601B2862E86C4
:100FA000A68597000000E780A0DB7C40BE9464C06B
:100FB00065B7CE862E86CE8597000000E78040DAA2
:100FC000C114D2944E9923220404A28793060401EB
:100FD00003C7070003C607038507318FA38FE7FE0A
:100FE000E398F6FE3044A285228597000000E78052
:100FF00020DD2699C1493306994063EC9900A9DCAC
:10100000A686A6851305040397000000E78040D557
:1010100079BF8147B306F4003307F60003470700A2
:1010200083C5060085072D8F2380E600E39437FFF4
:101030003044A285228597000000E78060D8C11463
:101040005DBF014582800DC11713FFFFE702230931
:101050001306800581459710FFFFE780400B05458B
:101060001713FFFF6700E30901458280814749C5E7
:10107000C1C51713FFFFE7028306FC4141462E84DA
:10108000AA846399C70413860501A2878146C145D6
:1010900003C7070003C507038507298F3305D6005B
:1010A000034505008506298FA38FE7FEE392B6FE70
:1010B0003044A285268597000000E78060D0228515
:1010C00097000000E78060F885473E851713FFFF13
:1010D00067002303138507031D8E81452295971012
:1010E000FFFFE780C0027C40130700F813060402EC
:1010F000A2972388E70251BF3E8582801713FFFF26
:10110000E702E3FD6D712E84B284AA859010280059
:10111000368997000000E780A0D309EDD55725A0B8
:1011200050400C40280097000000E78040E27DD549
:10113000FD142104F5F42C004A8597000000E78097
:1011400020F3814761DD3E8551611713FFFF670082
:1011500043FB1713FFFFE70283F841112EC432C689
:101160002C00054697000000E78080F94101171325
:10117000FFFF670003F91713FFFFE70243F60111B2
:101180002A842EC602C802CA02CC02CE97E0000012
:10119000E780C023B2462A86A2850808970000008F
:1011A000E78060FB1375F50F05611713FFFF6700FC
:1011B00043F51713FFFFE70283F27971B2872A84A0
:1011C00021462308B10013051101BE853AC436C675
:1011D00097E00000E78000FBB24693059101368559
:1011E00097000000E78060A82285141035460C089F
:1011F00097000000E78020F62A84224701E9214673
:101200000C103A8597E00000E780C0F72285456121
:101210001713FFFF6700E3EE1713FFFFE70223EC4E
:101220007171AE84AA850A85328497000000E78038
:1012300060BB11C90A86A685228597000000E78059
:1012400020B8814711E1C5473E854D611713FFFF67
:10125000670023EB1713FFFFE70263E51D712A8A7E
:10126000B289BE8435468547130511012E8CB68A96
:101270003A8BC28C468D2308F10097E00000E7808E
:1012800060F010100C085285231F01009700000029
:10129000E780C0F82A843DEDA1476313FD0893075A
:1012A000900591E0E5473546E28513051101139954
:1012B0000A012308F1001359090197E00000E780B3
:1012C00060EC1357890093978A00D98F90080C0817
:1012D0005285231FF10097000000E78020F42A8444
:1012E00015E9A1E49387FA0091831379F9003EC6CA
:1012F000631309004149668B8144C14B854DB24758
:10130000639F970C6A868C0033855C0197E0000030
:10131000E78040E7228525611713FFFF6700E3DCC4
:1013200093079004C9F0A547BDBF8347010509474E
:10133000C14B2308F10083471105A58FA308F100D5
:1013400093872400814463E1FB040147140833863A
:10135000E6008C08B386E400BA95DA9683C60600E8
:1013600083C505000507AD8E2300D600E390E7FE98
:101370004147639CE70490080C08528597000000E1
:10138000E780C0E925D181A0B3069B00BA87100889
:10139000B305F60090083E9603C506000346060016
:1013A00085078506298E2380C500E39277FF998FF4
:1013B00090080C085285BE9497000000E78000E674
:1013C0008947014749D12A84B1B790083E96034620
:1013D00006001408BE962380C600850759BFB24791
:1013E00085046387971481471808B306F7009808A7
:1013F0003E973386F900034707000346060085073A
:10140000318F2380E600E39177FF90080C08528526
:1014100097000000E78080E05DF53546E285130522
:1014200011012308B10197E00000E780A0D51397D0
:1014300004014183939784002183D98F10180C08ED
:101440005285231FF10097000000E78020DD25FD75
:10145000814710183387F9003E960347070003467B
:101460000600B306FB008507318F2380E600E39278
:1014700077FF65A81808B306F70098083E973386EB
:10148000F90003470700034606008507318F2380D4
:10149000E600E3E127FFCA87639E770990080C08FE
:1014A000528597000000E78060D711FD81479800C2
:1014B000B306F700900818103E973E9603470700C2
:1014C000034606008507318F2380E600E39177FF0E
:1014D0003546E285130511012308B10197E00000AC
:1014E000E78040CA139704014183939784002183C6
:1014F000D98F10180C085285231FF10097000000A7
:10150000E780C0D1E31105EC814710183387F9005B
:101510003E960347070003460600B306FB00850717
:10152000318F2380E600E3E227FFC109410BC1BBF5
:10153000814785B79408BE9683C6060018083E9773
:101540002300D700850789BF638006321713FFFF8A
:10155000E702E3B559712A84BE89B28B85473546C7
:10156000130511022E8B468C4289BA8A368A2300D3
:10157000F10297E00000E780E0C010180C1022850F
:101580002317010297000000E78040C96318051285
:10159000A147631FFC069307900563930900E54785
:1015A0003546DA851305110293140A012300F1026E
:1015B000C18097E00000E780E0BC93178A0013D752
:1015C0008400D98F90080C1022852317F102970010
:1015D0000000E780A0C47DE1639209049307FA004C
:1015E000BD88918391E0C144C207C183DE8C814AEA
:1015F0003EC6414DB24763E2FA0E6286B3854B01A7
:10160000881097E00000E78080B54DC93D557DA06A
:1016100093079004E39609F8A54759B78347010556
:101620000947C14C2300F10283471105B3C7F900F4
:10163000A300F10293872900814963E1FC048146FC
:1016400018103306D7008C083387D900B695569703
:101650000347070083C5050085062D8F2300E6009C
:10166000E390D7FE41476390E70690080C1022856F
:1016700097000000E78080BA35D189A0B3863A018F
:10168000BA871010B305F60090083E9603C5060011
:101690000346060085078506298E2380C500E39250
:1016A00097FF3387EC4090080C102285BA99970079
:1016B0000000E780A0B68947014741D16561171353
:1016C000FFFF670083A290083E96034606001410B1
:1016D000BE962380C600850779B7B247850A9399DD
:1016E0000A01939D8A0093D909016391570F854799
:1016F0003546DA85130511022300F10293D98900DA
:1017000097E00000E78000A8B3ED3D0190000C10C9
:1017100022852317B10397000000E78020B059FD10
:101720008147A68963EA970626860C084A8597E0D2
:101730000000E78020A581471810B306F7001008C5
:1017400098083E973E960347070003460600850724
:10175000318F2380E600E3E197FE639FA90590089F
:101760000C10228597000000E78040AB21F98147EB
:101770009810B306F700900818183E973E96034756
:101780000700034606008507318F2380E600E391BA
:10179000A7FF4109C10CB9BD18089000B306F700B6
:1017A0003E963387FC000347070003460600850783
:1017B000318F2380E600B5B798084E97034707009E
:1017C0001C10CE972380E700850941BF8547354629
:1017D000DA85130511022300F10293D9890097E0FD
:1017E0000000E780209AB3ED3D0190000C102285A7
:1017F0002317B10397000000E78040A2E31005EC37
:10180000814718089000B306F7003E963387FC0026
:1018100003470700034606008507318F2380E60053
:10182000E391A7FF41460C084A8597E00000E78056
:10183000609581471810B306F700100898083E9786
:101840003E9603470700034606008507318F238035
:10185000E600E391A7FF90080C1022859700000096
:10186000E780C09B1DD599BD7D5582801713FFFF72
:10187000E702E38601112A842E85930551003289FF
:1018800002C002C202C402C69304740097F0FFFFB4
:10189000E780A03D1D46A6851305910097E0000056
:1018A000E780408E10088A854A8597000000E7800F
:1018B000E09619ED93071400180883C60700034645
:1018C000070085070507B18EA38FD7FEE397F4FEC7
:1018D00005611713FFFF6700C3821703FFFFE702CD
:1018E000637E2E848C414111AA8983871500328939
:1018F000914463D30700A1449757FF1F938747A9DB
:101900009C43A1C7C1CA8D472310F10083C725009E
:101910004A852301F10083C73500A301F10083C785
:1019200045002302F10083C75500A302F10083C7DD
:10193000650093059100A30301002303F100230434
:10194000010097F0FFFFE78040320C404A860A858D
:1019500097F0FFFFE780803303280400835644009C
:10196000A6881D0881470147E51642868A854E856F
:1019700097000000E780408E2A8919E5A685228518
:1019800097B0FFFFE780A0C24A8541011703FFFF20
:10199000670083764A860A8597F0FFFFE780002F6D
:1019A0006DB71703FFFFE702E3712E848C414111ED
:1019B000AA89838715003289914463D30700A14423
:1019C0009757FF1F9387C79C9C43A1C7C1C68D47EC
:1019D0002310F10083C725004A852301F10083C746
:1019E0003500A301F10083C745002302F10083C73E
:1019F0005500A302F10083C7650093059100A3037E
:101A000001002303F1002304010097F0FFFFE780AA
:101A1000C0250C404A860A8597F0FFFFE780002723
:101A200083564400032804008A85858EC2061D085B
:101A3000C1822312D400A68881470147E516428659
:101A40004E8597000000E78060B041011703FFFF5B
:101A50006700836A4A860A8597F0FFFFE7800023C4
:101A60004DBF1703FFFFE7028367B335B0000111D5
:101A700085052A891315F601336515012308B10080
:101A80009305110136843AC632C03EC442C297F073
:101A9000FFFFE780801DA2471248425593D687007A
:101AA000230BF1009305910193578800A30AD100FD
:101AB000A30BF100230C010197F0FFFFE780E01A70
:101AC0003247024603280400B337E000835644003F
:101AD0009207914411C2A1444A85A68842860C0807
:101AE00097F0FFFFE78040772A8919E5A6852285D0
:101AF00097B0FFFFE780A0AB4A8505611703FFFFA2
:101B0000670023601703FFFFE702C35B01113EC6B6
:101B10008647B335B0008505AA891315F6015D8D9A
:101B20002308B1009305110136843A89B28442C476
:101B300046C297F0FFFFE7804013224892481645BF
:101B400093578800A30AF1009305910193D7880069
:101B5000230B0101A30BF100230C110197F0FFFFF0
:101B6000E780A0103247104083564400B337E000AE
:101B7000920703280900914891C0A1480C084E859E
:101B800097000000E780809CAA8401E98355440007
:101B90004A8597B0FFFFE78080A12685056117037E
:101BA000FFFF67006355AA959307F00F1707010021
:101BB000130747676317B50013C5F7FF1375F50FD4
:101BC000828005058346F5FFB58FBA9783C7070066
:101BD000D5B70357450014419307F00F17060100CE
:101BE00013064664369742074183139506014181E7
:101BF000631BE500AD8FB29703C50700130515F30E
:101C0000133515008280850603C5F6FFA98FB297AC
:101C100083C70700D9BF1703FFFFE702434CB28712
:101C200036842E86BA86AA853E85BA8497F0FFFF51
:101C3000E7806052634F0500228597D00000E7805F
:101C4000E0782A86A686A285268597F0FFFFE780A2
:101C500080501703FFFF6700C34A1703FFFFE70227
:101C600063465D712A8BAE8A17050100130505597D
:101C70002C00B284368ABA893E8997F0FFFFE7804C
:101C8000C04F2A845DE134104146DA85280097F080
:101C9000FFFFE780404C2A8449E98547A303F10010
:101CA000A6C2930771002408BEC4A68685470D46C8
:101CB0002C18281002DC02DED6C0BEC697F0FFFF4B
:101CC000E78000442A8435E183477102A6860D46E9
:101CD00093F7F7072300FA00C1473EDE2C18894727
:101CE000281026DCA303F10097F0FFFFE7804041B6
:101CF0002A8405ED4146A6854E8597D00000E780F1
:101D000060488D47A6860D462C182810A303F100C5
:101D100097F0FFFFE780C03E2A8401E94146A6858F
:101D20004A8597D00000E780E0452285616117036E
:101D3000FFFF6700633C1703FFFFE702433A97F793
:101D400000009387E7A1984383C7470079712A89E8
:101D5000AE84170501001305E54A0C083AC42306B2
:101D6000F10097F0FFFFE78040412A8405ED141051
:101D70004146CA85080897F0FFFFE780C03D2A84E6
:101D800015E1140815462C00081097F0FFFFE780B6
:101D9000803C2A8401E921462C08268597D0000042
:101DA000E780403E228545611703FFFF67006335EA
:101DB0001703FFFFE702A33297F700009387479AC4
:101DC0009C477971AA842E841705010013050544E8
:101DD0000C083EC697F0FFFFE780203A0DE914108B
:101DE0004146A685080897F0FFFFE780C03605E169
:101DF000140811466C00081097F0FFFFE780A0352B
:101E000019E58347F10193F7F7032300F4004561D7
:101E10001703FFFF6700E32E1703FFFFE702232CE2
:101E20003688A14881470147E54697F0FFFFE780E4
:101E3000A0421703FFFF6700C32C1703FFFFE70251
:101E4000032A3688A14881470147E54697F0FFFFFE
:101E5000E780C06F1703FFFF6700A32A1703FFFF88
:101E6000E702E32701112A842E850C0832C697F079
:101E7000FFFFE780803009ED324797060100938627
:101E800066371008C145228597000000E780E0D83A
:101E900005611703FFFF6700C3261703FFFFE70273
:101EA00003244111C1472EC032C48A8509463EC26F
:101EB0003EC697F0FFFFE780A02441011703FFFF14
:101EC000670023241703FFFFE70263214111AE8659
:101ED00013061009AA850A8502C002C202C402C6FE
:101EE00097F0FFFFE780202741011703FFFF6700FE
:101EF00043211703FFFFE702831E32879706010085
:101F0000938646312E869305000297000000E780F5
:101F1000C0D01703FFFF6700C31E1703FFFFE702D0
:101F2000031C7971C1472ACC2ED032D42C080D461F
:101F300028003ECE3ED23ED602C402C602C802CA25
:101F400097F0FFFFE780C01B45611703FFFF6700A5
:101F5000431B1703FFFFE70283180111AA842E8495
:101F6000170501001305852B8A8597F0FFFFE78091
:101F7000C02015E514084146A6850A8597F0FFFFA5
:101F8000E780601D09ED8347E1010347F101A207E6
:101F9000D98FCA07C9836177D98F2310F4000561EF
:101FA0001703FFFF6700E31515CD1703FFFFE702D7
:101FB00003139747FF1F938727EB90439745FF1F16
:101FC0009385C5EA1745FF1F130505E697D0000066
:101FD000E78000C51745FF1F130505E51703FFFF41
:101FE000670023121745FF1F130505E482808DCD7E
:101FF0001703FFFFE702A30E9747FF1F9387C7E66C
:10200000944301112E840A869745FF1F938505E6A8
:1020100097D00000E78040C60A850294014505611B
:102020001703FFFF6700E30D7D5582801703FFFF55
:10203000E702E30A97D00000E78080D19747FF1FAF
:1020400023A4A7E217F5FFFF1305E5C997B0000029
:10205000E780C0741703FFFF6700A30A1747FF1F3D
:102060001307C7E29317150008433E95FD57231049
:10207000F50082801703FFFFE70263062A84084009
:1020800009E51703FFFF6700C3071C4158401CC048
:102090006313E5005CC08347550023200500F99BCE
:1020A000A302F50097A0FFFFE780E07CC9BF1703FC
:1020B000FFFFE70223019747FF1F938727DF98431E
:1020C0002A8411CB8347350093F7070289C703554C
:1020D0000500894502971305440197B00000E78089
:1020E000403B835504000355E40097300000E7802F
:1020F000A00C485819C597A0FFFFE780C077232A96
:1021000004021305840397000000E780E0F6814491
:10211000B1499790FFFFE780E06A63CBA402834751
:1021200034002320040493F727FCA301F4000048A3
:102130009790FFFFE780006A1316150081452285FE
:102140009700FFFFE780A0FC1703FFFF6700C3FABB
:10215000B38734030329040385043E994A85970015
:102160000000E78060F12304090065B7834735006C
:1021700093F7070299E3014582808357E500E39CCA
:10218000B7FEC167FD176316F60005458280054559
:1021900099A81703FFFFE70283F493170601C1878D
:1021A000B2842A8401496359F002835705009DCB0C
:1021B00001456367F600034584003E953325A6007C
:1021C0001375F50F0DA01C4813171900BA9783D784
:1021D0000700E38E97FA05099790FFFFE780805F7D
:1021E000E343A9FE01451703FFFF670083F11703CF
:1021F000FFFFE70223EDAE89AA849790FFFFE780F7
:1022000020532A8497D0FFFFE780A02EAA8601479B
:102210001306840197050000938585E41745FF1F89
:10222000130505C79790FFFFE780A0192A8925C9E4
:102230008C441304C50022859E0593F5050897A0DC
:10224000FFFFE780003DCC4083877400E18163DDC0
:10225000070493E50508228597A0FFFFE780603B10
:102260000D4693854400228597A0FFFFE7808037C5
:1022700083D50400228597A0FFFFE780A03E83D589
:102280002400228597A0FFFFE780C03D03D64900C8
:1022900083A50900228597A0FFFFE780A0344A8527
:1022A0001703FFFF670043E593F5F5076DB71703C5
:1022B000FFFFE702C3E201112A84328532C697A0EC
:1022C000FFFFE780A0289780FFFFE78080318357DA
:1022D00004001747FF1F1307E7D43246231BF10002
:1022E000930700F8A30DF1001C471843231AA1001F
:1022F0008983858BB307F740B28548083ECE231CFF
:102300000100230D010097000000E78080EE0561C9
:102310001703FFFF6700E3DE1703FFFFE70283DA1F
:10232000004101453DC49304C40026853289AE892D
:1023300097A0FFFFE780802595452A8A2685035BC5
:10234000040197A0FFFFE780E021268597A0FFFF0B
:10235000E780203F8D45AA8A268597A0FFFFE7806A
:102360006020268597A0FFFFE780A03D5C48420AD9
:10237000135A0A01D2975CC42318640181476398F9
:102380003A0146054D81330625419337160013F572
:10239000F70F1703FFFF670023D61703FFFFE702BE
:1023A00083D189692A8BAE8B328AB68A81440144F3
:1023B000314CFD199790FFFFE780C04063CDA4002A
:1023C0009790FFFFE7800043018D33B5AA00170304
:1023D000FFFF6700C3D13389840383270B003E9935
:1023E00063170A008347890085043E94E1B70356CA
:1023F0000A00DE854A8533F6C90097000000E780B1
:10240000E0F16DD10545E1B71703FFFFE70223CDEA
:1024100001112A847C000355E5003ECAB707070076
:102420003ECC7C003ECE97200000E78020082A8921
:102430008545480897A0FFFFE780E039994548089F
:1024400097A0FFFFE780A016AA844A859720000086
:10245000E780A0082380A4009747FF1F938787BCCD
:102460009C434166130606F09396870113D78701B4
:10247000558F93D68700F18E558FA207B706FF00C0
:10248000F58FD98F11462C00138514003EC497D0C8
:102490000000E78020CF5008A382040089452285F0
:1024A00097000000E780E0E019C9AA8513058403BE
:1024B00097A0FFFFE780A0323C4085073CC0056144
:1024C0001703FFFF6700E3C31703FFFFE70223C102
:1024D0009790FFFFE78000322A8405049790FFFF62
:1024E000E78040303305A402F14791453305F502FA
:1024F00097200000E78020BA11E565551703FFFF1C
:10250000670023C09747FF1F23AAA7989790FFFF54
:10251000E780402E2A8405049790FFFFE780802CF7
:102520003305A4028945060597200000E780A0B680
:1025300069D59747FF1F23ABA7949790FFFFE780CC
:10254000602B2A8405049790FFFFE780A0293304BD
:10255000A4029747FF1F239D87929790FFFFE78074
:1025600060292A849790FFFFE780C0279307140013
:102570003385A7029747FF1F239DA7909707010068
:102580009387878D1747FF1F2328F7900145BDB715
:102590001703FFFFE70203B3AA842E89014497497A
:1025A000FF1F938929A8130A80069790FFFFE780F1
:1025B00060236347A40001451703FFFF6700C3B30F
:1025C0003305440383A709024A86A6853E959700F2
:1025D0000000E780E0B919E10504C1BF0545E9BF86
:1025E0001703FFFFE70223ADAA8A2E8BB28B368C2E
:1025F0003A8A814401448149974CFF1F938C8CA2F5
:10260000130D80069790FFFFE780C01D63C9A400EB
:1026100011E085494E851703FFFF670043AD3389FD
:10262000A40383A70C025E86D6853E994A8597004F
:102630000000E780E0B31DC19790FFFFE780801B9B
:102640000544636D4501D2866286DA851305090368
:1026500097000000E780A0D411C1854985045DB7CB
:102660001703FFFFE70203A6C16441112A89014451
:102670009749FF1F9389099B130A8006FD1436C6EC
:1026800032C42EC29790FFFFE780C01592452246C4
:10269000B2466348A400014541011703FFFF6700EC
:1026A000A3A53305440383A709023E9509C68347C2
:1026B0003500C18B9DC791C68347350093F707024C
:1026C0008DC3630699008357E500639C2701035778
:1026D000050001CB63E7E50083478500BA97E3CDAA
:1026E000F5FA050469BF1703FFFFE702A39DC16464
:1026F0002A8901449749FF1F9389C992130A8006CA
:10270000FD149790FFFFE780E00D6346A4001703D8
:10271000FFFF6700639E3305440383A709023E95CC
:102720008357E500638A9700630499006396270145
:1027300097000000E780E0970504E1B71703FFFF6B
:10274000E702E39689692A8AAE8A328BB68B814486
:10275000174CFF1F130C0C8D930C8006314DFD1987
:102760009790FFFFE780000863C6A4001703FFFFF0
:102770006700A3973389940383270C028355CA010A
:102780005A863E994A8597000000E780609E31C1D5
:10279000814D15A03384AD038327090303D60B00B5
:1027A000D68533F6C9003E94228597000000E78065
:1027B000E0B609E9850D9790FFFFE780A000E3CB25
:1027C000ADFC01A8228597000000E780E08A230481
:1027D0000400850471B71703FFFFE702C38D416949
:1027E000AA8A014A174BFF1F130BCB837D19C14BDC
:1027F000054C9790FFFFE780E0FE6346AA001703B1
:10280000FFFF6700C38E93098006B3073A0383294D
:102810000B02BE9983D7E900638E270163842A01E6
:10282000639A570103A4890301E84E8597000000CD
:10283000E780C0BD050A75BF835704016399770916
:102840009304C400268597A0FFFFE78020D4854528
:102850002A8D2685835C040197A0FFFFE78080D046
:10286000268597A0FFFFE78060E8620561856359D0
:1028700005048D45268597A0FFFFE780A0CE8945FA
:10288000268597A0FFFFE780E0CD8945268597A0A4
:10289000FFFFE78020CD8545268597A0FFFFE780D5
:1028A000A0CD83470500094793F7F707639AE70030
:1028B0009945268597A0FFFFE78000CCA3028501FC
:1028C0004848337D2D01231894016A9548C400407F
:1028D000A1BF1703FFFFE702838037E404008327CB
:1028E000041D82979737FF1F83C7C7601715FF1F07
:1028F0001305C5C3A300F5008327441C82978327D3
:10290000841C81461306F00F81450145829717F319
:10291000FEFF6700037F1737FF1F1307A74D1843FC
:102920009735FF1F83C5055D9737FF1F9387075BAB
:1029300083468703034697036397D5009737FF1FA6
:10294000238AC75A828083C587010347A703631779
:10295000B6009737FF1F238FE758828003C6870191
:102960006317C7009737FF1F2386D758828083C617
:102970008701130750026319D700930760021737C6
:10298000FF1F2309F756828083C687011306600262
:102990006315D60093077002DDB783C7870155BF63
:1029A0009737FF1F93878753D44B0947638DE608FA
:1029B00017F3FEFFE702A3721739FF1F1309494FF0
:1029C0003E8483470900918B9DCFB7E4040083A721
:1029D000041D829783A7441C1735FF1F1305C54D9F
:1029E000829783A7841C81461736FF1F0346C64E75
:1029F00081450145829721C583470900ED9B173723
:102A0000FF1F2307F74A8347040093F7F70F85CB8F
:102A100091471737FF1F232DF74C97000000E780E1
:102A200080EB97000000E78040EFB7E70400BC4F61
:102A3000414691451735FF1F0345C54A829717F355
:102A4000FEFF6700036C828017F3FEFFE702236935
:102A50008D4741116306F504C5476308F5028547B4
:102A60006310F5029737FF1F2388A748B7E70400D4
:102A7000BC4B930500101735FF1F0345A5468297F1
:102A8000410117F3FEFF6700C36785471737FF1F34
:102A90002304F746B7E70400BC4B93050020E1BFD1
:102AA0009737FF1F93878743D44B1147638DE60009
:102AB000B7E7040083A7071D8297B7E70400BC4B64
:102AC000930500044DBF05491737FF1F23222743F5
:102AD00083C7070032C62E8493F7F70FD5D3B7E428
:102AE000040083A7041D7D141374F40F8297E3760A
:102AF00089FCB245994703C61500E3F0C7FCFC44C6
:102B000009061735FF1F1305653F8297BC489305DB
:102B100000081735FF1F0345E53C829779BF17F37F
:102B2000FEFFE702C35B1737FF1F1307273B404732
:102B3000184B1C409736FF1F23A8F63A6316E40093
:102B40001737FF1F2324F73A130584FE9790FFFFE2
:102B5000E78020A7035564FF9780FFFFE780A06F01
:102B600097A0FFFFE78020D117F3FEFF67006359AE
:102B700017F3FEFFE702A3569737FF1F9387073629
:102B8000D84BDC4789C797000000E78080F985476C
:102B90001737FF1F232EF7349737FF1F938787259B
:102BA0009C43930500021735FF1F0345A53383C7D8
:102BB00087031737FF1F230FF732B7E70400BC4B1B
:102BC000829717F3FEFF6700C3539737FF1F23A9B0
:102BD000A730828017F3FEFFE702C34E37E40400FC
:102BE0007C4CA1451735FF1F0345C52F82977C48B4
:102BF000A1451735FF1F0345E52E9734FF1F93842A
